:020000040000FA
:040000006FD00400B9
:101000006F10404F00000000000000009020002002
:10101000DC270020A9BDF9F5A02800200000000071
:1010200000000000A0280020902000200000000008
:101030000000000090200020000000009020002010
:10104000000000009020002090200020707300001D
:10105000902000209020002064340020A02900204F
:10106000000000009020002090200020382900205F
:1010700090200020062900209020002090200020B1
:101080009020002090200020902000209020002020
:101090009020002001A04111B7170040985F3AC688
:1010A000945F3247E39CE6FE324541018280411164
:1010B000814601468145114506C697100000E7802C
:1010C00040C3B727004011472383E780B7F700E00C
:1010D00003A707D16D9B23A8E7D003A707D15D9B8A
:1010E00023A8E7D07300501001000100B240410175
:1010F00082800111814601468145114506CE971037
:101100000000E78000BFB727004011472383E78036
:10111000B717004083C6E70203C5E704130780083A
:1011200093F6C60F1365350093E6160073360780F5
:101130001376860832C001000100930570052380F4
:10114000B704130680FA2380C7040100010023823C
:101150000702238007040248732808800100010069
:10116000733807801378880842C201000100238089
:10117000B7042380C704010001002387D702238717
:10118000A704238007049246F3A60680010001000D
:10119000F336078093F6860836C4010001002380E9
:1011A000B7042380C7040100010083C6B70493E697
:1011B0000602A385D70423800704A246F3A606806F
:1011C00001000100B7F600E003A506D11365450054
:1011D00023A8A6D003A506D15D9923A8A6D07300A5
:1011E00050100100010073370780137787083AC653
:1011F000010001002380B7042380C704010001001F
:1012000003C7B7041377F70DA385E704238007040A
:10121000B247F3A7078001000100F2400561828018
:101220003971B7F5070022DC81462A843010E105C8
:10123000194506DE02D42316010297100000E7804C
:1012400040ABB717004083C6E7041307800893E656
:101250003600733607801376860832C40100010019
:10126000930570052380B704130680FA2380C70412
:101270000100010023820702238007042245732511
:1012800005800100010073350780137585082AC6A3
:10129000010001002380B7042380C704010001007E
:1012A0002387D70423800704B246F3A606800100F3
:1012B0000100F336078093F6860836C80100010066
:1012C0002380B7042380C7040100010003D507026F
:1012D000F176FD16E98E2390D70223800704C246DB
:1012E000F3A606800100010037F500E0832605D152
:1012F00093E646002328D5D083D6070265751105ED
:1013000093F60660C18EC98EC206C182733507800E
:10131000137585082ACA010001002380B7042380C1
:10132000C7040100010003C5F70013650504A38786
:10133000A7002390D70223800704D246F3A6068095
:10134000010001001165618D1DE973370780137776
:1013500087083ACC010001002380B7042380C7042A
:101360000100010003C7B70413670702A385E70460
:1013700023800704E247F3A707800100010037F745
:1013800000E0832707D1DD9B2328F7D0730050109E
:101390000100010013078008F337078093F78708DF
:1013A0003ECE01000100B717004093057005238071
:1013B000B704130680FA2380C7040100010083D616
:1013C0000702C606C5822390D70223800704F2468F
:1013D000F3A6068001000100F336078093F6860825
:1013E00036D0010001002380B7042380C704010028
:1013F000010003D80702F176FD16B3F6060123902B
:10140000D702238007048256F3A60680010001005C
:1014100021E173370780137787083AD20100010072
:101420002380B7042380C7040100010003C7B70469
:101430001377F70DA385E704238007049257F3A7DA
:10144000078001000100514597000000E780E0415E
:10145000F250625421618280397152D481462A8AC5
:1014600001468145114522DC26DA06DE4AD84ED6F1
:101470003714004097100000E780A0878347E402FC
:101480000347E4049304800893F7C70F13673700FA
:1014900093E71700F3B6048093F6860836C601007A
:1014A00001009309700523003405130980FA230015
:1014B0002405010001002302040223000404B246B3
:1014C000F3A6068001000100F3B6048093F68608B7
:1014D00036C8010001002300340523002405010063
:1014E00001002307F4022307E40423000404C24795
:1014F000F3A70780010001001305500297000000C8
:10150000E780400EB7F700E003A707D11367470055
:1015100023A8E7D073B70480137787083ACA01007D
:1015200001002300340523002405010001000347C6
:10153000F40013670704A307E400230004045247E0
:10154000732707800100010073B7048013778708B1
:101550003ACC0100010023003405230024050100DA
:1015600001002167336AEA002310440323000404C6
:101570006247732707800100010003A707D15D9B25
:1015800023A8E7D0730050100100010081460146F6
:101590008145114597000000E780A075F3B40480F1
:1015A00093F4840826CE01000100230034052300B3
:1015B0002405010001008347640493E71700230317
:1015C000F40423000404F247F3A70780010001009C
:1015D000F2506254D2544259B259225A2161828047
:1015E000011113078008F337078093F787083EC27D
:1015F00001000100B7170040930570052380B70470
:10160000130680FA2380C7040100010083C6B704D3
:1016100093F6F60DA385D704238007049246F3A61C
:1016200006800100010093760502D5CEF3360780CF
:1016300093F6860836C4010001002380B704238096
:10164000C70401000100B70614007D89558D88C7C5
:10165000010001000100010023800704A246F3A657
:1016600006800100010073370780137787083AC6A8
:10167000010001002380B7042380C704010001009A
:10168000010001003727004093061005A303D7800F
:1016900023800704B247F3A70780010001009307E6
:1016A0008008F3B7078093F787083ECE010001005A
:1016B000B7170040130770052380E704130780FA6B
:1016C0002380E7040100010003C7B704136707087C
:1016D000A385E70423800704F247F3A707800100EE
:1016E00001000561828093760504BDC6F33607804C
:1016F00093F6860836C8010001002380B7042380D2
:10170000C70401000100B7061400938606047D8912
:10171000558D88C7010001000100010023800704E6
:10172000C246F3A6068001000100733707801377D5
:1017300087083ACA010001002380B7042380C70448
:10174000010001003727004093062005A303D7803E
:1017500023800704D24781B7733707801377870840
:101760003ACC010001002380B7042380C7040100A4
:10177000010098471367070C98C723800704E247C6
:1017800019BF0111814601468145114506CE9700DA
:101790000000E780005693078008F3B7078093F7AF
:1017A00087083EC601000100B71700401307700507
:1017B0002380E704130780FA2380E7040100010077
:1017C00003C76704136717002383E7042380070414
:1017D000B247F3A7078001000100F2400561828053
:1017E0004111814601468145114597000000E7807F
:1017F000405013078008F337078093F787083EC4EB
:1018000001000100B7170040130670052380C704CC
:10181000930680FA2380D70401000100FD5523962A
:10182000B70223800704A245F3A50580010001004B
:1018300073370780137787083AC6010001002380B9
:10184000C7042380D7040100010003C7670413679E
:1018500017002383E70423800704B247F3A7078018
:101860000100010001A0BD473305F50201007D150F
:1018700075FD8280411122C426C206C6AA84014495
:1018800063179400B24022449244410182800504CF
:101890001305803E420497000000E78000FD418070
:1018A000C5B700009305000273A045808245739080
:1018B000153492402242B2424243D2436244F2443F
:1018C000025592552256B2564257D2576258F25894
:1018D00006499649264AB64A464BD64B664CF64CC4
:1018E000065D965D265EB65E465FD65F0961730053
:1018F00020304111B7170040985F3AC6945F3247D5
:10190000E39CE6FE324541018280B7170040130791
:1019100000032388E7028547171700002320F744B8
:1019200073002030411122C406C63704002097609E
:1019300000E0E780200E1C408297D5BFB7370040FB
:1019400003C7470091463D8B6309D700994663144E
:10195000D70083C757407300203017370000034774
:1019600027299306700C63ECE602930617001736DE
:101970000000230FD62683C6870097370000938781
:10198000A71ABA972380D700B7E70400BC4F0946CF
:101990008945171500000345A5F482976DBF83C7DD
:1019A0008700DDB7B787004003C76700098B63096D
:1019B000071003C777009306000313770703630D2F
:1019C000D708173800000348785E17360000130662
:1019D000265D0547B30606012380E60083C5770030
:1019E000173700001307475C429793F5F50F230064
:1019F000B70003C58700973500009385A55AC295A7
:101A00001375F50F2380A500034707008945137759
:101A1000F703630CB70C63E7E50A6306071A85450D
:101A2000630CB7129737000083C757583307F60087
:101A3000034707001377F70F19CB850793F7F70FC5
:101A40000D476363F71A17370000A301F756B787EE
:101A5000004009472383E700B787004083C777002A
:101A6000E207E18763DE07049737000083C7175456
:101A7000173700001307C7523E9785462300D7004B
:101A800017370000130747523E97930600032300C1
:101A9000D700173700001307E7503E97A146850788
:101AA0002300D70093F7F70F0D476364F714173738
:101AB0000000A30DF74EB787004009472383E700D6
:101AC00073002030930610026300D70E93062002A5
:101AD0006305D70693060002E316D7F403C727026F
:101AE0001377C70F13672700D5A803C767001377BD
:101AF000070465CB03C7A702173800001308C82BDB
:101B00001735000013050523134707082385E7024F
:101B100003C7A7021377370F136787002385E702F0
:101B2000814713070004B305F5008C41B306F800A4
:101B300091078CC2E399E7FEF5B503C7A7021347E7
:101B400007042385E70203C7A7021377C70F1367AC
:101B500027002385E702F9B503C767001377070459
:101B600049C303C76702173800001308A8181735C0
:101B700000001305E50F134707082383E70203C797
:101B800067021377370F136787002383E7028147C4
:101B900013070004B305F5008C41B306F800910764
:101BA0008CC2E399E7FEBDBD03C767021347070474
:101BB0002383E70203C767021377C70F1367270062
:101BC0002383E70285B503C767001377070411CBAA
:101BD00003C727021377370F136787002381E702B4
:101BE00091B5238006003DBD97370000A380073CD8
:101BF000B9BD97370000A38B073A75BD2303048056
:101C000015472303E48001002302A4808280830718
:101C10006480E3CE07FE2303048082808307648010
:101C2000E3CE07FE03454480828083076480E3CED1
:101C300007FE2302A4808280411126C44AC24EC0FE
:101C400006C61377F50BAD47AA892E899544630C18
:101C5000F700194597000000E78080FA9700000020
:101C6000E78020FB8D444E8597000000E78040F917
:101C7000FD59FD1463983401B240A24412498249CF
:101C800041018280135509011375F50F970000007B
:101C9000E780E0F92209F1BF011126CC06CEB70496
:101CA000080097000000E780C0F615459700000087
:101CB000E78000F597000000E78080F697000000BD
:101CC000E78000F62AC697000000E78080F43245DE
:101CD0009377150089EB136515001375F50FF24026
:101CE000E24405618280FD14E9F00145CDBF397100
:101CF00026DC4ADA4ED852D656D45AD25ED006DE08
:101D000062CE66CCB7E700E07D5783AA070022C603
:101D100003AA470023A0E71823A2E718B71700403B
:101D2000130770052380E704130780FA2380E70474
:101D300083C74704930B75FFB684E20793FBFB0F41
:101D40008546AA892E8B328937240040E1870157C6
:101D500063FA76016308D50089461307000263130E
:101D6000D5000157D98F93F7F70FB71C0040238296
:101D7000FC0411472303E4801305F00F97000000D3
:101D8000E78000E8094C97000000E78080E8636581
:101D90007C15B7050700DA9537870700795563FE8C
:101DA000E504B3879500636AF704370B0800A94779
:101DB00033EB65016395F90881E8814497000000E1
:101DC000E78020E5268515A8DA85094597000000FB
:101DD000E780C0E605090345F9FFFD14050B9700F0
:101DE0000000E780C0E481C49377FB0FE5F797001C
:101DF0000000E780A0EA69F17D55B717004013079E
:101E000070052380E704130780FA2380E70403C7E3
:101E10004704418B2382E704F250B7E700E023A098
:101E2000571123A24711E25432445259C259325A2F
:101E3000A25A125B825B724CE24C21618280A54700
:101E4000639BF90685691309F00FB3069900B37413
:101E50002B01B6941349F9FFB3749900856B33795C
:101E60006901416B9387F9FFB3F7270199E363FC9D
:101E7000340193D94900C147E3E637FF3DBF056907
:101E8000C1697D19D9B71305800D638869011305F0
:101E900000026384790113051008CA8597000000C9
:101EA000E780C0D997000000E78040DF31D54E9928
:101EB000B38434416DBFDA852D4597000000E7807B
:101EC000E0D7CA94E30B99EE050997000000E7807C
:101ED00020D5A30FA9FEFDB79387F9FF93F7F70F5E
:101EE000636DFC0C83C71C04130730086315F706E9
:101EF000370708006361EB06B3079B00B7061000C5
:101F000063FBD704334BEB0089476399F90689805B
:101F1000D549E38404EADA85094597000000E780A3
:101F2000E0D111090327C9FF91472320E48003076B
:101F30006480E34E07FE23033481FD17EDFBFD149F
:101F4000110B81C49377FB0FE9FF97000000E78036
:101F5000E0D461F155B5B717004003C75704B70780
:101F600008001377070219E3B78707007955E3766E
:101F7000FBE833079B00E3F9E7F841B58547E380C9
:101F8000F9F0DA852D4597000000E78020CB938992
:101F9000F4FFE38404E297000000E78060C893F751
:101FA000390091EB83260480032709009307490039
:101FB000E396E6E03E89CE84D9BFB5476399F90040
:101FC0001305900B97000000E78080C3FDB3B14775
:101FD0001305B00AE388F9FE99476397F904B7053A
:101FE0000800B365BB002D4597000000E78000C5E1
:101FF00081448D4BA14997000000E78060C2639641
:102000007401832704802320F9008504E39534FFBD
:102010008327048013172B01635507002312F9004F
:1020200069BB2322F90051BB9D47639FF90281459B
:102030001305B00497000000E78040C0BD44232092
:10204000090023220900FD5997000000E78040BDE8
:1020500093F77400CA9703C70700FD14398D2380D6
:10206000A700E39334FF91BBA1476397F90697005C
:102070000000E780A0C28144630D0B008D479304EC
:10208000C0036308FB009304000563048B01930401
:1020900040041375C507E30295D219459700000067
:1020A000E78000B697000000E780A0B605459700DE
:1020B0000000E780E0B4268597000000E78020B7A5
:1020C000094597000000E78080B697000000E78090
:1020D000E0BCE31405CE0DB39147639FF9001305EF
:1020E000600697000000E780A0B197000000E7803D
:1020F00040B213059009F9B5E38109CCF1547DB9DB
:10210000BD6601471736000013068607938606A6AC
:1021100085458347060093F7F70F91C38280050733
:10212000E3F9E6FE97370000238CB704DDB77D1690
:102130006206618693178601E18763D40700014533
:102140008280931726003307F500AE9718439C430F
:1021500063E7E7007D16E37FF7FC7D558280054548
:102160008280FD15E205E18513978501618793F76C
:10217000F50F63480700FD15139725002A9758436C
:1021800065D7138517006205618582803308B50223
:102190001C4283A80600B335B502C29733B50701C8
:1021A000AE98469585486367B5006394A50063E3E0
:1021B000070181480C43C6950CC388C21CC28280AB
:1021C00081471397870161876343B7008280139724
:1021D00027002A97232007008507E5B78147014795
:1021E00093968701E18663C5B60013351700828098
:1021F00093962700AA9694428507558FD5B793D713
:1022000055408A07AA979C4305453315B5007D8D37
:10221000828017F3FFDFE702833D2A8497000000E6
:10222000E78060F405C5931725003E940327C4FF9B
:10223000814711EB7D1516053E954205418517F343
:10224000FFDF6700033D05838507E5B70145C5BF8F
:1022500081471397870161876343C7008280139783
:102260002700B386E50094422A97850714C3D5B7A3
:102270007D1662066186014793178601E18763D563
:10228000070013351700828093172600B306F50068
:10229000AE9794429C437D16B58F5D8FF1BF8A0542
:1022A000AA9501476363B500828083A6C5FFF11537
:1022B00093D71600D98F9CC11397F601E5B72A83EF
:1022C0000148014701456343D7008280B387050178
:1022D00083A80700B30706019C43C697AA976384A7
:1022E000F80033B517010507B3080301620723A0FF
:1022F000F80061871108C1BF2A8301478147014562
:1023000063C3D70082803388E50083280800330E3A
:10231000E600032E0E003388A8403308C8416384CA
:10232000080133B508018507B308E300E20723A0DD
:102330000801E1871107E9B717F3FFDFE702232B55
:102340000111B286B2842E86AA850A859700000004
:10235000E780C0FA2A84A6850A8597000000E780F6
:1023600020E833348000060413351500018D056123
:1023700017F3FFDF6700E32917F3FFDFE702A3246A
:102380004111AA89AE8A328BB68402C202C402C647
:102390000144131C8401135C8C4163499C02939B90
:1023A0001400FD1B0549138CF4FFF15C3304890113
:1023B000620461846340740792478E04CE9423AE16
:1023C000F4FE410117F3FFDF6700632313192400B4
:1023D000B30B2B01014A93172A00D69783A50B0054
:1023E000884378003400500097000000E78040DA0E
:1023F000050A93178A01E187F11BE35EFCFC924713
:102400004E9905042320F900A2473EC2B24702C6F6
:102410003EC441B7131A8901135A8A41131D24007F
:1024200093178A01E18763CF970092470A044E947D
:102430001CC0A24705091379F90F3EC2B24702C674
:102440003EC4ADB7B3079A0313152A005695084149
:10245000780034005000050AEA97DA978C43970019
:102460000000E780E0D26DBF197106C212C416C623
:102470001AC81ECA22CC26CE2AD02ED232D436D6A4
:102480003AD83EDA42DC46DECAC0CEC2D2C4D6C694
:10249000DAC8DECAE2CCE6CEEAD0EED2F2D4F6D684
:1024A000FAD8FEDA971500009385C58A8841E700BF
:1024B000050092402242B2424243D2436244F24477
:1024C000025592552256B2564257D2576258F25888
:1024D00006499649264AB64A464BD64B664CF64CB8
:1024E000065D965D265EB65E465FD65F0961730047
:1024F00020300000972100209381C1B017410020B7
:102500001301413017F5FFFF130505B097050020B3
:10251000938545AF171600201306C6FD63FAC50064
:102520008322050023A0550011059105E3EAC5FEAD
:10253000170502001305450F97150020938585FBAD
:10254000171600201306066563FAC50083220500EE
:1025500023A0550011059105E3EAC5FE17150020DB
:1025600013054563974500209385450D6377B500B6
:10257000232005001105E36DB5FEFD42739002BCFA
:102580008D4273904280B7220000938282887390BC
:102590000230970200209382E2A693E23200739009
:1025A0005230975200009382A2B4739012346FB0ED
:1025B000342573002030397101436EC619A039717A
:1025C00041536AC866CA62CC5ECE19A03971015304
:1025D0005AD056D252D44ED64AD826DA22DC06DE5B
:1025E00033016140828241114AC026C222C406C61C
:1025F0008282B24D4101024D924C224CB24B4101BC
:10260000024B924A224AB249410102499244224471
:10261000B240410182803D432A876373C3029377AE
:10262000F700BDEFADE5937606FF3D8ABA960CC381
:102630004CC30CC74CC74107E36BD7FE11E2828045
:10264000B306C3408A069702000096966780A600EC
:102650002307B700A306B7002306B700A305B700FA
:102660002305B700A304B7002304B700A303B700F2
:102670002303B700A302B7002302B700A301B700EA
:102680002301B700A300B7002300B700828093F5B1
:10269000F50F93968500D58D93960501D58D61B77D
:1026A000939627009702000096968682E78086FA26
:1026B0009680C1171D8F3E96E374C3F8A5B73367A4
:1026C000B500FD530D8B79E7B7877F7F9387F7F7C9
:1026D00010419441B372F6003363F600BE92B3E248
:1026E00062006397720C6318D6065041D441B372EE
:1026F000F6003363F600BE92B3E262006398720A9A
:10270000631BD60410459445B372F6003363F6009C
:10271000BE92B3E262006391720A631ED602504514
:10272000D445B372F6003363F600BE92B3E26200A2
:10273000639A72086311D60210499449B372F60085
:102740003363F600BE92B3E26200639372085105F0
:10275000D105E30FD6F61317060193970601631C04
:10276000F7001357060193D706013305F740937519
:10277000F50F91E982804183C1833305F74093755A
:10278000F50F91E182801377F70F93F7F70F330579
:10279000F74082800346050083C6050005058505D0
:1027A0006313D60065FA3305D64082801105910582
:1027B000E312D6FE014582802105A105E31CD6FC6B
:1027C000014582803105B105E316D6FC01458280C2
:1027D0004105C105E310D6FC01458280B7170040D2
:1027E00003C777051377E70FA38BE704130700F8F8
:1027F000A38DE7043D47238CE70413075003A38C04
:10280000E70403C7A7051377D70F238DE70482805A
:10281000B717004003C7E7040D8941111377C70FAD
:10282000498F93068008F3B6068093F6860836C66D
:1028300001000100930670052380D704930680FAF7
:102840002380D704010001002387E70423800704C5
:10285000B247F3A707800100010041018280B7174A
:10286000004003C7E7020D8941111377C70F498F55
:1028700093068008F3B6068093F6860836C60100F4
:102880000100930670052380D704930680FA238005
:10289000D704010001002387E70223800704B24721
:1028A000F3A70780010001004101828041112A83C2
:1028B000014E930E407E130F0019930F400663E5FF
:1028C0006E129308001913034006B3781503854E62
:1028D0000D4FA14F337365020D891335150063EF5A
:1028E000BE121308F6FF7946729842081358080181
:1028F0003307C70213D61700BE0732976146B3F6F7
:10290000C60213068070B386C6023697A166F58F9D
:1029100042075D8FB716004083C7F60293F707089A
:10292000A303F1000346710083C7F60293F707087B
:10293000E394C7FE83477100B716004093F7F70F83
:102940006388071293078008F3B7078093F7870817
:102950003EC401000100B7170040930670052380B4
:10296000D704930680FA2380D7040100010023AA2C
:10297000070383C6170393E60608A388D7022380BC
:102980000704A247F3A70780010001001166B717EB
:1029900000407D16D45BC85F93854703A98EF18EF6
:1029A000F5FA93068008F3B6068093F6860836C6D5
:1029B00001000100930670052380D704930680FA76
:1029C0002380D7040100010098C103C717031367D0
:1029D0000704A388E70223800704B247F3A7078010
:1029E00001000100410182807D133368E3039308F5
:1029F000E016630E08003368F3039308D0166308EB
:102A000008009378330093B818009388D8163308D9
:102A10001E01131E0801135E0E0155B56393E503F5
:102A20000548638608000148630303002A8871088B
:102A30007298FD15131E0801C205135E0E01C181B7
:102A400079BD13F8150063F4BF007908D5B71338C2
:102A50001800E5BF83C7F60293F70708A303F10048
:102A60000346710083C7F60293F70708E394C7FE95
:102A70008347710093F7F70FF1DFE9B531714AD958
:102A800066CB06DF22DD26DB4ED752D556D35AD190
:102A90005ECF62CD6AC96EC7AA8C02D897100000BB
:102AA000E780C0B92A8993078008F3B7078093F7B6
:102AB00087083EDA01000100B717004013077005D0
:102AC0002380E704130780FA2380E7040100010054
:102AD00003C7F7021377770FA387E70203C7F7024D
:102AE00013678700A387E70223800704D257F3A761
:102AF000078001000100054597000000E78060D6CF
:102B0000130780C13347E902116A93070AE8930665
:102B10005002BD69930BA004814A014B1304800845
:102B2000930470057D1AB347F9023307D7023EC0FC
:102B3000FD873ECC938709A69309803E3347F70271
:102B40003AC27D873AC4334739038549B39999011D
:102B500093D93940B306D702B30B7703B3C6F60255
:102B6000B3CBFB0236C6FD8636C893D6FB4136CEC4
:102B7000B7460F00938606243349D90285669386AB
:102B800006FAB3969601B389E90213076055330933
:102B9000D90293060010B389E9023349D902B3C9B7
:102BA000F9029316390036CA37190040FD8636D02F
:102BB000930D090493D7F9413ED2F336048093F67E
:102BC000860836DC01000100930770052380FD00B4
:102BD000930680FA2380DD00010001008346390559
:102BE00093F6860FA309D9048346390593E61600A8
:102BF000A309D90423800D00E256F3A60680010044
:102C00000100130C80FA116DF336048093F68608E8
:102C100036DE01000100930770052380FD0023804C
:102C20008D010100010083463905216693E6060205
:102C3000A309D90483560905B3E6A6012318D904CC
:102C400083560905D18E2318D90423800D00F2562E
:102C5000F3A60680010001008346390593F60602BB
:102C60006381061A03463905218A6DDE081897101C
:102C70000000E780A0A07336048013768608B2C2F5
:102C80000100010023809D0023808D0101000100CF
:102C9000B717004003C637051376F60DA389C7049E
:102CA00003C6370513660602A389C70483560905C0
:102CB0002166B3E6A6012318D90483560905D18EEF
:102CC0002318D90423800D009646F3A60680010040
:102CD00001008346390593F60602638B061483468A
:102CE0003905A18AEDFE97F0FF1FE780C03AAA865A
:102CF00036D497F0FF1FE780003AA256E30AD5FECC
:102D0000835609054255B3E6A6012318D904971046
:102D10000000E780609883463905A18AEDDE0356FE
:102D200009058346290582473376CA00B306DA02CD
:102D300093D5F641B296B388F640E24733B8C60061
:102D40002E983308F840A247B3B616013308D8408E
:102D500063C70701631DF800924763FA1701C24772
:102D6000634FF80E63950701B24763EAF80E894690
:102D700063E9660FF2469315180013D3F8015E86D7
:102D800013951800B365B30042D646D497C001002E
:102D9000E78020A83258050B137BFB0F6347000127
:102DA000631A0838A2586387083813081500B33629
:102DB000A800B69513D6F5013298B336C800AE9682
:102DC00013581800FE06B3E6060173360480137626
:102DD0008608B2C60100010023809D0023808D017A
:102DE000010001000356C902B296C206C182231631
:102DF000D90223800D00B646F3A60680010001002B
:102E000021B5F336048093F68608B6C001000100B0
:102E100023809D0023808D01010001008346390538
:102E200093E60602A309D90423800D0086460DB55A
:102E3000F336048093F68608B6C4010001002380AF
:102E40009D0023808D01010001008346390593E632
:102E50000602A309D90423800D00A646BDB5E30BE5
:102E60000BF0F336048093F68608B6C80100010023
:102E7000930680FA23809D002380DD00010001007D
:102E80008346390593F5FC0F93F6860FA309D90401
:102E900083463905CD8EA309D90423800D00C6468B
:102EA000F3A6068001000100130580FA03463905E8
:102EB000930639051D8A631C9629733604801376A0
:102EC0008608B2CC01000100130680FA23809D0021
:102ED0002380CD000100010003C606001376F60D25
:102EE0002380C60003C60600136606022380C600C0
:102EF000835609051166D18E2318D9048356090516
:102F00002166D18E2318D90423800D00E646F3A64E
:102F1000068001000100130680FA8346390593F606
:102F200006026380062683463905130C3905A18AFB
:102F3000FDDA081897000000E7804074F33604803B
:102F400093F68608B6D001000100930680FA23802C
:102F50009D002380DD000100010083460C00116606
:102F600093F6F60D2300DC0083460C0093E6060280
:102F70002300DC0083560905D18E2318D90483561B
:102F800009052166D18E2318D90423800D008656A9
:102F9000F3A6068001000100130680FA8346390576
:102FA00093F60602638A062083463905A18AEDFE60
:102FB00097F0FF1FE780200E2A8C97F0FF1FE78015
:102FC000800DE30C85FF8356090511664255D18EAD
:102FD0002318D90497000000E780006C8346390568
:102FE00013063905A18AFDDAF336048093F68608C4
:102FF000B6D401000100930680FA23809D0023804F
:10300000DD00010001008346060093F6F60D230063
:10301000D60023800D00A656F3A60680010001000D
:103020008356090503462905D247B376DA003306ED
:10303000CA021305800C9355F6413696330DF640BF
:103040008257333CD6002E9C3336A601330CFC400D
:10305000330CCC403308850392564E86B335A50316
:103060003305A503C29597B00100E780807A6346D7
:103070008001631E0C16630C0D1613061500333504
:10308000A6002E959356F5013696B335D600AA952F
:103090009396F50105828585D18E6346B000639DC8
:1030A000051A638B061A0356C90215823305D6002A
:1030B0003336C500B2956348B0006391052413060A
:1030C000F00F637DA622894663F3561593078008A7
:1030D000F3B7078093F78708BED6010001003717C2
:1030E0000040930770052300F704930780FA23003C
:1030F000F704010001008356C70289678117D58F45
:10310000C207C1832316F70223000704B657F3A7AB
:10311000078001000100FA506A54DA544A59BA593A
:103120002A5A9A5A0A5BFA4B6A4CDA4C4A4DBA4D03
:10313000296182801308F5FF3335A800FD152E950F
:103140001356F5013298B336C800AA9695B9F336EE
:10315000048093F68608B6CA0100010023809D0012
:103160002380AD000100010083463905CD8EA309FF
:10317000D90423800D00D646F3A606800100010085
:1031800035B3F336048093F68608B6CE010001000D
:1031900023809D002380CD00010001008346390576
:1031A00093E60602A309D90423800D00F646F3A690
:1031B00006800100010095B3F336048093F686087B
:1031C000B6D20100010023809D002380CD000100C4
:1031D00001008346390593E60602A309D90423803A
:1031E0000D009656F3A606800100010045BB93062C
:1031F000F5FF33B5A600FD152E959355F501AE9656
:10320000B3B5B600AA951396F501858269B5F33674
:10321000048093F68608B6D801000100930680FA70
:1032200023809D002380DD00010001008356C90238
:103230000566011693F6F60FD18EC206C1822316DB
:10324000D90223800D00C656F3A6068001000100B6
:10325000850A93FAFA0F95B233E6B60045C20356D3
:10326000C9023305D0403338A000B305B040B38560
:10327000054115826345B000D1E16371A608894616
:1032800063F0560593078008F3B7078093F7870824
:10329000BEDA01000100B717004013077005238054
:1032A000E704130780FA2380E7040100010003D735
:1032B000C7027D8B2396E70223800704D65781BD82
:1032C000F336048093F68608B6DC0100010093060D
:1032D00080FA23809D002380DD00010001008356D9
:1032E000C9020566011693F6F60FD18EC206C18299
:1032F0002316D90223800D00E656B9B7930780083C
:10330000F3B7078093F78708BEDE01000100371787
:103310000040930770052300F704930780FA230009
:10332000F704010001000356C70293975600B297B5
:10333000C207C1832316F70223000704F657C1BB57
:10334000914763EEB70217D70100130727388A05A4
:10335000BA959C41BA978287B717004003A7470BDD
:103360001345F5FF698F23AAE70A03A7070B698FA7
:1033700023A8E70A03A7070A798D23A0A70A82805A
:10338000B717004083A6470B1347F5FFF98E23AA12
:10339000D70A83A6070B558D23A8A70A83A6070A79
:1033A000758F23A0E70A8280B717004003A7470B59
:1033B000498F23AAE70A03A7070B1345F5FF45BF6B
:1033C000B717004083A6470B1347F5FF758F23AA55
:1033D000E70A03A7070A598D4DB7B717004003A79F
:1033E000470B498FEDB7914763EEB70217D701003E
:1033F0001307072F8A05BA959C41BA978287B7179A
:10340000004003A7470D1345F5FF698F23AAE70C7A
:1034100003A7070D698F23A8E70C03A7070C798D75
:1034200023A0A70C8280B717004083A6470D13473F
:10343000F5FFF98E23AAD70C83A6070D558D23A877
:10344000A70C83A6070C758F23A0E70C8280B71703
:10345000004003A7470D498F23AAE70C03A7070DD8
:103460001345F5FF45BFB717004083A6470D134727
:10347000F5FF758F23AAE70C03A7070C598D4DB7ED
:10348000B717004003A7470D498FEDB79357E500E5
:1034900093F70730C98FC2070547C1836382E504EC
:1034A0008DC10947638DE5040D476380E506371735
:1034B0000040231FF70883562709D58F2319F708E3
:1034C0008280371700400356670993C6F7FFF18ED5
:1034D000231BD7088326C70C558D2326A70CC1BFF5
:1034E000371700400356670993C6F7FFF18E231B79
:1034F000D7088326870C558D2324A70C4DBF37177B
:10350000004083566709DD8EE1B7371700408356C8
:103510006709DD8EE9BF797122D43714004026D2C5
:103520004AD0035924028354040206D64209C20435
:103530004ECE52CC56CA13590901C1802DE11379E0
:10354000F9F793F4F49F4209C20413590901C180A9
:1035500093078008F3B7078093F787083EC40100FC
:103560000100930770052300F404930780FA2300F9
:10357000F40401000100231124032310940223000A
:103580000404A247F3A7078001000100B2502254AF
:1035900092540259F249624AD24A45618280B7F593
:1035A000070081463000B105194597F0FF1FE780FD
:1035B0000074A24713972701E34A07FC136909081F
:1035C00093E4044093098008F3B7098093F78708D0
:1035D0003EC001000100930A700523005405130A40
:1035E00080FA230044050100010023112403231065
:1035F0009402230004048247F3A70780010001001E
:10360000294597F0FF1FE7800026F3B9098093F959
:1036100089084EC20100010023005405230044051F
:10362000010001008357040293E707202310F402EE
:10363000230004049247B9B7B717004088474205F2
:1036400041819377050491EB9377F5013755E801B4
:10365000130505803345F50282809377050C130727
:1036600000046397E7009377F50137459C1CCDB7BD
:103670002165130505D0828037E700E01C435443E1
:10368000A183E206D58F1CC1FD572320F718232202
:10369000F718828013178500B7E700E023A0E71032
:1036A000618123A2A7108280B7F700E08847CC474A
:1036B0008280814737370040A14663C4C700328506
:1036C00082800345B740E38EA6FE3385F5000345AF
:1036D000050085072304A740CDB7970700209387EF
:1036E00067E19C4317370020130747F53E95636E4B
:1036F000E500173700201307E7F86368A7001707EE
:1037000000202329A7DE3E858280FD57EDBF828001
:10371000411122C406C62A8497000000E78000F207
:103720002947B307E502B2408D83B3D7870222440D
:103730009507B3D7E70237370040C207C183231686
:10374000F70041018280716541111305052006C60D
:1037500097000000E78000FCB7370040130770F8BF
:103760002381E7000D47A381E70013070004A3802E
:10377000E70005472387E700B240410182803737E1
:103780000040834727001A0593F7F703C98F93F783
:10379000F70F2301F7008280B737004003C71700F7
:1037A00019C9D98DA380B70003C707001367870025
:1037B0002380E700828093C5F5FFF98DA380B700D1
:1037C0008280AE872A87B7360040214637380040CE
:1037D00089E7170300006700C3F383C8B600E30955
:1037E00016FF05078348F7FFFD17C20723041801DA
:1037F000C183F9BF411122C406C62A849700000084
:10380000E780C0E32947B307E502B2408D83B3D711
:10381000870222449507B3D7E70237370040C20733
:10382000C1832316F7404101828071654111130560
:10383000052006C697000000E78000FCB73700406F
:10384000130770F82381E7400D47A381E740130772
:103850000004A380E74005472387E740B2404101C9
:103860008280CC41411106C6328503C6150083C54E
:10387000050022064D8E42068D654186138875A28D
:10388000630C0611634BC804138845A26300060D40
:10389000634AC800938535A26301B60823900600E9
:1038A00029464DA0138855A26305060D938565A290
:1038B000E316B6FE8D451D4663E6E5081146198EF2
:1038C00063F3C7003E86B7E704002390C600FC47B9
:1038D00097D50100938505E39DA0138895A2630306
:1038E0000611634E060D1388A5A263000613938587
:1038F00005A5E315B6FA99451D4663E5E504198E5D
:1039000063F3C7003E86B7E704002390C600FC4778
:1039100097050020938545C81DA09D451D4663E37E
:10392000E5022146198E63F3C7003E86B7E704001F
:10393000FC472390C6009705002093852526BA955D
:1039400082970146B240328541018280AD451D46D5
:10395000E3EAE5FE3146198E63F3C7003E86B7E71A
:1039600004002390C600FC4797D50100938505DC31
:10397000F9B7B1451D46E3E7E5FC3546198E63F31B
:10398000C7003E86B7E704002390C600FC4797D5E2
:1039900001009385A5DA65B78D451D46E3E4E5FA98
:1039A0001146198E63F3C7003E86B7E704002390E3
:1039B000C600FC4797D50100938585D549B78D454D
:1039C0001D46E3E1E5F81146198E63F3C7003E8614
:1039D000B7E704002390C600FC4797D50100938504
:1039E000A5D7B1BFA5451D46E3EEE5F42946198EDE
:1039F00063F3C7003E86B7E704002390C600FC4788
:103A000097D50100938585D11DBFB5451D46E3EBD4
:103A1000E5F23946198E63F3C7003E86B7E7040026
:103A20002390C600FC4797D501009385A5CC01BF24
:103A3000B7E7040003A30713970600209386C6B4D4
:103A40004146A54517050020130505AB02832D450A
:103A50005DE703C505000947631FE50803A84500A6
:103A6000411106C6034718003285034608002207A5
:103A70004168518F930828FE6307170563E9E80042
:103A800005186303070323900600294591A8130630
:103A900048FE630AC7041518E31707FF15463E875B
:103AA000637BF600154701A8130600023E87637486
:103AB000F60013070002B7E704002390E600FC4776
:103AC0001316070111A83E8691C30546B7E7040007
:103AD000FC472390C6004206CC45418282970145AF
:103AE000B24041018280130600083E87E375F6FC70
:103AF00013070008C9B7239006000545828082801D
:103B0000416779176304E504411122C406C685475D
:103B10002A84639FF500B7E7040022852244B2405F
:103B200003A3871397050020938585214101028314
:103B300089476399F500B7E7040083A7070B85451C
:103B4000829771D9B240224441018280828079718A
:103B500022D452CC2E842A8A97D501009385C5C1E0
:103B600017D501001305C5C306D63AC626D24AD0DA
:103B7000B68432894ECE97B00100E780C014A68586
:103B800017D501001305C5C297B00100E780A01347
:103B9000294597B00100E780E0178347840093F739
:103BA0000702E1E7834904008947054532476396E8
:103BB000F908544083C7160083C60600A207D58FB4
:103BC000C166138616FE638CC7028D16638FD706F7
:103BD0008D669386269029456391D706B7E7040042
:103BE000A285225403A34714B250F249A6864A86FE
:103BF000925402595285624A8547456102832D4598
:103C00000DEF93070002354563E99702B7E704001B
:103C1000FC47484413060002CA85829781499707EA
:103C200000209387A7129C43014581CB9C4391C7F9
:103C30004E852686CA8582970145B25022549254F9
:103C40000259F249624A456182802D457DF793070A
:103C5000700F3545E3E397FEB7E70400FC4748449F
:103C60001306700FCA8582975DBF2145F9B74111D0
:103C700022C437E404008327841326C2AA84416542
:103C800006C6970500209385A50B7D15829783278F
:103C9000C40A170500001305E5E68588829795C0DC
:103CA000032304132244B2409244970600209386D3
:103CB00026A04146C545170500201305658E410124
:103CC0000283B2402244924401454101828019C5D9
:103CD0009707002023ACA7060145828045458280D6
:103CE0001147636AA70A97D601009386A6A70A051B
:103CF00036951841411106C63697AE87B2850287C0
:103D0000130700026145639DE700B7E70400FC4725
:103D100013060002170500201305C5E88297014528
:103D2000B2404101828005476145E39BE7FEB7E76A
:103D30000400FC470546170500201305A5E8F9BF58
:103D40001307700F6145E39DE7FCB7E70400FC47EC
:103D50001306700F17050020130505E7C1B71307F9
:103D600000086145E39EE7FAB7E70400FC47130645
:103D70000008170500201305A5F44DB71547614548
:103D8000E390E7FAB7E70400FC4715461705002063
:103D9000130545FB61B709458280411126C2B7E48E
:103DA000040083A7C41322C44AC006C62E84970504
:103DB00000209385E5F82A898297058905C597F73C
:103DC000FF1F9387E77D83D7A70BA28503A3440D2D
:103DD0002310F4002244B24092444A85024901462D
:103DE00041010283B24022449244024949454101C3
:103DF0008280114517F3FFFF670083C84111939636
:103E00002500AA852D4506C697F0FF1FE78020EE06
:103E1000B240014541018280011122CC06CE371407
:103E2000004026CA4AC84EC652C483447405034A99
:103E3000B405834984050349940597F0FFFFE780A3
:103E4000209A8347A40593F4F40F137AFA0F93E7AB
:103E50001700230DF40493F9F90F1379F90FB7172D
:103E6000004003C7A705058B6DFF03D5C705A38DCC
:103E70004705238C3705A38C2705A38B9704F240B5
:103E80006244D2444249B249224A056182804111CA
:103E90009397050122C406C626C2C1872E8463D02B
:103EA0000702B7E40400FC54829719C1BC548297FE
:103EB0002165218DB240224492444101828093F7D2
:103EC000150013C51500FDF79397250163D8070268
:103ED000B7E4040083A7C41E829797000000E78020
:103EE00080F1BC4C37F60200130606E08965170521
:103EF0000020034525E68297096565BF9397150164
:103F00000145E3D907FA17D501001305659297B06B
:103F10000100E78020F3B7E70400BC4F13060064FC
:103F20009165170500200345E5E28297116551B7B9
:103F30002D71232A9110FD74E98C232C81102328E4
:103F40002111232631112A84AE893289930600106B
:103F50000A86A6852D45232E111097F0FF1FE780B6
:103F600000D913154401B7E70400FC4751810A0545
:103F700013962900CA850A958297A685856601460B
:103F8000254597F0FF1FE78080D60A86A685930611
:103F90000010294597F0FF1FE78060D58320C111ED
:103FA0000324811183244111032901118329C110A4
:103FB00015618280B7F7070003C70701411106C6E4
:103FC00022C426C24AC0A547631DF700970000001F
:103FD000E78040F6B2402244924402490145410143
:103FE000828013942500AA843289A286AA8501467C
:103FF000254597F0FF1FE78080CFA2864A86A685D9
:10400000294597F0FF1FE78080CEE9B71D71A2CC4C
:1040100037E404005C5C485886CE494697C50100E9
:104020009385857C829711E917C501001305057DED
:1040300097B00100E78000E101A0B7F600E07957F2
:1040400098CAFD57DCCA0567B7E700E023A0E71070
:104050001306F00290C223A0E71801000100370701
:10406000002018471306000481459706002023A16D
:10407000E6CE4157A38AE7403C4408088297970759
:1040800000209387E7693EC8856793870740231A16
:10409000F1009D673ECCB7070105938707103ECE20
:1040A0009307B00F2310F10285472301F102970710
:1040B00000009387E7D4BEC2970700009387C7EF3D
:1040C000BEC4930750112312F10297F7FFFF9387A5
:1040D000E75D3ED897070000938747D43EDCB7F5ED
:1040E000070097070000938707D13EDE81469707B8
:1040F00000009387E71D3000E10519453EDA97F08F
:10410000FF1FE780C0BE18088147994630003E96E1
:104110000346060085070507A30BC700E398D7FEF3
:10412000C24791C70357410185676373F70001A038
:10413000B7E7040083A7470A08088297AA8511C930
:1041400017C501001305C56C97B00100E780A0B743
:1041500001A0F640664425618280411126C2B7E481
:10416000040083A7040806C622C41705000013052F
:1041700045D28297170400201304C4BD2300A40075
:1041800097000000E780000797000000E780E0222A
:1041900003450400224403A38405B240924413065D
:1041A0000032896541010283411193078008F3B70A
:1041B000078093F787083EC601000100B71700404B
:1041C000130770052380E704130780FA2380E704B0
:1041D00001000100C8DB23800704B247F3A7078072
:1041E000010001009707002023A807B64101828043
:1041F000797106D622D413078008F337078093F726
:1042000087083EC201000100B71700409305700502
:104210002380B704130680FA2380C704010001003D
:1042200083C6F70293F6A60FA387D702238007045D
:104230009246F3A6068001000100733707801377CA
:1042400087083AC4010001002380B7042380C70413
:104250000100010003C7F70213672700A387E702E5
:1042600023800704A247F3A707800100010005454A
:1042700097E0FFFFE780E05E97000000E780A0B7CF
:10428000014781468147054685451305407E97E0F5
:10429000FFFFE780E06137E404003C4468005146DA
:1042A00081458297B707C0A83EC8B787E8039387C0
:1042B00007D03ECA97E7FF1F9387A7633EC67C5887
:1042C00068008297B250225445618280011126CA4B
:1042D00006CE22CCAA8497300000E780600371C923
:1042E00093070004138404FC63E797003704C0A815
:1042F000130404FC2694680097F0FFFFE780003861
:1043000097E0FF1FE78020D9B307A4406376A4009D
:10431000B707C0A8A297898F3747F6A6811713075A
:1043200007C6637DF700324597F0FFFFE780C03690
:104330000945F2406244D24405618280228597009B
:104340000000E780A0E6324597F0FFFFE780C03429
:10435000373700408347574093F70704A9CB97307E
:104360000000E7800007970700209387E79E9C43A3
:10437000A9E31165690597E0FF1FE78060EA05453D
:1043800097E0FFFFE7800049054597F0FFFFE780D2
:10439000C01897E0FF1FE78000D02AC497E0FF1FF6
:1043A000E78060CFA247E30BF5FE014559B7010056
:1043B00055B70D45BDBF011106CE22CC13078008AD
:1043C000F337078093F787083EC401000100B71751
:1043D0000040930570052380B704130680FA2380FC
:1043E000C7040100010083C6E70093E69601238716
:1043F000D70023800704A246F3A60680010001002F
:1044000073370780137787083AC6010001002380BD
:10441000B7042380C7040100010003C71703136713
:104420000702A388E70223800704B247F3A70780A7
:1044300001000100B707001037E400E02320F4106A
:104440008545414597F0FFFFE78020FA89454145C2
:1044500097F0FFFFE780C003B70704002320F410A4
:10446000F240624405618280411197D50100938535
:1044700065A217C501001305A53206C697B0010055
:10448000E780608417D50100130585B997B0010056
:10449000E7806083B2402945410117B301006700FE
:1044A0006387411197D50100938505A017C50100C9
:1044B0001305052F06C697B00100E780C08017D509
:1044C00001001305A5B497A00100E780C07FB240AA
:1044D0002945410117B301006700C383411122C47C
:1044E00006C6834705002A849DC797D5010093859A
:1044F00065A117C501001305A52A97A00100E78053
:10450000807C4C4017D501001305C5C597A001005C
:10451000E780607B3DA058410DEF97D50100938562
:10452000659E17C501001305A52797A00100E78028
:10453000807917D50100130565C497A00100E780B5
:1045400080782244B2402945410117A30100670049
:10455000637CA1679386D7036313D70297D50100C5
:104560009385459A17C501001305852397A001007F
:10457000E780607517D50100130545C17DBFED07C4
:1045800097D501009385059817C5010013054521AE
:10459000631BF70097A00100E780E07217D50100C8
:1045A000130505C059BF97A00100E780C0714C40BA
:1045B00017D501001305C5C091BF411197D5010062
:1045C0009385C58F17C501001305851D06C697A0E5
:1045D0000100E780406FB2402945410117A3010067
:1045E00067004373797122D426D24AD02E842A8957
:1045F0008145B2844800714606D697E0FFFFE78008
:10460000C00197F7FF1F9387672BDC4783D707000D
:10461000231421012313F10097500000E780E08B61
:104620009547A305F1009307401F3EC6FD5723059C
:10463000A100230AF10097500000E780409E2686E3
:10464000A285480097500000E780008CB2502254A9
:104650009254025945618280971700202399075888
:1046600097170020238E074AB7E70400BC47411183
:1046700006C641468145170500201305E5F88297D7
:1046800097200000E780005E97200000E780203937
:10469000014597500000E780E02B170700200347F3
:1046A000A7F89307F00A6315F7029307F0F8894516
:1046B00017050020130545F7170700202306F7F616
:1046C00097070020A38207F697500000E7808058E4
:1046D00097500000E780606A81453705040097071E
:1046E000002023A107F297070020239B07F09707DC
:1046F0000020238807F097070020239907E89707F1
:104700000020239707E697070020239A07EE9707D4
:104710000020239307F097300000E78000CF014589
:1047200097500000E780005C97C501009385857B6A
:1047300017C501001305C50697A00100E780A05822
:1047400017D50100130505AE97A00100E780A0571B
:10475000B2402945410117A301006700A35B411145
:1047600022C406C626C293F715002E84638F071055
:10477000814617F6FF1F1306A61185451705002071
:104780000355C5DE97C00000E780A0C515C997C5D1
:1047900001009385E57517C501001305650097A015
:1047A0000100E780405217C501001305251797A0A7
:1047B0000100E7804051294597A00100E78080551E
:1047C00097C501009385C57217C50100130545FD06
:1047D00097A00100E780204F17C50100130545157C
:1047E00097A00100E780204E294597A00100E780AF
:1047F000605217F5FF1F1305650C5C4505472390B4
:10480000E70097300100E780207697C50100938587
:10481000256E17C501001305A5F897A00100E780D4
:10482000804A17C501001305E51197A00100E78034
:104830008049294597A00100E780C04D930710F8F3
:10484000170700202302F7DE9707002083D7C7D180
:1048500017070020A30AF7DC170500201305C5DCA5
:10486000A1839145170700202301F7DC970700205B
:10487000A38D07DA97500000E780C03D1345140070
:10488000B240224492444101828093F72500E1C363
:10489000170700200357C7D645CB970600209386FD
:1048A00066D6944297D701009387C79917060020D0
:1048B000034626D58145170500201305E5D49770DA
:1048C0000000E78060D1AA8441C197C501009385AB
:1048D000E56817C501001305A5EC97A00100E78066
:1048E000803EA68517C501001305450797A0010066
:1048F000E780603D294597A00100E780A041970728
:104900000020239F07CE930710F817070020230DE0
:10491000F7D09707002083D727C517070020A305E6
:10492000F7D0A183170700202301F7D091458D47C9
:1049300017050020130545CF17070020A307F7CE62
:1049400097500000E78000311345240015BF93F70E
:104950004500D1C397C501009385456017C5010087
:10496000130505E497A00100E780E03517C50100B5
:104970001305850097A00100E780E034294597A042
:104980000100E7802039930720F817070020230D46
:10499000F7C89707002083D767BF17070020A30534
:1049A000F7C8A183170700202301F7C88547170719
:1049B0000020A30CF7C697400000E780406617056B
:1049C0000020130565C6914597500000E7808028B8
:1049D0001345440075B593F78500A9C797C5010035
:1049E0009385C55717C50100130585DB97A0010006
:1049F000E780602D17C50100130545F997A0010058
:104A0000E780602C294597A00100E780A030970738
:104A10000020239707BE97700000E780C0CB1345A6
:104A20008400B9BD93F70501D1C385451705002062
:104A30000355C5B597500100E780E07D97C501009B
:104A40009385C55117C50100130585D597A00100B1
:104A5000E780602717C50100130585F497A00100C2
:104A6000E7806026294597A00100E780A02A9307E8
:104A700030F8170700202309F7BA9707002083D7DB
:104A8000E7B017070020A301F7BA170500201305A8
:104A9000A5B9A1838D45170700202308F7B89750C3
:104AA0000000E780201B13450401D9BB93F70502E2
:104AB000D1C797C501009385654A17C50100130545
:104AC00025CE97A00100E780002017C5010013053F
:104AD00065EF97A00100E780001F294597A001001E
:104AE000E7804023930740F817070020230EF7B212
:104AF0009707002083D7C7A717070020A306F7B2A0
:104B0000A183170700202302F7B28547170700206B
:104B1000A30DF7B097070020239C07A4974000003F
:104B2000E780E04F17050020130505B09145975029
:104B30000000E78020121345040299B393F705049F
:104B4000FDC397C501009385654117C50100130595
:104B500025C597A00100E780001717C501001305C0
:104B6000E5E797A00100E7800016294597A001001E
:104B7000E780401A9707002083C707AB1307700A26
:104B80006386E7061307800A638CE7081307600A49
:104B90006393E704930760F8170700202306F7A83C
:104BA0009707002083D7A7A517070020A30EF7A615
:104BB000A18317070020230AF7A6854717070020BF
:104BC000A309F7A6B145170500201305E5A59750E1
:104BD0000000E780200897400000E780404413452C
:104BE000040497070020239C07A059B9930770F885
:104BF00017070020230AF7A29707002083D727A0D2
:104C000017070020A302F7A2A18317070020230E95
:104C1000F7A0854717070020A30AF7A0994565B7B5
:104C2000930780F8F1B793F705080145E38A07C4B5
:104C300097C501009385853217C50100130545B658
:104C400097A00100E780200817C50100130585DA49
:104C500097A00100E7802007294597A00100E78081
:104C6000600B9307A0F817070020230FF79A970708
:104C7000002083D7679A17070020A307F79AA1831C
:104C8000170700202303F79A854717070020A30E74
:104C9000F798970700202391079897400000E78036
:104CA00000381705002013052598914597500000FE
:104CB000E78040FA13450408E1B6411122C497C5C4
:104CC0000100938565252A8417C50100130545ADAC
:104CD00006C697A00100E78000FF4C4017C5010001
:104CE0001305C54597A00100E780E0FD294597A081
:104CF0000100E7802002034704009307F00F631FC1
:104D0000F70297C501009385252117C501001305FA
:104D100025A997A00100E78000FB4C4017C50100C2
:104D20001305C54297A00100E780E0F92244B24094
:104D30002945410117A301006700C3FDB240224489
:104D400041018280B1C1411122C417C50100130580
:104D500025A52E8497C501009385051706C697A043
:104D60000100E78040F6A28517C5010013054549FB
:104D700097A00100E78020F52244B2402945410177
:104D800017A30100670003F98280411122C426C2E3
:104D90002E84AA8497C501009385C51317C5010009
:104DA000130505A006C697A00100E780C0F117C54E
:104DB00001001305A54597A00100E780C0F0294533
:104DC00097A00100E78000F597C501009385851045
:104DD00097F7FF1F239C977817C501001305459C83
:104DE000854497F7FF1F2391877897F7FF1F239E2E
:104DF000977697170020239C87DE97A00100E78015
:104E000080EC9715002083D585DE17C501001305BA
:104E1000654097A00100E78000EB294597A00100BD
:104E2000E78040EF97170020238C97CE9720000053
:104E3000E780E0BE228597500000E780A0B10545DD
:104E400097500000E78000EA97F7FF1F938707A7B6
:104E5000DC4703D70700C167FD176312F70222443E
:104E6000B7E70400B240924403A3870517F5FF1F7C
:104E70000345C5EE1306000A854541010283B24091
:104E80002244924441018280011122CC37E4040083
:104E90005C5C06CE26CA354697C501009385851908
:104EA00017D50100130505DE829711E917C501002A
:104EB0001305C59497A00100E780C0F801A097F7FB
:104EC000FF1F938767EA3EC4B7F50700856793879E
:104ED0000780814617F6FF1F130686E8E10519458E
:104EE0003EC697E0FF1FE78080E07C44194697F5B7
:104EF000FF1F9385E5E617F5FF1F13056569829788
:104F0000340017F6FF1F1306A6E597C50100938529
:104F1000656A17C501001305656B97600000E7809F
:104F2000A040AA8421C197C501009385250217C519
:104F300001001305E58697A00100E780C0D8A6858B
:104F400017C501001305051097A00100E780A0D741
:104F5000294597A00100E780E0DBF2406244D2449B
:104F60000561828097E00000E780E0A217C501009C
:104F70001305450497500000E780C03497A0000057
:104F8000E78020F797500100E780A05B17F5FF1F2F
:104F90001305458F97500100E780404417C5010075
:104FA0001305450297500100E780205CAA849760B2
:104FB0000000E780009B97000100E7808033978026
:104FC0000100E780A0CC97700000E78040F3976075
:104FD0000000E780001197300100E780E0F497C5FA
:104FE00001009385A5F617B501001305657B99C8E7
:104FF00097A00100E78020CDA68517C50100130505
:10500000A50699B797A00100E780E0CB17C501007E
:105010001305C50797A00100E780E0CA294597A0BE
:105020000100E78020CF97300100E780C0D097F0E3
:105030000000E78080EF630F051085453705040009
:1050400097200000E780603C97C50100938505F03C
:1050500017B501001305C57497A00100E780A0C62D
:1050600017C501001305050497A00100E780A0C53E
:10507000294597A00100E780E0C997E7FF1F9387C4
:10508000A77383D70700171700202312F7B68547A9
:10509000171700202306F7A897200000E78000B725
:1050A00097200000E780A09717150020035525B42E
:1050B00097500000E780008A97F7FF1F83C71766A5
:1050C000ADEBA30301008327441713067100854548
:1050D00013055030829797C50100938525E717B5D2
:1050E00001001305E56B97A00100E780C0BD17C55F
:1050F0000100130565FD97A00100E780C0BC2945AC
:1051000097A00100E78000C197C50100938505E4E1
:1051100017B501001305C56897A00100E780A0BA84
:1051200017C501001305450097A00100E780A0B94D
:1051300005B597C50100938565E117B50100130515
:10514000256697A00100E78000B817C50100130588
:1051500025FB55B797C50100938545DF17B50100BD
:105160001305056497A00100E780E0B517C50100AD
:105170001305450B97A00100E780E0B4294597A0EF
:105180000100E78020B9014597500000E78080B515
:10519000A5BF411122C437E404008327041A06C6C0
:1051A000829797500000E78000848327040817F552
:1051B000FFFF1305055B829797F7FF1F2380A7BAB0
:1051C00017E5FF1F1305856F97400000E780C017A4
:1051D0002244B240410117030000670023CBB7E728
:1051E0000400FC471171A2DDCAD986DFA6DBCED749
:1051F0002E8432892E86AA8517F5FF1F1305C54216
:10520000829717F7FF1F130727428347070093066C
:1052100080029387E70793F7F70FE3ECF610BA895C
:105220008A0717B701001307E760BA979C43BA973C
:1052300082878D4797C50100938585D317B50100F7
:1052400013050556630FF40097A00100E780A0A79F
:1052500017C501001305859097A00100E780A0A65F
:10526000BDA497A00100E78000A617C501001305A3
:10527000659097A00100E78000A5294597A001004F
:10528000E78040A9930720F8114697F5FF1F938503
:10529000A5394A8517F7FF1F2308F73897F7FF1F2F
:1052A000A385073897F0FFFFE78000342A841DC9E3
:1052B00097C501009385C5CB17B501001305454E71
:1052C00097A00100E78020A0A28517C50100130563
:1052D000258E97A00100E780009F294597A0010037
:1052E000E78040A397C50100938585C817B50100E5
:1052F0001305054B97A00100E780E09C17C501004E
:105300001305458C97A00100E780E09B294597A0F5
:105310000100E78020A04165930730FA054697F524
:10532000FF1F938565307D1517F7FF1F230EF72E9E
:1053300097F0FFFFE780402B2A841DC997C5010025
:10534000938505C317B501001305854597A0010096
:10535000E7806097A28517C501001305658597A0B2
:105360000100E7804096294597A00100E780809AD8
:10537000B7E70400BC4F0566130606C8A14517F53C
:10538000FF1F0345A59D8297FE506E54DE544E5973
:10539000BE591161828091476303F40297C50100F1
:1053A000938505BD17B501001305853F97A0010042
:1053B000E780609117C501001305058471BDB7E74B
:1053C0000400FC4F914517F5FF1F0345259982976F
:1053D00097C501009385C5B917B501001305453C74
:1053E00097A00100E780208E17C501001305858274
:1053F00097A00100E780208D294597A00100E78054
:10540000609197400000E78080C1914535A48547B1
:105410006303F40297C50100938585B517B50100B4
:105420001305053897A00100E780E08917B5010052
:105430001305C57F15B597F7FF1F23992715B7E704
:1054400004000566BC4F130606C8C1450DBF8D4755
:105450006303F40297C50100938585B117B5010078
:105460001305053497A00100E780E08517B501001A
:105470001305857DD5B3930740F8114697F5FF1FB7
:105480009385851A4A8517F7FF1F230FF71897F79B
:10549000FF1FA38C071897F0FFFFE780E0142A8412
:1054A000E30405EE97C50100938585AC17B50100AF
:1054B0001305052F97A00100E780E080A28517B5AE
:1054C00001001305E56E97900100E780C07F294534
:1054D00097A00100E780008445BD9147E31CF4F6E6
:1054E000B7E70400FC4F9305000217F5FF1F0345C3
:1054F000E586829797C50100938585A717B50100BA
:105500001305052A97900100E780E07B17B501009D
:1055100013050575F1BD894763E3870297C501004F
:10552000938505A517B50100130585279790010000
:10553000E780607917B501001305C57331BB97F497
:10554000FF1F83C4840E97F7FF1F83C7F70D97C50E
:1055500001009385E5A1A20417B5010013054524B8
:10556000DD8C97900100E7800076A28517B50100D9
:105570001305857197900100E780E074C204294506
:1055800097900100E7800079C1849305D4FF93963A
:105590000401C1824A8693F5F50F17F5FF1F130525
:1055A000D50897200000E78000EAE35F90DC9307CE
:1055B00050F817F7FF1F2309F70683C73900228623
:1055C00097F5FF1F9385450685074A8517F7FF1F47
:1055D000A30DF70497F0FFFFE78000012A84E3059D
:1055E00005DA97C501009385A59817B50100130545
:1055F000251B97900100E780006DA28517C501006B
:10560000130505BFC9B5894763E3870297C5010044
:105610009385059617B5010013058518979001002D
:10562000E780606A17B501001305C56735B197407B
:105630000000E780C09EA28517F5FF1F1305C5FE79
:1056400097400000E780006181B38D476303F40257
:1056500097C501009385C59117B501001305451441
:1056600097900100E780206617B501001305456596
:10567000E5B6B76602000146B7750200054597D04A
:10568000FF1FE780C066930760F817F7FF1F230D21
:10569000F7F897F7FF1FA38A07F89307000617F795
:1056A000FF1F2305F7F8894717F7FF1FA300F7F837
:1056B00097F7FF1F238D07F697F7FF1FA38907F6BC
:1056C000C14717F7FF1F2305F7F6930720F917F7D0
:1056D000FF1FA30FF7F4314697F7FF1FA38BA7F423
:1056E00097F5FF1F938545F44A8597F7FF1F23829F
:1056F00007F497F0FFFFE78020EF2A84E30605C850
:1057000097C501009385C58617B5010013054509A6
:1057100097900100E780205BA28517B50100130573
:10572000A55B55B3B1476303F40297C501009385A8
:10573000258417B501001305A50697900100E780A1
:10574000805817B501001305E55A39B6B7E70400CC
:10575000FC4F9305000417E5FF1F03452560829762
:1057600097400000E780A08BB145F9B5914763E30E
:10577000870297B501009385A57F17B50100130532
:10578000250297900100E780005417B5010013052A
:105790002558D9B497F4FF1F83C444E997F7FF1F36
:1057A00083C7B7E8A204DD8C8E04B77702006D14BE
:1057B000BE942286A68517B501001305A5569790BD
:1057C0000100E7804050B7E70400FC47228697F5C8
:1057D000FF1F9385B5E52800829793160401C182C7
:1057E0003000A685094597D0FF1FE78040502A84E6
:1057F00009C917B501001305A55497900100E7806A
:105800006064930770F8194697F5FF1F9385C5E10B
:105810004A8517F7FF1F2309F7E097F7FF1FA387B4
:1058200087E097F0FFFFE78020DC2A84E30E05B4D1
:1058300097B501009385C57317B50100130545F6AB
:1058400097900100E7802048A28517B50100130555
:10585000255095B99947630BF41297B501009385CC
:10586000257117B501001305A5F397900100E78096
:10587000804517B501001305254FF9BA914763E339
:10588000870297B501009385A56E17B50100130532
:1058900025F197900100E780004317B5010013053B
:1058A000254E5DBA97F4FF1F83C444D897F7FF1FB6
:1058B00083C7B7D7A204DD8C8E04B77702006D14BE
:1058C000BE942286A68517B501001305A54C9790B6
:1058D0000100E780403FB7E70400FC47228697F5C8
:1058E000FF1F9385B5D42800829793160401C182C7
:1058F0003000A6850D4597D0FF1FE780403F2A84E2
:1059000009C917B501001305A54A97900100E78062
:105910006053930780F8194697F5FF1F9385C5D00C
:105920004A8517F7FF1F2301F7D097F7FF1FA38FB3
:1059300087CE97F0FFFFE78020CB2A84E30605A4FB
:1059400097B501009385C56217B50100130545E5BC
:1059500097900100E7802037A28517B50100130555
:10596000654695B699476303F40297B501009385A0
:10597000256017B501001305A5E297900100E780A7
:10598000803417B5010013056545F9B0B7E7040089
:10599000FC4F9305000417E5FF1F0345253C829744
:1059A00097300000E780A067994579B18D47630380
:1059B000F40297B501009385A55B17B501001305A7
:1059C00025DE97900100E780003017B50100130530
:1059D000654259B017B501001305C5429790010003
:1059E000E78040461305C01297D0FF1FE78080E88C
:1059F000014597E0FFFFE78060C80D459710000064
:105A0000E780009F294597D0FF1FE780A0E697D049
:105A1000FF1FE78000D78DBA99476303F40297B55B
:105A200001009385E55417B50100130565D79790DC
:105A30000100E780402917B501001305653D29B82D
:105A400017F7FF1F034797BE97F7FF1F83C707BED0
:105A500022075D8F9166BA96C2061166C18213064F
:105A6000F6EF8D476365D60297E7FF1F938707E53B
:105A70009C4B17F6FF1F034656BB9386C7002DC2EB
:105A800003D6070069CA8907E39CD7FE8947130735
:105A9000A0F8114697F5FF1F938505B94A8597F63B
:105AA000FF1F2383E6B817F7FF1FA300F7B897F08F
:105AB000FFFFE78060B32A84E308058C97B50100F7
:105AC0009385054B17B50100130585CD979001000F
:105AD000E780601FA28517B501001305A534E5B264
:105AE00003D60700630EE60A8907E39BF6FE8D479F
:105AF00079BF91476304F40297B501009385454748
:105B000017B501001305C5C997900100E780A01BD8
:105B100017B50100130585326FF00FF4B7E70400E5
:105B2000FC4F9305000817E5FF1F034525238297C7
:105B3000C9B897B501009385A54317B501001305B2
:105B400025C697900100E780001817B501001305DE
:105B500065306FF06FF02390E70017E5FF1F130526
:105B6000E5D597200100E780804297B50100938535
:105B7000254017B501001305A5C297900100E780E5
:105B8000801417B501001305E52D97900100E780FB
:105B90008013294597900100E780C0178147C5BD54
:105BA0002390070017E5FF1F130545D1972001003B
:105BB000E780E03D97B501009385853B17B501006F
:105BC000130505BE97900100E780E00F17B50100AF
:105BD0001305C52A5DBF411122C406C683470500CF
:105BE0002A849DC797B501009385453417B50100F8
:105BF000130505BB97900100E780E00C4C4017B5FA
:105C000001001305256597900100E780C00BE1A016
:105C10005841B707CF009387777D631DF70697B587
:105C200001009385A53017B50100130565B797905E
:105C30000100E78040091C448356E4008355C400FA
:105C400003C6070017B501001305456297900100D0
:105C5000E7806007294597900100E780A00B035774
:105C6000E4009707002083D787F86309F70083557E
:105C7000C400084497E0FFFFE780E0B40356E40067
:105C80008355C40008442244B240410117F3FFFF8A
:105C900067002355B707CC009387777D6315F7041A
:105CA00097B501009385852817B50100130545AF09
:105CB00097900100E78020011C448356E40083553F
:105CC000C40003C6070017B501001305255A9790B5
:105CD0000100E78040FF2244B2402945410117936B
:105CE000010067002303B707CE009387777D630425
:105CF000F70297B501009385652317B501001305D9
:105D000025AA97900100E78000FC4C4017B50100E0
:105D10001305054BCDBDB240224441018280B7E757
:105D20000400FC4741112E8606C622C426C24AC082
:105D30002E842A89AA8517F5FF1F1305E58E829701
:105D400097B501009385852417B50100130545A576
:105D500097900100E78020F797F5FF1F83C5C58C5A
:105D600017B50100130585CA97900100E780A0F5DB
:105D7000294597900100E780E0F997F4FF1F93848D
:105D8000A48A83C7040041479387070693F7F70F58
:105D9000636AF75C17B70100130707B48A07BA975D
:105DA0009C43BA9782879D476307F40297B5010029
:105DB0009385C51D17B501001305859E97900100B9
:105DC000E78060F017B501001305C5C49790010086
:105DD000E78060EFADAC97F7FF1F83C7F784DDCB9B
:105DE00017F7FF1F0347778497F7FF1F83C7E783E2
:105DF00022075D8F97F7FF1F83C74783C2075D8F19
:105E000097F7FF1F83C79782E207D98F17E7FF1F16
:105E1000232AF77E83C7640097B501009385051791
:105E200017B501001305C59717E7FF1F230BF77C74
:105E300097900100E78020E997E7FF1F9387877C11
:105E40008C4317E6FF1F0346C67B17B501001305F9
:105E500025BE97900100E78000E729459790010053
:105E6000E78040EB97E7FF1FA380077C2244B24006
:105E700092440249930700F817E7FF1F2306F77AB9
:105E80009D4517E5FF1F1305257A410117430000C3
:105E9000670043DC97600000E780609397E7FF1F8F
:105EA0002385A7789357850017E7FF1FA30FF77681
:105EB000935705012A8417E7FF1F2309F7769357A5
:105EC0008501014517E7FF1FA302F77697600000E1
:105ED000E780A09097E7FF1F238BA77497B5010079
:105EE0009385C50A17B501001305858B97900100AE
:105EF000E78060DD17E6FF1F03466673A28517B5CE
:105F00000100130565B4B1B7CD476303F40297B53B
:105F100001009385A50717B50100130565889790C3
:105F20000100E78040DA17B50100130565B379BDBC
:105F300037E404007C44414697E5FF1F9385D56E06
:105F400017E5FF1F1305456C829717E5FF1F130523
:105F5000A56B97100000E78080C497100000E780D1
:105F600000AC97E7FF1F83C7476D17E7FF1F034785
:105F7000B76CA20703238405D98F17E7FF1F2311EE
:105F8000F7681306000A89452244B2409244024948
:105F900017E5FF1F034585DC410102838D4763033D
:105FA000F40297B50100938565FE17A5010013055E
:105FB000257F97900100E78000D117B501001305F8
:105FC000E5B929B517E4FF1F0344246697E7FF1FCF
:105FD00083C7976597B50100938545FB220417A5F4
:105FE00001001305E57B5D8C97900100E780A0CD53
:105FF000A28517B50100130525A897900100E78039
:1060000080CC294597900100E780C0D00D4697E5E8
:10601000FF1F93856561228597E0FFFFE780C05CE5
:10602000AA8421C197B50100938545F617A5010003
:106030001305057797900100E780E0C8A68517B59E
:1060400001001305A5A497900100E780C0C7224472
:10605000B24092440249294541011793010067006B
:1060600063CB97E7FF1F23938752B7E704001166BE
:1060700003A38705130606E8914539B78D476303E7
:10608000F40297B50100938565F017A5010013058B
:10609000257197900100E78000C317B50100130533
:1060A000A5BA2DB317E4FF1F0344245897E7FF1F39
:1060B00083C7975797B50100938545ED220417A52F
:1060C00001001305E56D5D8C97900100E780A0BF8E
:1060D000A28517B501001305A59C97900100E780E4
:1060E00080BE294597900100E780C0C20D4697E524
:1060F000FF1F93856553228597E0FFFFE780C04E21
:10610000AA841DC197B50100938545E817A5010034
:106110001305056997900100E780E0BAA68517B5D9
:1061200001001305259905B797E7FF1F23928744C0
:10613000B7E70400116603A38705130606E8930575
:10614000000299B5894763E3870297B501009385FB
:10615000E5E317A501001305A56497900100E7800A
:1061600080B617B501001305E5B08DB197E4FF1FA8
:1061700083C4A44B97E7FF1F83C7174B97B5010054
:106180009385C5E0A20417A5010013056561DD8CA8
:1061900097900100E78020B3A68517B5010013058D
:1061A000E59297900100E78000B2294597900100A1
:1061B000E78040B6228697E5FF1F9385E546268552
:1061C00097E0FFFFE78040422A84630E051A97B5E7
:1061D00001009385A5DB17A501001305655C979069
:1061E0000100E78040AEA28517B501001305458F79
:1061F00099BD854763F98718834519002244B24049
:1062000092440249B335B00097E7FF1F238AB7389D
:1062100017B501001305058E4101179301006700B2
:1062200083AAA2852244B24092444A850249410190
:10623000170300006700032299476303F40297B530
:1062400001009385A5D417A5010013056555979006
:106250000100E78040A717B50100130565BBBDB677
:1062600017E4FF1F0344643C97E7FF1F83C7D73B36
:1062700097B50100938585D1220417A50100130568
:1062800025525D8C97900100E780E0A3A28517B5A9
:1062900001001305A58797900100E780C0A229455A
:1062A00097900100E78000A7194697E5FF1F9385A7
:1062B000A537228597E0FFFFE7800033AA841DC140
:1062C00097B50100938585CC17A501001305454DB1
:1062D00097900100E780209FA68517B50100130560
:1062E000E58395B397E7FF1F23988732B7E704004C
:1062F000116603A38705130606E89305000869B134
:10630000854797B50100938565C817A5010013055A
:106310002549630BF40097900100E780C09A17B5F8
:1063200001001305E5805DB497900100E780A09916
:1063300017B501001305458197900100E780A098EB
:10634000294597900100E780E09C2244B2409244A6
:10635000024997E7FF1F2395072A410117530000C1
:106360006700633797B50100938545C217A5010003
:106370001305054397900100E780E09417B50100ED
:10638000130545ADA1B4B2402244924402494101F3
:106390008280411106C622C497E0FFFFE780C02437
:1063A0009377F50FA1C32A8497B50100938585BF24
:1063B00017A501001305C53E97900100E780A09046
:1063C0009375F40F17B50100130585E2979001004E
:1063D000E780608F2244B2402945410117930100B4
:1063E00067004393B240224441018280411122C49C
:1063F00091462A8417E6FF1F130646319D652D45F9
:1064000006C697D0FF1FE780808EB7F7070003C747
:106410000701A5476313F70001A09306001001468A
:106420009D65254597D0FF1FE780608C97E7FF1F8C
:10643000238E872C2244B240914617E6FF1F130695
:10644000E62C9D652945410117D3FF1F6700238A6C
:106450005171CAD137E904008327C904A2D52E8619
:1064600086D7A6D32E84AA8517E5FF1F1305C51B63
:10647000829797E7FF1F83C7271B1307700A63875D
:10648000E710636CF7001307600A6384E704BE50EB
:106490002E549E540E596D6182801307800A6388C2
:1064A000E7161307900AE394E7FE8D476309F41C8F
:1064B00097B50100938505E717A501001305452E43
:1064C00097900100E780208017B501001305C5E211
:1064D00025A08D47630CF40297B50100938585E4F0
:1064E00017A501001305C52B97800100E780A07D4B
:1064F00017B50100130585D997800100E780A07CBE
:10650000294597900100E780E08051B7854717B58E
:106510000100130565D917E7FF1F2303F7089790BC
:106520000100E7802092B7750200B76602000146BD
:10653000054597C0FF1FE780807B930760F817E74A
:10654000FF1F2303F70E97E7FF1FA380070E930794
:10655000002617E7FF1F232BF70CE577938707210A
:1065600017E7FF1F2316F70CB14597E7FF1F23829C
:10657000070C97E7FF1FA38EA70A17E5FF1F130558
:10658000A50A97300000E780E06C11B7914763E3FC
:10659000870297B501009385E5D817A5010013057B
:1065A000252097800100E780007217B501001305D0
:1065B000A5D199B797E4FF1F83C4440797E7FF1F4E
:1065C00083C7B706A204DD8C8327C9046D14228615
:1065D00097E5FF1F93859505280082978E049316F3
:1065E0000401B7750200C1823000A695094597C025
:1065F000FF1FE780C06F930770F817E7FF1F2305A1
:10660000F702994597E7FF1FA382A702BDB79147FD
:1066100063E3870297B501009385C5D017A50100F4
:106620001305051897800100E780E06917B50100A0
:10663000130505CBD1B597E4FF1F83C424FF97E76B
:10664000FF1F83C797FEA204DD8C8327C9046D1446
:10665000228697E5FF1F938575FD280082978E049B
:1066600093160401B7750200C1823000A6950D454E
:1066700097C0FF1FE780A067930780F8BDBF17B5DD
:1066800001001305A5C897800100E780A07B1305D2
:10669000C01297C0FF1FE780E01D014597D0FFFFA4
:1066A000E780C0FD0D4597000000E78060D42945D4
:1066B00097C0FF1FE780001C97C0FF1FE780600C9A
:1066C000F9B341114AC097F6FF1F83D6465232896B
:1066D00017D6FF1F0356A62022C426C206C62A8448
:1066E000AE8497000000E780C05F35C12DC0994798
:1066F00063FF97048347140003470400A207D98F60
:1067000013978700A183D98FC2073167C18313070D
:10671000C755639EE70297D7FF1F83D7471CA30186
:10672000F400A1832302F40097F7FF1F83D7274CBF
:1067300091C7A302F400A1832303F400A68517B533
:106740000100130525C297800100E780C05797F725
:10675000FF1F83C7E73CB9CF97D5FF1F83D5251807
:1067600017B501001305C5C197800100E780A0554A
:106770002686A28517D5FF1F0355651697000000D2
:10678000E78060C16301090497E7FF1F83C707F92A
:106790009DCB95C897E7FF1F83C787E08DE72285CC
:1067A0002244B2400249A6859244410117330000B9
:1067B0006700434A17B50100130585BD97800100A6
:1067C000E7804068C1B7B240224492440249410187
:1067D0008280834755008345450017B501001305A6
:1067E00025B7A207DD8D178301006700C34D17B5DC
:1067F00001001305E5B4178301006700A3648D470A
:1068000063FBB70A011126CA06CE22CC0344350029
:1068100097E4FF1F83C494F097B50100938505B8F2
:10682000B337800017E7FF1FA30AF7EE09C497B537
:106830000100938565B717B50100130565B797800B
:106840000100E780404897E7FF1F83C737ED638665
:10685000970097000000E780802697E7FF1F83C717
:10686000F7EB8DC785472306F100B7E7040083A740
:1068700047177000854513055030829717B5010002
:10688000130505B497800100E780C05B9967938783
:1068900057EE2316F100680085479145A307810054
:1068A0002307F10097300000E780C03AF2406244CD
:1068B000D244056182808280894763F7B70801115D
:1068C00022CC06CE26CA8344250085472A84639DB0
:1068D000F404914763F5B70403454500834734004A
:1068E00022055D8D97D7FF1F239BA7FE9700000011
:1068F000E78000489967938767EE2314F100834788
:10690000340023059100A305F10083474400954519
:1069100028002306F10097300000E780A033F24002
:106920006244D24405618280FDF89967938767EEDF
:106930002314F10097D7FF1F83D767FAA305F1004F
:1069400023050100A183E1B782800111996722CC60
:10695000D51717F4FF1F1304A41C2314F100834759
:10696000040026CA97F4FF1F938464282305F100CE
:1069700083D7040028009545A305F100A18306CE26
:106980002306F10097300000E780C02C03D60400F6
:106990008345040017B50100130505A49780010085
:1069A000E7806032F2406244D244056182809D6794
:1069B0007971D9172316F10097F7FF1F83C7471680
:1069C00006D62307F100A9C3B7E70400FC474146F8
:1069D00097E5FF1F938545C31305F1008297680073
:1069E000CD4597300000E780E02697F5FF1F83C56F
:1069F000251317B50100130525A197800100E78035
:106A0000802CB25045618280B7E70400BC47414604
:106A100081451305F1008297D9B7B76702045D710C
:106A2000938757AA3EC08567938707B02312F1006A
:106A300097F7FF1F9387C70E83C70700A2C4A3035E
:106A400001002303F10097F7FF1F9387471A83D7AD
:106A5000070037E4040086C62314F10097D7FF1F10
:106A60009387E7E783D70700414668002315F100C5
:106A70007C4497E5FF1F938525B98297F1450A85E8
:106A800097000000E780E021231EA1007C448A8556
:106A90000810794682973C441305E1030946814575
:106AA0008297101093050002014597D0FFFFE78001
:106AB0006023B640264461618280B7C7A55A0111A0
:106AC0009387C7333EC497E7FF1F83C737C53EC6CA
:106AD000B7F7070003C7070106CE22CCA54763130B
:106AE000F70001A01164930504F09306001001461D
:106AF000254597C0FF1FE780801F3000930504F0F5
:106B0000A146294597C0FF1FE780601E97E5FF1F3C
:106B100083C5D5C017B501001305C59F9780010037
:106B2000E780601AF240624405618280011191653C
:106B3000A1463000938505F02D4506CE97C0FF1F76
:106B4000E780E01A2247B7C7A55A9387C733631473
:106B5000F702B24517B501001305058FB335B00034
:106B600097E7FF1FA38CB7BA97800100E780A015B5
:106B7000F24005618280814517B501001305058F3C
:106B800097E7FF1FA38C07B897800100E780A01349
:106B900097000000E780A0F2E1BFB7C7A55A79715E
:106BA0009387F7353EC6B7E70400FC47AA8506D6AB
:106BB00022D4414608088297B7F7070003C70701A8
:106BC000A5476313F70001A01164930504E8930639
:106BD00000100146254597C0FF1FE7804011700057
:106BE000930504E8D146294597C0FF1FE780201090
:106BF00017B501001305C59597800100E780802433
:106C0000B25022544561828079719165D1467000FD
:106C1000938505E82D4506D697C0FF1FE780200D18
:106C20003247B7C7A55A9387F73517B50100130543
:106C3000E58B6310F702B7E70400FC4717E5FF1F79
:106C40001305859C41460C08829717B50100130572
:106C5000E58797800100E780E01EB25045618280A1
:106C6000B7F7070003C70701A5476313F70001A0A3
:106C700091654111930600100146938505E825456D
:106C800006C697C0FF1FE7808006B24017A5010027
:106C90001305C5794101178301006700A31AC16775
:106CA00069768146FD1705061397060141836364E3
:106CB000B7003E8582803307D50003470700B98FB0
:106CC000214713F81700858363050800B18FC207B9
:106CD000C1837D171377F70F6DF78506F1B741C5AF
:106CE000A547054763F2B70883471500034705002A
:106CF0003168A207D98F13978700A183D98FC20764
:106D0000C1831308C855054763900707411106C69C
:106D100022C426C203442500914763F087049307E9
:106D2000540063ECF502A301C50021822302C500D3
:106D30009304340091C6A302D500A1822303D50099
:106D40002A84A68597000000E780A0F526942300FA
:106D5000A4002181A300A4000147B2402244924430
:106D60003A854101828005473A858280B7C7A55A96
:106D700001119387E7343EC42AC6B7F7070003C75B
:106D8000070106CE22CC26CAA5476313F70001A04F
:106D900091642A84938504EE9306001001462545EC
:106DA00097C0FF1FE780A0F43000A146938504EE52
:106DB000294597C0FF1FE78080F3A28517A5010032
:106DC0001305457797800100E780E0EF970000000A
:106DD000E780E0C4F2406244D24405618280011140
:106DE0009165A1463000938505EE2D4506CE97C0EE
:106DF000FF1FE780C0EF2247B7C7A55A9387E73444
:106E00006318F702B24517A501001305256897D747
:106E1000FF1F2396B7ACC205C18197800100E780B0
:106E200080EA97000000E78080BFF2400561828021
:106E3000D147D14517A501001305456717D7FF1F97
:106E4000231FF7A897800100E780E0E717D5FF1F11
:106E50000355E5A897000000E78080F1F9B701111C
:106E600026CA06CE22CC93F71500AE848DCBAD6733
:106E7000371700409387A7AA1CC3B7E70400BC4F8D
:106E800013060019854517D5FF1F034525A58297D1
:106E900013C51400F2406244D2440561828093F726
:106EA00025006386071897A501009385656E2D461A
:106EB000480097800100E780A0D597F5FF1F83C5A4
:106EC000E5D2854793C4240063E5B7049DC9854591
:106ED00017F5FF1F130505C597200000E78080B850
:106EE00097E7FF1F83C7878389CF97F5FF1F83C568
:106EF000E5CF17F5FF1F1305E5C297300000E780C7
:106F000060D51395040197F7FF1F238107CE4181B8
:106F100051B717F4FF1F0344E4C097F7FF1F83C75F
:106F200077C022045D8CAD67C2059387B755C181D8
:106F3000630DF40C63E18704A9679387A755630F7A
:106F4000F40C17F5FF1F1305E5BD97200000E7803F
:106F500060B197D7FF1F83C7677CD1CF97F5FF1F1D
:106F600083C5C5C817F5FF1F1305C5BB97300000C3
:106F7000E78040CE49A0B1679387C7556302F40408
:106F8000B5679387D755E31EF4FA17F5FF1F13056E
:106F900065B997300000E780E0CB97F5FF1F83C508
:106FA000E5C4894763F9B704F915C205C18117F52E
:106FB000FF1F130545B797200000E780A0AA25A86A
:106FC000054617F5FF1F1305E5B597F0FFFFE780AE
:106FD000806F97F7FF1F83C7A7B491EF4800978092
:106FE0000100E780E0EE93150501C181480097C0DC
:106FF000FFFFE780407DA28517A5010013054557D7
:1070000097800100E78020CCEDBD17F5FF1F130529
:1070100065B197F0FFFFE780007CF1BF17F5FF1F18
:10702000130545B097F0FFFFE780A07CE9B793F721
:1070300045000145E38007E617A5010013058554C7
:1070400097800100E78000E097300000E780A0D43F
:1070500013C5440081B5411122C437E404005C5CCF
:1070600006C6354697A501009385C5FC17B50100F6
:10707000130545C1829711E917A5010013050552B3
:1070800097800100E78000DC01A08327041C829721
:107090002A84054597C00000E780408F9760010073
:1070A000E780601497600100E78060E997B0000016
:1070B000E780C0A02285B24022444101828015674A
:1070C000B71700401307575598C3D8439D66558F8F
:1070D000D8C3D843FD76758FD8C3D8431367F70F4D
:1070E000D8C335671307C7CC98C3828041111305F5
:1070F000800406C622C426C297B0FF1FE780404E18
:1071000097000000E780C01A85457D5597C0FFFFB6
:10711000E780402385457D5597C0FFFFE780E02C41
:10712000371400408327840A8D451305002093E718
:1071300007202324F40A97C0FFFFE780A020B7E4CC
:10714000040097C0FFFFE780806EC8589780010059
:10715000E78040CF17B501001305C5B29780010045
:10716000E78040CE8327840C8545414593E7070897
:107170002324F40C97C0FFFFE78020278D451305DB
:10718000000897C0FFFFE780402697C0FFFFE78019
:10719000C05B014597C0FFFFE780A05E85450545C0
:1071A000894717F7FF1F2305F7A497C0FFFFE78064
:1071B000E05E37070004B7E700E023A0E71097D0B0
:1071C000FFFFE780E0E497D0FFFFE78040F99700FA
:1071D0000000E78080E897000000E7806095970056
:1071E0000000E78000C097E0FFFFE780C0FA97004B
:1071F0000000E780201E97000000E780001983A7A9
:107200000408170500001305C5C5829797C7FF1F1F
:107210002386A76CBC4C13060064854582979700B3
:107220000000E78000EA97B0FF1FE780A06F0145EC
:107230008280B7F7070003C70701A547AE8663162C
:10724000F7009397450191C301A0AA850146254502
:1072500017C3FF1F6700A3A94111B2862E86AA8516
:107260002D4506C697C0FF1FE78060A8B2400145C4
:10727000410182809307000463E8C7021D71A2CC1C
:107280002A84080886CE32C697800100E78040989D
:10729000B2461008A285294597C0FF1FE78020A5A8
:1072A000F64066442561828039558280411105454A
:1072B00006C697C0FFFFE7804026B24097F7FF1F42
:1072C00023AA079241018280B7E70400FC5F4111C5
:1072D00022C406C62A8482979307803EB307F4022D
:1072E00013071027B3D7E7023E9597F7FF1F938741
:1072F00067909C43B307F5406356F00097F7FF1F74
:1073000023AAA78EB240224441018280011106CEF9
:1073100022CC26CA97100000E780E073814729E15C
:1073200017D7FF1F0347873F85471DEBA3070100C2
:10733000B7E4040083A784179305F10013055030C8
:1073400082970DE58347F10095C397F7FF1F938759
:10735000678A8043FC5C82973305A440932715001D
:10736000F2406244D2443E85056182808147CDBFB0
:10737000371700408357E709C18B81C7C147231FD7
:10738000F7087300203041110D658D4506C697C082
:10739000FFFFE78020FBB71700408D6623A6D70AC2
:1073A00017F5FF1F130545851387C70A9387870ABB
:1073B0001CC15CC5856689675CC958C114C518C9FC
:1073C000B7E70400B24003A3871E41010283828015
:1073D00097F7FF1F83C7C78399EF411106C6971020
:1073E0000000E7806061B240854717F7FF1F230167
:1073F000F78241018280828011C589C517C3FFFFD2
:107400006700633C8280411126C2AE848D4522C450
:1074100006C62A8497C0FFFFE78020FDB71700400B
:1074200099C803A5C70C418D23A6A70CB2402244DE
:1074300092444101828003A5870C418D23A4A70CAF
:10744000F5B78347050003471500A207D98FC20788
:107450006177C18713072720639AE70083452500DA
:107460003705040017030000670023FA828017E63F
:10747000FF1F1306267A8147B2861303F00FA9482F
:107480003308F6000348080013F7F70F6307A80C4A
:10749000630668008507E39517FF2947B387E60071
:1074A0002380A70097E7FF1F938787775DA8411187
:1074B00013D765001347170006C693F63500058BF2
:1074C000954791CA054699476387C60009469D4777
:1074D0006383C600A14713F645003336C00093F618
:1074E0008503050685C2A145638BB604E145638A21
:1074F000B604930580026388B60493058003639302
:10750000B600914697F5FF1F2381F59897F5FF1F69
:10751000238CC59697F5FF1FA388D596BE8517A522
:1075200001001305251197700100E780C079B24072
:10753000854717F7FF1FA30AF7944101828085460C
:10754000D1B78946C1B78D4675BF17A50100130590
:10755000E510177301006700037717E7FF1F130794
:10756000276CBA972380B700E147E302F5F493074D
:107570007002E30CF5FC82802A8723800500814796
:1075800017E5FF1F130505691308F00F2946B30619
:10759000F50083C606006396E60297E6FF1F938612
:1075A0002668B69783C7070005452380F5009947ED
:1075B000636EF7029D4763FDE700E147630DF70047
:1075C0008280638506018507E393C7FC0145C5B743
:1075D000238005008280B737004003C7370083C788
:1075E000050093F70704D98F2380F5008280797115
:1075F00026D24AD097F4FF1F83C4049B17F9FF1FBC
:107600001309C99906D622D44ECE52CC56CA5AC8AE
:10761000B307990083C7070093F7F70FA5C79387B0
:10762000140093F7F70F0D476361F70C17F7FF1F6F
:10763000230CF79697F7FF1F9387C796A69783C7E4
:1076400007001307100293F7F703638FE7286363BC
:10765000F70A054463808720E389076E0947638939
:10766000E71413070002E38EE758B7E700E0370797
:10767000400023A0E71801000100CA942380040001
:1076800023A0E710B787004003C76700058BE30F0F
:10769000077897F6FF1F83C646910547E39AE6767B
:1076A00029472381E70209472383E7022385E7026D
:1076B00097E7FF1FA38C077C97F7FF1FA387078E11
:1076C000B7870040A381070017E7FF1FA302077CCD
:1076D00005472383E700B250225492540259F249DD
:1076E000624AD24A424B4561828097F7FF1F238D41
:1076F000078A89B7130730026386E70A63E6E7144F
:1077000013074002638AE70813070003E39FE7F4C7
:1077100097F7FF1F9387C788A69703C70700A1475E
:107720001377F70FE31AF71C17EAFF1F130A0A5023
:1077300083476A0097E6FF1F2380F67497E7FF1FD1
:1077400083C7374F91C7FD5797E6FF1F2386F67211
:1077500097E5FF1F83C5954D97E7FF1FA38EB77071
:1077600097E7FF1F83C7874C93F907089306000428
:1077700093F707066393D7529307A009638DF51A11
:1077800063EAB7169307F005638AF54E930750092D
:107790006388F52E014479ABFD5717E7FF1F230CD3
:1077A000F76CE1B5FD5717E7FF1F2305F76C75BDB3
:1077B00017A50100130505FC97700100E78080689C
:1077C00097E7FF1F9387C77DA69703C407008149EA
:1077D00017EAFF1F130A0A5E1374F40F97AA010039
:1077E000938ACAF963C78904294597700100E78025
:1077F0006052854717E7FF1FA30CF75A17E7FF1FD3
:107800002309875A17E7FF1F2302F76837E700E0CD
:10781000B70640002320D71801000100378600403A
:107820008347A60293F7370F2305F6022320D710CC
:107830002DBDB3073A0183C50700568585099770AA
:107840000100E780404879BF854717E7FF1F230104
:10785000F75621BD17A501001305C5F1977001006A
:10786000E780405E97E7FF1F93878773A69703C45F
:107870000700814917EAFF1F130A8A471374F40FA0
:1078800097AA0100938A8AEF63C5890429459770F6
:107890000100E7802048854717E7FF1FA308F7444A
:1078A00017E7FF1F2305874417E7FF1F2300F75E35
:1078B00037E700E0B70640002320D7180100010099
:1078C000378600408347660293F7370F2303F6029B
:1078D000B1BFB3073A0183C5070056858509977084
:1078E0000100E780403E4DB7854717E7FF1F230F94
:1078F000F73EA5BB9307400A638DF5349307200B31
:107900006388F5369307100AE396F5E883072A00A3
:10791000014463D1074297E7FF1F83C7573193F6AE
:107920003700638E061A0546638EC62209466399A0
:10793000C61A1D4775A217E5FF1F0345452FC94706
:1079400017EAFF1F034ABA2E97E5FF1F83C5452E8E
:1079500017E4FF1F0344D42D6319F510CD476316B8
:10796000FA1093077008639CF5021307300FB717DE
:107970000E006308E4001307900DB7B7040063140A
:10798000E40817E7FF1F232FF74EBE8517A5010058
:10799000130545DF97700100E780E032E5BB9307F0
:1079A0008008639DF50033048040B7774600137468
:1079B000F40F938787CDB3D78702E1B79307900879
:1079C000639AF5003304804091671374F40F938732
:1079D000C766D5B79307A008639BF50033048040C2
:1079E000B7173D001374F40F93870790E9B7930717
:1079F000B008639AF5003304804091671374F40F64
:107A0000938797D04DBF93F5F5078D47639BF5009E
:107A100033048040B7975B001374F40F938707D843
:107A200059BF8947639BF50033048040B7770B004B
:107A30001374F40F9387071BBDBF8547639AF50046
:107A400033048040DD671374F40F938767E3A5B7B1
:107A500089E9330480408D671374F40F938777DCD2
:107A600099BFF1679387072029BF97000000E7803F
:107A700040A0A285528597000000E780809F19BB37
:107A80009305610017E5FF1F0345651A17E4FF1F03
:107A90000344F41997000000E78040AE930571009D
:107AA000228597000000E78060AD3C0017E7FF1FCC
:107AB0002324F74E834761002304F10083477100BC
:107AC000A304F100894717E7FF1F2307F73A8357FD
:107AD000810017E7FF1F231BF7140944A1AC1547CA
:107AE00093F64700B336D00093F78703850685C326
:107AF0002146638BC7066146638AC7061306800268
:107B00006388C706130680036393C700914717E68F
:107B1000FF1F230BD63697E6FF1FA387F63697E79E
:107B2000FF1F2384E73617E7FF1F0347671093768D
:107B3000070497E7FF1F83C7B70F8DEE1377770C06
:107B400093067008630CD7021377F7078D46631E00
:107B5000D70AB307F040B7955B0093F7F70F93850B
:107B600005D881A81947ADBF854755B7894745B79F
:107B70008D4771BF930670086311D7021307300F4A
:107B8000B7150E006389E7021307900DB7B504001F
:107B90006383E7021307700845BF9306800C6311E7
:107BA000D702B307F040B775460093F7F70F9385F8
:107BB00085CDB3D5F50297E7FF1F23A5B72CF9B301
:107BC0009306900C631AD700B307F040916593F7C2
:107BD000F70F9385C566F1BF9306A00C631BD70012
:107BE000B307F040B7153D0093F7F70F9385059065
:107BF000C9B79306B00CE319D7F4B307F040916509
:107C000093F7F70F938595D06DB78946631BD7001F
:107C1000B307F040B7750B0093F7F70F9385051B7B
:107C200049BF8546631AD700B307F040DD6593F777
:107C3000F70F938565E3B5BF09EBB307F0408D659A
:107C400093F7F70F938575DCADB7F1659385052044
:107C50009DB783472A00C18B99C7854717E7FF1F48
:107C6000230FF72005BE97E7FF1F238A07201DB6C5
:107C7000854717E7FF1FA30AF72029BE3C0017E737
:107C8000FF1F232BF7300947930700032314F1004C
:107C900097E6FF1F2382E61E2DBD639A0758A9476A
:107CA00063ECB74417A70100130707968A05BA9536
:107CB0009C41BA97828717E4FF1F034454F7094A8F
:107CC000630C440F636C8A0885476309F40A9307C1
:107CD000F00F17E7FF1F0347271A63F6E70017E7C0
:107CE000FF1F230BF71817EAFF1F034AEA18930731
:107CF00000041374FA0F63F447011304000497E7B8
:107D0000FF1F9387672983AA0700228617E5FF1FB5
:107D10001305C5F1D685330A8A40A29A97700100EF
:107D2000E78000EF97E7FF1F2388471597E7FF1FBE
:107D300023A4572797E7FF1F83C717141547639A94
:107D4000E762B7E700E03707400023A0E71801002B
:107D50000100B7860040238086028DA58D47630C05
:107D6000F40A9947E315F4F697A701009387479023
:107D700017E7FF1F2322F722A947A1BF17E7FF1F1D
:107D80000347A72297E7FF1F93870711494697A547
:107D900001009385E5966306870097A5010093850A
:107DA00025923E8597700100E78080E617E7FF1F68
:107DB0002324A71EC94731BF97E6FF1F83C6E61ECF
:107DC000054797E7FF1F9387270D6394E6023E85DB
:107DD0001306700297A50100938505909770010026
:107DE000E78000E317E7FF1F2328A71A9307700215
:107DF000CDB53E851306300497A50100938505880F
:107E000097700100E780C0E017E7FF1F2326A7183F
:107E1000930730047DBD97E5FF1F83C545E117A596
:107E200001001305659797700100E780C0E9854A56
:107E300017EBFF1F034B6B1797E5FF1F83C525DF6C
:107E400017A501001305459563185B0B977001009A
:107E5000E78060E797E7FF1F83C767DDB5CBE3687F
:107E6000F4E617A401001304E48D638C670117A4E2
:107E700001001304A48D6386470117A401001304B5
:107E8000648E228597700100E78080041375F50FDA
:107E900093071500860717E7FF1F230FF7FE8D478F
:107EA00017E7FF1FA30AF7FE97E7FF1F9387C7FE99
:107EB0000147BE861376F70F89076365A60297E729
:107EC000FF1F23ABD70C97E7FF1F83C7E7FC11B554
:107ED00097A701009387078017E7FF1F232EF70A54
:107EE0009147C5BB3306E40003460600A3800700A4
:107EF00005072380C7007DBF97700100E780A0DCE5
:107F000097E7FF1F83C7A7D2E1D7E362F4DC17A48A
:107F1000010013042480638C57011794010013049B
:107F2000E47F6386470117A401001304A48022851F
:107F300097700100E780C0F91375F50F93071500DE
:107F4000860717E7FF1F2309F7F48D4717E7FF1F81
:107F5000A304F7F497E7FF1F938707F40147BE8652
:107F60001376F70F8907E37CA6F43306E400034693
:107F70000600A380070005072380C700D5B797E553
:107F8000FF1F83C5C5CA17A501001305A5819770FA
:107F90000100E78040D397E7FF1F83C7B7EF93E760
:107FA000470017E7FF1FA307F7EE83472A0017E7ED
:107FB000FF1FA30FF7EC6FF0EFFD179501001305FE
:107FC000A57F97700100E780E0E797E7FF1F9387A1
:107FD00027EC83C7070017E7FF1F2309F7C417E43F
:107FE000FF1F034464E933348000A9B317950100EF
:107FF0001305C57D97700100E780C0E497E7FF1F78
:1080000083C757E993E7070117E7FF1FA304F7E8C2
:1080100083472A0017E7FF1F230CF7E66FF08FF75F
:10802000179501001305C57B97700100E78080E17B
:1080300003470A007D8B51EFB787004003C76702F3
:108040001377C70B136727002383E70203C7A70231
:108050001377C70B136727002385E70203C7E702DF
:108060001377C70B136727002387E70203C727038C
:108070001377C70B136727002389E702854717E7A4
:10808000FF1F2305F7C617E7FF1F2303F7D217E7E4
:10809000FF1F2301F7DE17E7FF1F230EF7DC97E72B
:1080A000FF1FA38507C497E7FF1FA38307D097E7A8
:1080B000FF1FA38107DC97E7FF1FA38E07DA97E76F
:1080C000FF1FA38507DC97E7FF1FA38007EE6FF074
:1080D0006FEC89476312F70297E7FF1F83C747B525
:1080E0009146638CD70863E0F604638EE70C6369FE
:1080F000F70A05476380E70EFD5717E7FF1FA30D3B
:10810000F7D637074000B7E700E023A0E7180100E3
:108110000100B78600401306F0FC2381C60223A0AD
:10812000E7106FF08FD4130720086382E7086362BB
:10813000F70213071008E391E7FC378700408347F5
:10814000670293F7C70B93E727002303F7026FF04B
:108150006FE4130730086389E70213074008E39DC3
:10816000E7F8378700408347270393F7C70B93E768
:1081700027002309F7026FF0EFE1378700408347BC
:10818000270393F73707F5B7378700408347E702A0
:1081900093F7C70B93E727002307F7026FF08FDFF2
:1081A000378700408347E70293F73707F5B73787EC
:1081B00000408347A70293F7C70B93E727002305E7
:1081C000F7026FF02FDD378700408347A70293F750
:1081D0003707F5B7378700408347670293F73707BC
:1081E000ADB7179501001305A56097700100E780F2
:1081F00060C597E7FF1F238B07A2D5B31795010032
:108200001305056097700100E780C0C397E7FF1F63
:10821000239E07A097E7FF1F938707C603C40700A5
:10822000894763F3870009441374F40F21B61307D9
:108230000002E393E7EC6399090A638FF500930763
:1082400020026381F508179501001305E55E97701C
:108250000100E78040A74DB5179501001305055BA8
:1082600097700100E78000BE0144179B0100130BCB
:108270002B5BA14AB3078A0083C507005A85050412
:1082800097700100E78020A4E31654FF17950100C2
:108290001305C5B797700100E780C0BA17E4FF1F48
:1082A0000344049911E497E7FF1F2384079659B408
:1082B0008947E313F4E4854717E7FF1F230BF7947F
:1082C0006FF04FCD17E6FF1F0346769697E5FF1F29
:1082D00083C5E595179501001305055597700100B5
:1082E000E780609E6FF00FCB638FF5049307100259
:1082F000E39BF5F497E5FF1F83C585931795010070
:108300001305855497700100E780E09B97E7FF1FF6
:1083100023A447C997E7FF1F9387C7B6944383D722
:10832000470017E7FF1F034747B617E6FF1F232F36
:10833000D68E1D4497E6FF1F239CF68E97E7FF1FFE
:108340002389E78EC5BA97E5FF1F83C5658E17950C
:1083500001001305E55097700100E780C09697E78C
:10836000FF1F2388078A97E7FF1F2391078C6FF071
:10837000CFF62547E387E79C19476391E702B78665
:10838000004023808602B7E700E03707400023A0C3
:10839000E71801000100130600FC41B31307100A9F
:1083A0006391E702B786004023808602B7E700E0CA
:1083B0003707400023A0E71801000100130680FCE6
:1083C000A9BB1307A009E38FE7FC1307400AE38B5F
:1083D000E7FC13072002E386E7960547E383E79669
:1083E000B7E700E03707400023A0E718E3910996BC
:1083F00001000100B786004023808602130620FC9E
:1084000029BB17E7FF1F034737A76308F71E63E77A
:10841000E7029547630EF70E99476308F704B7869E
:10842000004023800602B7E700E03707400023A0A2
:10843000E718010001001306A0FCC5B19307F00581
:10844000630AF700930750096306F70093071002C9
:10845000E317F7FCB7E700E03707400023A0E71871
:1084600001000100B786004051BF97E9FF1F83C993
:10847000A9A093070004CE8A63F43701930A00048D
:1084800097E7FF1F938747B103AA070013F4FA0F7A
:108490002286D28517D5FF1F130545799760010005
:1084A000E7800077B3878940529417E7FF1F2305C1
:1084B000F79C97E7FF1F23A187AE638E0902B7875A
:1084C000004023805703B7E600E03706400023A0B2
:1084D000C6180100010003C72702134707042381C0
:1084E000E70203C727021377C70F2381E70223A000
:1084F000C6106FF08F97B786004023800602B7E75B
:1085000000E03707400023A0E71801000100FDB597
:10851000378700408347370097E6FF1F83C656978B
:1085200093F70708D58FA301F700B7064000B7E718
:1085300000E023A0D718010001001306A0FC2301CE
:10854000C70223A0D7106FF04F9297E7FF1F9387C2
:1085500027A5A69783C7070093F7F70FD9CF97E70B
:10856000FF1F83C787A4D1EB17E7FF1F0347D790EF
:10857000930700026313F70897D7FF1F9387076BD2
:1085800003AB070097DAFF1F83CA8A6A17DAFF1F57
:10859000034A1A6A97D9FF1F83C9A969D2875687E8
:1085A000CE865A8697D5FF1F83C5A566179501000D
:1085B0001305852C97600100E780E07097E7FF1FA7
:1085C00023A2678D97E7FF1F2380578D97E7FF1F33
:1085D000A38C478B97E7FF1F2389378B97D7FF1F04
:1085E000A3888762B7E700E03707400023A0E718B9
:1085F00001000100B7860040D1B3B7E700E03707BC
:10860000400023A0E71801000100B786004025B50F
:1086100029472381E70209472383E7022385E702ED
:108620002387E7022389E7026FF08F8803C767007B
:10863000118B6302078A83C75700918BB5CF17E769
:10864000FF1F0347879685476313F70697E7FF1FCA
:10865000A38DE78297D7FF1F238A076897D7FF1F4D
:108660002388077497E7FF1F2386078097E7FF1F7C
:108670002383078097D7FF1FA38A076697D7FF1F1B
:10868000A388077297D7FF1FA386077E97D7FF1F80
:10869000A383077E97D7FF1FA38A077E97E7FF1F55
:1086A000A3850790B787004011476FF08F8217D7D7
:1086B000FF1FA30FF75479BF854717D7FF1F230765
:1086C000F76217D7FF1F2305F76E17D7FF1F230386
:1086D000F77A17D7FF1F2300F77A69BF854717D7A7
:1086E000FF1F2305F76017D7FF1F2303F76C17D76A
:1086F000FF1F2301F77817D7FF1F230EF77617D731
:10870000FF1FA305075E17D7FF1FA303076A17D72D
:10871000FF1FA301077697D7FF1FA38E07748280E0
:10872000411106C697000000E78080FBB787004034
:1087300023800700130740FC2386E7001307C004CB
:10874000A386E70017D7FF1F1307474E2398E700BC
:1087500017D7FF1F13078751239AE70017D7FF1F6B
:108760001307075D239CE70017D7FF1F13078768D0
:10877000239EE70029472381E70209472383E70275
:108780002385E7022387E7022389E702A381070005
:10879000930600F8A380D700930690022380D700A9
:1087A000FD562383D7002381E700B706400037E753
:1087B00000E02320D71003C7170013671700A3801A
:1087C000E700B24097D7FF1F2394076C41018280D6
:1087D000411106C697000000E78080F0B78700408F
:1087E00023800700130700FC2386E7003147A38698
:1087F000E70017D7FF1F130767432398E70017D732
:10880000FF1F1307A746239AE70017D7FF1F130779
:108810002752239CE70029472381E7020947238346
:10882000E7022385E702A3810700930600F8A380EF
:10883000D700930690022380D700FD562383D700EC
:108840002381E700B706400037E700E02320D71078
:1088500003C7170013671700A380E700B24097D73C
:10886000FF1F2397076241018280F16793870720EA
:1088700017D7FF1F2328F760854717D7FF1F23153A
:10888000F760A14717D7FF1F2301F76097D7FF1F96
:10889000A38D075E97D7FF1F238A075E97D7FF1F19
:1088A0002389073697D7FF1FA3840736814717D53B
:1088B000FF1F13052536FD5517D6FF1F1306463635
:1088C0002947B306F5002380B600B306F6002380DF
:1088D00006008507E397E7FE97D7FF1F2380076C05
:1088E00097D7FF1FA38C076A97D7FF1F2389076AB3
:1088F00097D7FF1FA383075897D7FF1FA381075858
:1089000097D7FF1F238C075697D7FF1F238707563C
:1089100097D7FF1F2386075697D7FF1FA3800756B9
:1089200097D7FF1F238D075497D7FF1FA38907668B
:10893000828017D7FF1F0347476785476316F700F5
:1089400017030000670003E917030000670083DDD9
:10895000411122C406C617D7FF1F03470765854785
:108960002E8613F4F50FAA856317F70417D5FF1F9A
:108970001305054097600100E780802997D7FF1F06
:1089800023880742B787004023848702B7E600E0C8
:108990003706400023A0C6180100010003C7A70244
:1089A0001377C70F2385E702B240224423A0C610E5
:1089B00001454101828017D5FF1F1305252F9760C0
:1089C0000100E780E02497D7FF1F23810732B78794
:1089D000004023828702B7E600E03706400023A06C
:1089E000C6180100010003C767021377C70F23836E
:1089F000E7025DBF411106C697000000E78020E74F
:108A0000B2404101170300006700E3F2411106C6BE
:108A100097F0FFFFE780E0BD97D7FF1F83C7172DB3
:108A200095C797D5FF1F83C5852C89C917D5FF1F0B
:108A30001305052C97F0FFFFE780409C97D7FF1F99
:108A4000A386072A97D7FF1F23820744B24041011C
:108A5000828017D5FF1F0345A5433335A0008280D0
:108A600041C9D9C597D7FF1F83C78742D1C3011119
:108A700022CC4AC84EC656C25AC006CE26CA52C4D6
:108A80002E89AA890144930A0004371B03006377E7
:108A90002403B3078940C207C183BE8463F4FA008C
:108AA00093040004C204C180130A1BD497D7FF1F8C
:108AB00083C7C7239DE37D1A631C0A00F24062440A
:108AC000D2444249B249224A924A024B056182800D
:108AD00097F0FFFFE780E0B1D1BF3385890026948E
:108AE000A685420497000000E780C0E6418045B7B4
:108AF000828097D7FF1F9387E74E18429C4383D607
:108B000045000345070083C5C7000356460063962A
:108B1000A50083D5E700638DD502011106CE23861B
:108B2000A7002397D700B705CF00DC4B9385757D51
:108B300005077D162EC2230001003AC42316C1008A
:108B40002317D10099C30A858297F240056182807C
:108B50008280DC4DDC4B81CFB7E70400904503A356
:108B60008705914517D5FF1F03450548028382807D
:108B70006D713C083EC6B707E500232291103EC840
:108B8000AA843C083285232611103ECA2324811072
:108B9000232021112E8997300000E780205D2A8450
:108BA000979501009385C5D017850100130545BF32
:108BB00097600100E7802011A28517950100130539
:108BC000A5DF97600100E78000102945976001004C
:108BD000E7804014B705CB009385757D680097103A
:108BE0000000E7804066A285680097300000E780BB
:108BF000404A014781467000CA85268597200000BB
:108C0000E780C08905CD2A8497950100938545CAE0
:108C1000178501001305C5B897600100E780A00A19
:108C2000A285179501001305E5D997600100E7803B
:108C30008009294597600100E780C00D8320C1109D
:108C40000324811083244110032901105161828083
:108C500097D7FF1F9387073918429C43797122D415
:108C600006D60348070083C807012A8483D6450037
:108C7000035546006396080183D82701638DD80207
:108C80002388070105072399D7003708CC00DC4B60
:108C90001308787D3ACC1307F5FF42CA2308010078
:108CA000231EE100231FD10099C7080832C62EC435
:108CB00082973246A245228597000000E78080EB2C
:108CC000B2502254456182806D713C083EC0B707A6
:108CD000E5003EC23C083EC4232611102324811027
:108CE00023229110231701002318010023190100EA
:108CF000231A0100231B010097B7FF1F83D787C0EA
:108D000099E3C167FD172316F10097B7FF1F83D7BB
:108D100087BF91EB97D7FF1F9387C72C9C439C433A
:108D2000DC4783D7070017B4FF1F1304A4BD584CBA
:108D30002317F10083574400484B2318F10031E119
:108D4000979501009385C5BD17850100130545A5BD
:108D500097600100E78020F717950100130585BD96
:108D600097600100E78020F6294597600100E780C1
:108D700060FA8320C11003248110832441105161C3
:108D8000828097B7FF1F83C757B889EBB7E7040006
:108D9000BC5782975C4C23AA0700E1BFFD1797B62A
:108DA000FF1FA384F6B603560701834704014C470F
:108DB0000A85230BF10097300000E780A02A97D79F
:108DC000FF1F938727229C430147814688430A86D9
:108DD0006C0097100000E780606CAA8429C1979509
:108DE00001009385E5B3178501001305659B976026
:108DF0000100E78040EDA68517950100130545B4F5
:108E000097600100E78020EC294597600100E7802A
:108E100060F0584CB7E70400BC57484B9DBF97B76C
:108E2000FF1F83C797AEF5D7B7E70400BC4F1044C8
:108E3000854517D5FF1F0345251B82971DBF5C4E37
:108E4000DC4BB9CFB1CD411122C417850100130508
:108E500025952E84979501009385C5AA06C697602F
:108E60000100E78040E6A28517950100130505B0D3
:108E700097600100E78020E5294597600100E780C1
:108E800060E9B7E704002244B24003A3870517D581
:108E9000FF1F0345651513064006914541010283F6
:108EA0008280411122C417B4FF1F130464A31C4C19
:108EB00006C689C7DC4399C34C488297584CB7E72C
:108EC0000400BC57484B82975C4CB240224423AA12
:108ED00007004101828017B7FF1F130767A283476E
:108EE00007009306F00B850793F7F70F63E9F60089
:108EF00097B6FF1F2386F6A00345070082809307DD
:108F000000F8FDB7835745006386071001114AC872
:108F100017B9FF1F1309099F52C4032AC90106CEBE
:108F200022CC03274A0126CA4EC656C2F15735E362
:108F30001307D00DFD57636EC704B7E9040083A77C
:108F400009072A841305860042054181B284AE8A4E
:108F50008297232AAA000325C9015C49A9E79795AE
:108F60000100938525981785010013056583976097
:108F70000100E78040D517950100130565A79760AC
:108F80000100E78040D4294597600100E78080D840
:108F9000DD57F2406244D2444249B249224A924AE1
:108FA0003E850561828093874400B705CF00231971
:108FB000F5009385757D310597100000E780A028A6
:108FC0000325C90183456400310597300000E7801F
:108FD000400C0325C9012686D6853105973000004F
:108FE000E78040087146A2854A8597600100E780C6
:108FF00020C2504419CA83A78905854517D5FF1F8C
:10900000034585FE8297814769B797000000E78096
:10901000E0CBD5BFFD573E858280411126C297B473
:10902000FF1F9384248ED84C22C437E404003C54A0
:10903000484B06C68297DC4C0323C4052244B24049
:10904000924423AA070017D5FF1F0345E5F985457C
:1090500041010283411126C297D4FF1F938484F8F3
:109060009C4006C622C44AC0D5C3DC43C5C35CC10C
:109070002300B5002A84979501009385E581177533
:1090800001001305E57197600100E780C0C3294521
:1090900097600100E78000C89C4023A4070023A23A
:1090A000070097B7FF1F9387A783DC4FDC4B91C75F
:1090B000295597000000E78000DF97B7FF1F9387CF
:1090C0006784DC4FDC4B89C797000000E78020F500
:1090D00037E904008327C905894517D5FF1F0345D4
:1090E000A5F082978327C905914517D5FF1F034532
:1090F000A5EF82979C4003A34701630903002285E3
:109100002244B2409244024941010283B2402244C7
:1091100092440249410182800111328506CE22CC5F
:1091200026CA2E8497300000E7804004AA849785E1
:1091300001009385A5791775010013056566976091
:109140000100E78040B8030784000356640083559C
:109150004400A6861795010013054583976001001A
:10916000E78060B6294597600100E780A0BA97A71D
:10917000FF1F83C74777639D970001459700000055
:10918000E78060D281450A8597000000E780C0EC47
:10919000F2406244D244056182806D7123248110C3
:1091A000232611102322911093F745002E84638704
:1091B00007143C083EC0B707E5003EC23C083EC469
:1091C000231701002318010023190100231A0100AD
:1091D000231B010097A7FF1F83D7877099E3C167FF
:1091E000FD172316F10097A7FF1F83D7876F91EB19
:1091F00097D7FF1F938707DF9C439C43DC4783D7A8
:10920000070017A7FF1F1307A76D2317F100544F7F
:10921000835747002318F100DC4AA1E79785010036
:109220009385056F17750100130585579760010039
:10923000E78060A9178501001305C56F97600100DD
:10924000E78060A8294597600100E780A0AC13453E
:1092500044008320C11003248110832441105161F4
:10926000828097A7FF1F83C717682555D9C3FD17AD
:1092700017A6FF1FA309F66603D606018347070159
:10928000CC460A85230BF10097300000E78080DD93
:1092900097D7FF1F938707D59C4317A7FF1F130777
:1092A0002764978601009386E66B88430A866C00E4
:1092B00097100000E780801EAA8451D9978501008D
:1092C00093850565177501001305854D97600100AD
:1092D000E780609FA6851785010013056566976086
:1092E0000100E780409E294597600100E78080A249
:1092F000268597000000E78000BB91BF93F725000B
:109300009DC7B7E70400BC474146814528088297BE
:10931000255597000000E78000B928089305F00F55
:1093200097000000E78040D3134524001DB793F752
:109330001500014599DF97000000E780209913454B
:10934000140001BF5C4D411106C688C317D7FF1F2B
:10935000232AF7C8B7E7040083A70708170500000A
:109360001305E5E38297B24097D7FF1F238EA7C668
:1093700001454101828001119307700F2316F1000E
:1093800006CE97D7FF1F83C7B7C78DE7B7E704009F
:1093900083A7870D17A6FF1F0346C6596C0017D574
:1093A000FF1F035525C682973335A00097D7FF1FAF
:1093B000A388A7C4F24005618280411193970501FB
:1093C00022C406C626C2C1872E8463D40702B7E42E
:1093D0000400FC5417A5FF1F0345C555829719C10A
:1093E000BC5482972165218DB240224492444101B0
:1093F000828093F715008DC7B7E7040083A7471A4B
:1094000017A6FF1F1306065297D5FF1F938585BE2B
:1094100017A5FF1F03450552829713451400E9B7AE
:1094200093F7250099CFB7E70400BC4F13060064FB
:10943000894517A5FF1F0345E54F82971345240073
:1094400065B793F785009DC7B7E7040003A8871A9F
:109450001307401F97A7FF1F83C7C74D89461306F1
:109460000003E14517D5FF1F0355C5B90298134501
:1094700084009DBF93F745000145BDD7B7E40400C4
:1094800083A7041817D5FF1F0355C5B78297BC4C97
:1094900013060064914517A5FF1F0345A549829750
:1094A0001345440091B797D7FF1F83D7A7B563989B
:1094B000A70217D7FF1F2318B7B417D7FF1F23150D
:1094C000C7B417D7FF1F2312D7B42E861785010004
:1094D00013050569BE85175301006700C37E178514
:1094E000010013056569176301006700A395035721
:1094F0004500011106CE22CC97D7FF1F83D787B036
:1095000017850100130545676310F706C167F91752
:1095100017D7FF1F2328F7AE37E4040097D7FF1FA4
:1095200023A407AE7C4C894517A5FF1F0345854042
:1095300082977C4C914517A5FF1F0345A53F829755
:1095400097B7FF1F83C7971D85CB8547A307F100FA
:10955000832744171306F100854513055030829781
:10956000178501001305855597600100E780808D00
:10957000F24062440561828097C7FF1F83C7475A44
:109580001785010013054558E5F38547A307F1004A
:10959000832744171306F100854513055030829741
:1095A000178501001305C553C1B77D15954763E7BE
:1095B000A71C178701001307274D0A053A951C4180
:1095C000011122CC06CE26CABA972E84828717852F
:1095D00001001305E55A97600100E780A08691A27B
:1095E00003C7250099476311F7022E8597000000F5
:1095F000E78020F083456400178501001305455975
:1096000097500100E780206C0965130505F497B7B2
:10961000FF1F2385071097E0FFFFE78020CB17850A
:1096200001001305A55845BF03C7250095476319D9
:10963000F702C16717D7FF1F0357C79CF91703D558
:10964000A5006309F702B7E7040083A7C71782974D
:10965000178501001305855697500100E780807E2D
:10966000854717B7FF1F230BF70A1785010013055E
:10967000655795B797D7FF1F2396A79883D7E5001F
:10968000B7E40400096617D7FF1F231EF79683D798
:1096900005011306069017A5FF1F0345A52917D737
:1096A000FF1F2313F79683D72501A14517D7FF1F67
:1096B000231DF794BC4C8297BC4C13060064914563
:1096C00017A5FF1F0345052782970356E40083551E
:1096D000A400178501001305A54F97500100E780EE
:1096E000805EBDBF1785010013058550EDB583C5AC
:1096F00025009147639CF5028547178501001305F6
:10970000A550A307F10097500100E780A073B7E7C9
:10971000040083A747171306F10085451305503051
:109720008297F2406244D2440561828099476392F5
:10973000F502228597000000E780A0DB83456400E6
:10974000178501001305C54497500100E780A05715
:10975000C9BF9547639FF500834714001785010033
:109760001305854AE39907E6178501001305854B24
:109770009DB5178501001305654BF9B782806D71A2
:10978000232481102326111023229110328401CD2D
:109790008947630AF5028320C110032481108324C2
:1097A000411051618280178501001305E548AE84A0
:1097B00097500100E7800069A285268597C0FFFFCA
:1097C000E7802056C9BFB7E70400FC47280082970E
:1097D000178501001305054797500100E780806653
:1097E0008347810039C41307000B6380E7021387A6
:1097F000A7051377F70F8D4663EDE602A2852800D3
:1098000097D0FFFFE78000C579B78547E3F587F874
:1098100083459100177501001305C52DB335B000C0
:1098200097B7FF1F238EB7D697500100E780A04956
:109830009DB703479100A207D98F35671307D75506
:109840006385E7086368F7022D671307B7556387D9
:10985000E70631671307C755638AE70429671307CB
:10986000A7556394E702A285280097D0FFFFE78001
:1098700040F815B739679306E765638DD70663E946
:10988000F6001307E7556380E706A28528003DB779
:109890003D679306F7556386D7061307F766E39689
:1098A000E7FE97D0FFFFE780C010F5B50146A2851F
:1098B000280097D0FFFFE78000E1F1BDA2852800D6
:1098C00097D0FFFFE78020F1F9B58947E3F587ECF2
:1098D0009305E4FFC205C1811305A10097A0FFFF16
:1098E000E78060EE4DBDA285280097D0FFFFE7809E
:1098F00040F155B5A285280097D0FFFFE78000FC16
:1099000059BD97D0FFFFE780800471B5411122C493
:1099100017A4FF1F13044403AA8617860100130629
:1099200026182285C14506C697500100E780C0521F
:109930000357440097A7FF1F938707022393E7006D
:10994000035764002394E700B2402244410182801F
:10995000011106CE22CC97000000E78060FB37E4BF
:1099600004008327841417A6FF1F1306E6FDD545C0
:1099700001458297832784179305F1001305503022
:1099800082978347F100A1C7A307010083274417EB
:109990001306F1008545130550308297832744173D
:1099A00017A6FF1F130646FBCD451305703082979F
:1099B0008547A307F100832744171306F100854567
:1099C000130550308297F2406244056182808327FC
:1099D000441717A6FF1F130626F8CD451305703050
:1099E000D5B761712324811A37E404008327040862
:1099F0002326111A2322911A2320211B232E3119E9
:109A0000170500001305A59B829717A9FF1F1309CF
:109A100069F2994785442300A900231CF10097852A
:109A200001009385E51093074006177501001305A3
:109A300025D7231CF1082308910097C9FF1F93899C
:109A4000091B97500100E780002883D5090017857E
:109A500001001305A50597500100E780C0262945A0
:109A600097500100E780002B03D509008569970016
:109A70000000E780E0E983274417100885451305B7
:109A8000503082978327441717A6FF1F1306C6EC92
:109A9000CD451305703082978327441717A6FF1F03
:109AA000130686E9B545130560308297832744176E
:109AB00030088945130510318297832744173009F0
:109AC000894513052031829783274415938509C85A
:109AD0000D45829783274415938509C811458297C0
:109AE000A3059100230691002308910002CD230CC9
:109AF0000100832784163009914513057040829731
:109B0000832784161306B10085451305004082970C
:109B1000832784167000854513051040829783279C
:109B200084163008854513052040829783278416C4
:109B300010088545130550408297832704157D55ED
:109B40008297832744137D5582977D5597A0FFFF09
:109B5000E78020128327440C829797A0FFFFE780BD
:109B600060ED8327841417A6FF1F1306E6DDD54595
:109B70000145829789471306700F814528092306FE
:109B8000F1009790FFFFE78040A98D47130600087A
:109B900081452808230CF1089790FFFFE780E0A794
:109BA0009147230CF100977701009387E7B0984322
:109BB00083C747003AC8230AF10097D0FFFFE78028
:109BC00000E670008545054597A0FFFFE7808011FE
:109BD00030099305700F094597A0FFFFE7808010BB
:109BE0003008930500080D4597A0FFFFE780800F20
:109BF00010089545114597A0FFFFE780A00EC167AB
:109C000017C7FF1F13070740F9171CC323220700BC
:109C100017A5FF1F1305C5D197A0FFFFE780600BB5
:109C20008327C41D17C5FF1F1305453C82973C4879
:109C300003450900854582978320C11A0324811AB0
:109C40008324411A0329011A8329C1195D61828085
:109C5000C16717C8FF1F0358E83AF9176301F808EE
:109C60003DCDB5CD011126CAB7E4040083A7841207
:109C700022CC2E862315B10006CE2A8401478146C8
:109C8000ED45428582972AC611ED1785010013051F
:109C900025EB97500100E780E01AF2406244D2447D
:109CA00005618280FC440356A100A28582972C00A6
:109CB00017C5FF1F0355053597A0FFFFE780200E4E
:109CC00069DD178501001305E5E897500100E7807D
:109CD000601783A7C412ED45280082977DBF82805C
:109CE000011106CE22CC2DC9854717A7FF1FA30A55
:109CF000F7C497A7FF1F238707C437E4040083270F
:109D000084179305F1001305503082978347F100C3
:109D1000A9CBA3070100832744171306F10085454B
:109D20001305503082978327441717A6FF1F130689
:109D3000A6C0B5451305603082978547A307F1009B
:109D4000832744171306F100854513055030829789
:109D5000F24062440561828097A7FF1FA38307BE7C
:109D600049BF8327441717A6FF1F1306E6BCB54556
:109D700013056030E9BFC16717C5FF1F035585286C
:109D8000F9176307F500B7E7040003A3C7170283B9
:109D9000828001118547A307010017C7FF1F230118
:109DA000F726B7E7040083A7471706CE1306F1008E
:109DB0008545130550308297F240056182801793E4
:109DC000FFFFE702E3802A8408452E89B28919C97A
:109DD00000C1971500009385A586610597300100A5
:109DE000E780800181447D5A97100000E780E039C8
:109DF00063C7A404814497100000E780003A63C859
:109E0000A40497C7FF1F938767209C43DC47B307D1
:109E1000F94091872302F400638309048327C90072
:109E2000B307F4409587A302F4001C4C89C79C47F4
:109E300099C3228582971783FFFF6700A37C5C4448
:109E4000139714008504BA972390470171BF1C48EB
:109E5000139714008504BA972390070069BF8327DE
:109E600089000547B307F4409587A302F4008357A0
:109E70000400638EE7028DC309476384E7040D473E
:109E8000E395E7FA978701009387872E1CCC978785
:109E900001009387E72E11A8978701009387C7F4E5
:109EA0001CCC97870100938727F55CC8BDBF9787B7
:109EB0000100938767E01CCC978701009387C7E078
:109EC000EDB7978701009387672F1CCC9787010018
:109ED0009387C72FD9BF95E51783FFFFE702E3708C
:109EE000004618448347940075839D8B6317F700E1
:109EF00097100000E78060B448C41783FFFF670035
:109F0000037182801783FFFFE702836C138935009A
:109F1000C16442094111AA890144F114135909018C
:109F2000054A2EC697100000E7802026B2456348F8
:109F3000A400014541011783FFFF6700A36C83A7BD
:109F4000090013171400BA9783D707006388B70076
:109F50006394970063742A010504E1B70545D9BFEE
:109F60001783FFFFE702E365AA892E89328BB68447
:109F70003A8ABE8A97A00000E78020FB71C9268537
:109F800097200000E78020098D4763E7A7007D55F3
:109F90001783FFFF6700636683DB440097100000B0
:109FA000E780A0242A8497100000E78040259307CB
:109FB000740031443305850263CDA7029710000079
:109FC000E780A02297100000E78020222A849710C3
:109FD0000000E780C02293077400314433058502F6
:109FE00063C3A70497100000E78020209307450073
:109FF00029A897100000E780802033058502130709
:10A00000F0179307C017E35FA7FA2D55E3C277F95E
:10A0100063040B02D6865286A6854A8597200100E6
:10A02000E78020BAB5B797100000E780401D3305E0
:10A0300085029307C5FFD1BF832749001385C90057
:10A0400083D5270097000000E78000EC61F581B719
:10A0500069553DBF97C7FF1F239CA7FA97C7FF1FEE
:10A060009387C7FA904381470C463307F5004207B0
:10A0700041836393B7008280544613984700850755
:10A08000C2962390E600D5B797C7FF1F938707F8BE
:10A090009C4303C58700828017C5FF1F035545F702
:10A0A00082801783FFFFE7024354C1671387D7FFFE
:10A0B000630BE502636AA700F1176300F50201452F
:10A0C0001783FFFF6700A3541387E7FF6302E502CE
:10A0D000FD171D8D13351500E5B797500000E7807B
:10A0E000C0267D15C5BF97500000E78040FBD5BF57
:10A0F00097500000E78060F9EDB71783FFFFE70294
:10A10000C34E4111AA8401442EC697100000E78077
:10A11000C008B2456348A400014541011783FFFF11
:10A120006700E34E9C48131514003E9583570500C5
:10A13000E385B7FE0504C9BF03485500814693F780
:10A14000F60F63E5070181473E8582805845939766
:10A150005600BA9703D727006316B70003D7070046
:10A16000E304C7FE8506E1BF8346450001479377B8
:10A17000F70F63E4D700814711A81C451316570059
:10A180000507B29703D60700E313B6FE3E8582802B
:10A190001783FFFFE702C34393170501C18797CADF
:10A1A000FF1F938AAAE6635BF00883A70A00C047F3
:10A1B0009C4703570400198D420541816368F500EF
:10A1C000014422851783FFFF6700C34312052A94C9
:10A1D000CDBFDC4713944900014A3E9483474400B5
:10A1E0006341FA02014A834754006349FA02850930
:10A1F000C20993D9090183A70A009847E3EBE9FC58
:10A20000C1B71C4413195A00A6853E994A85970088
:10A210000000E780C0EE05E1050AC9B75C441319E8
:10A220005A00A6853E994A8597000000E78020EDF8
:10A2300019E1050A4DBFE30C09FA61B7AA84814907
:10A240005DBF1783FFFFE702433A1C452A8481E77D
:10A250009307C5001CC51C44231204001CC09307AF
:10A26000F00F63EDB70093F5F50F228597200000FE
:10A27000E78020E21783FFFF6700633993940501AD
:10A28000C167C18063F9F500A6852285972000008B
:10A29000E78040E5C5B7C18193F5F50F228597208A
:10A2A0000000E78000DFA685228597200000E78078
:10A2B00040E0C9B797C7FF1F938747D5884382807F
:10A2C0001C4599C797C7FF1F23A2A7D401458280C9
:10A2D0007D55828097C7FF1F938747D39843834755
:10A2E0004500484792073E9582801783FFFFE702AB
:10A2F000C32F617100451C183EC6B70780013EC8D8
:10A300001C183ECA8357440002CE02D002CC231E42
:10A31000F100834784002A8902D22301F1023C081C
:10A320003ED402D697000000E78000FB835705006B
:10A330002316F10297500000E78060C42307A102B2
:10A340005C4003556400F18313F717008347F10263
:10A3500052055181F99BD98FA307F1029710010093
:10A36000E780807539CDAA840355050097A00000C9
:10A37000E78080BC83D704002AD26800231CF10048
:10A3800083D72400231DF1001C4803D647008C43CB
:10A3900097200000E78000CD8347B400CA86178667
:10A3A00001001306E68A8117A305F4006C0048102B
:10A3B00097200100E780E0805D611783FFFF670061
:10A3C00003252155D5BF1C45B1CF03C5A70089463C
:10A3D00013576500630BD7028D46630ED70285467F
:10A3E0006300D702130740063305E50203C7B70031
:10A3F000418B15CB83C7B700BD8B3355F5408280A9
:10A400001375F5031307803EC5B709671375F50388
:10A4100013070771D1BF372709001375F503130719
:10A42000077CD9B7014582801783FFFFE702E31B52
:10A4300003A98500630C09048347B900AE8493F730
:10A44000070E85C303459900930520030D8105057B
:10A45000B305B5028844610597300100E780E0A9A3
:10A4600035A02E8597000000E78020F62A8419CDBC
:10A4700097000000E780605C8325C900B307B54002
:10A4800063FA87002E94B305A440E9F51783FFFF14
:10A490006700E31785457DBF1783FFFFE702E314DD
:10A4A0002A8403D50500011132C636C43AC22EC033
:10A4B00002CA02CC02CE97A00000E780E0A7824546
:10A4C0002ACA22852ECC97000000E780E0E00357DF
:10A4D0000500231EE10097500000E78040AAA24635
:10A4E00032469247230FA10036874C08B286228558
:10A4F000014697000000E780E0A605611783FFFF93
:10A500006700E3101783FFFFE702230E61711C1839
:10A510003EC6B70780013EC81C183ECA3C0800452D
:10A520003ED4AA8402CC02CE02D002D202D6970038
:10A530000000E78060DA8357050035592316F102E1
:10A5400097500000E780A0A32307A10209C4835706
:10A55000440081EB21594A855D611783FFFF670045
:10A56000030B035564005205518197100100E780E9
:10A57000A0542A8965D18347B40093F7070E99C781
:10A580001305840197300100E780609983574400E8
:10A59000231EF100834784002301F1025C40035530
:10A5A0000900D98313F7070883471102231CA10070
:10A5B00093F7F707D98FA300F10283572900231DD2
:10A5C000F1005C40F18313F717008347F102F99B18
:10A5D000D98FA307F10297A00000E780E0952AD267
:10A5E00035D9834794006800139757008347B40018
:10A5F000FD8BD98FA305F4001C4803D647008C437C
:10A6000097200000E78000A6A687177701001307B0
:10A610002764740005464C10268597000000E780EB
:10A6200060942A890DD98347B400A685FD8BA305C4
:10A63000F40097000000E78060DF31BF1783FFFF61
:10A64000E702A3FA832485FE2A8441112685970018
:10A650000000E78080D7834734FF93F7070E8DCB48
:10A660002AC6268597000000E78060C809CD834789
:10A6700034FFB245FD8BA309F4FE91C522859730C6
:10A680000100E780808741011783FFFF670023F8FF
:10A690007DD98327C4FF2685829775F5834734FFCC
:10A6A00093F7070E91C7228597300100E780208736
:10A6B000032584FE97000000E78000E5E9B71783D3
:10A6C000FFFFE70283EF9C4141112A8903C707007E
:10A6D00089472E84935667006380F6040D4663888D
:10A6E000C6049307F0076304F7022E859720000045
:10A6F000E780C0A7AA848149C16B130C490097C7A2
:10A70000FF1F9387A7909C43984763E4E9044101A6
:10A710001783FFFF670023EE03D745008547E3F863
:10A72000E7FE2E8597200000E780A0A9E1B703D7B8
:10A730004500E3FEE7FC2E8597200000E78000A39C
:10A74000AA84228597200000E78060A4C204C98CF7
:10A750005DB7DC470355A900139A49003E9A931749
:10A760000501C187635DF00083570A006397A70264
:10A7700063E774038327CA00034D5A002DA0A16725
:10A780002167A98F1307F7EFE374F7FE63970900BA
:10A7900097000000E780209161FD85098DB7832730
:10A7A0008A00034D4A00835DA90003576900216AAE
:10A7B000138BC7003AC6814A33CA4D01631E5D013F
:10A7C00097C7FF1F938707859C43E1DBA2866286BC
:10A7D000814526858297D1B7A1679387F7EF930CC0
:10A7E0004BFF63F24703B2455A8597F0FFFFE780BE
:10A7F000A0710DC103278B00104709CE104363825F
:10A80000C4023107D5BFEE85668597000000E7805A
:10A81000008F71F993861A0093FAF60F130B0B024F
:10A8200071BF835644005C43E3E9F6F622853AC6DD
:10A8300097100000E780807DA1679387D7042A8A5C
:10A84000035D4400324763E897008347D90093E7EC
:10A8500007F8A306F9001C4766852286E2858297E1
:10A86000C1670844FD17337AFA00529508C02312D5
:10A87000A40125B797B7FF1F93874779984381476E
:10A8800015C31447814763FFD500939745004C4794
:10A89000BE9519C903C7550081476375E600DC45BD
:10A8A0001606B2973E85828003C745008147E37B49
:10A8B000E6FE16069C45F5B71783FFFFE70243D176
:10A8C000AA892E8A814497BAFF1F938A2A7483A784
:10A8D0000A00984763E6E4001783FFFF670083D20E
:10A8E000DC471394440001493E9413BB1400834792
:10A8F0004400634BF900014913BB14008347540023
:10A90000634FF9008504E1B7084493175900528753
:10A91000DA860146A2853E9582990509C9BF484459
:10A92000931759005287DA860546A2853E9582998B
:10A930000509E9B71783FFFFE70223CB814517F528
:10A94000FFFF1305054897B7FF1F2393076C970078
:10A950000000E780A0F61783FFFF670043CB97B79F
:10A96000FF1F9387A76A9C4395C31783FFFFE702E6
:10A97000C3C7814517F5FFFF1305A54497000000E5
:10A98000E780C0F31783FFFF670063C882801783E7
:10A99000FFFFE702E3C337E4040083278412411179
:10A9A0002315E100AE893289368A3A86814601470D
:10A9B000ED45AA8482972AC621C90356A100D285F3
:10A9C00097400100E780C0248327C413CE852685E5
:10A9D0008297058905C98327440D23142101014667
:10A9E0002C00268582972A8401C9B7E7040083A733
:10A9F000C712ED4528008297228541011783FFFF8A
:10AA0000670043C04944D5B76554FDB75C41FD17A5
:10AA10005CC182801783FFFFE70223BDB7E7040014
:10AA2000FC5F829795473305F50281450D811783B9
:10AA3000FFFF6700C3BD1783FFFFE70203BBB7E754
:10AA40000400FC5F829795473305F5020D8117835B
:10AA5000FFFF6700C3BB1783FFFFE70203B9B7E738
:10AA6000040083A7870B0355050082971783FFFF18
:10AA70006700E3B91783FFFFE70223B7035505001B
:10AA80003287AE861796FF1F035626F397B5FF1F32
:10AA90009385855897000000E780A0EF1783FFFF9C
:10AAA0006700E3B61783FFFFE70223B4B7E70400AC
:10AAB00083A7C71782971783FFFF670043B51783E4
:10AAC000FFFFE70283B2B7E7040083A7871397B5B8
:10AAD000FF1F93856554829701451783FFFF670029
:10AAE00003B31783FFFFE70243B0B7E7040083A770
:10AAF000C71F81451795FF1F035525E882971783C8
:10AB0000FFFF6700C3B01783FFFFE70203AEB7E79D
:10AB1000040083A7871397B5FF1F9385E55082979D
:10AB200001451783FFFF670083AE1783FFFFE7022E
:10AB3000C3ABB7E7040083A7C71F81451795FF1F65
:10AB40000355A5E982971783FFFF670043AC17837E
:10AB5000FFFFE70283A92E8597800000E780E0AF22
:10AB600097800000E780E0EC1783FFFF670023AACF
:10AB70001783FFFFE70263A797800000E780E0F6F6
:10AB80001783FFFF6700A3A85C49E1175CC95CC598
:10AB900083572501A1072319F50083570501A10754
:10ABA0002318F5008280F1473305F50297B7FF1FA0
:10ABB000938787499C433E9582808D476315F608AD
:10ABC00003D74600854763F0E7081783FFFFE702D6
:10ABD000C3A1368536842E8997100000E78000597E
:10ABE00029C98357440093140501C18063E3970486
:10ABF000228597100000E7806057FD14231294000F
:10AC00009307A0026300F5029307B0026307F50201
:10AC100093079002631FF500228597000100E780EB
:10AC2000C08501A80146CA85228597A00000E7805B
:10AC300060B01783FFFF6700839D22859710000097
:10AC4000E780C003FDB7828097B6FF1F938606405A
:10AC50009C42014599CF9843D44217B6FF1F232742
:10AC6000E63E6396D70097B6FF1F23A3E63E138503
:10AC7000C7FE82801783FFFFE7022397970000003B
:10AC8000E780A04B71443305850291459790000001
:10AC9000E78020E911E565551783FFFF67002397DB
:10ACA00097B7FF1F23A0A73A97000000E780E0486E
:10ACB00033058502914597900000E78080E661DDCD
:10ACC00097B7FF1F23A2A73897000000E780E04650
:10ACD00097B7FF1F2392A73697000000E780E04553
:10ACE00097B7FF1F239BA73497770100938787FBB4
:10ACF00017B7FF1F2326F73497070000938707E94C
:10AD000017B7FF1F232CF732014579B71783FFFFD1
:10AD1000E702A38DAA8517B5FF1F1305E53197102C
:10AD20000000E780C05B1783FFFF6700438E178337
:10AD3000FFFFE702838B97000000E78060FD97101C
:10AD40000000E780405B97B7FF1F938727309C4345
:10AD500091CF1387C7FE19CB83D5C7FF17B5FF1F48
:10AD60001305452F97200100E78020191783FFFF67
:10AD70006700E3891783FFFFE7022387970000003E
:10AD8000E780C0EC09CD834785002A8493F7070448
:10AD900099EB0355E50097000000E78080F91783E1
:10ADA000FFFF6700C3868347C5009304450117B9B9
:10ADB000FF1F1309A92985E3832709005CC997B7F9
:10ADC000FF1F23A5972883274900F1FB97B7FF1F93
:10ADD00023A09728E9B7FD172306F50061059780A2
:10ADE0000000E780C0D68307840063CB0704834755
:10ADF000840093E707F82304F400B7E704009C5F9E
:10AE000082974205A94741813375F5028347840043
:10AE100093F707FCC98F2304F4008347D4003E95C1
:10AE20001C402318A40089CF984319CB8347C40042
:10AE30005040814585073305F5024205418102975F
:10AE4000832709005CC897B7FF1F23A1972083279A
:10AE5000490089E797B7FF1F23AC971E8347C400BB
:10AE60009DDF8355040117B5FF1F1305A51E97200D
:10AE70000100E780800825B71773FFFFE702E3763C
:10AE800097B7FF1F938747429C4701448583858B73
:10AE900085E3AE84B2853A8697100000E780804B48
:10AEA0002A8419C597100000E780C041829408CC1D
:10AEB00022851773FFFF670083751773FFFFE70293
:10AEC000237141112E8932C6AA8997000000E780BC
:10AED000C031324713060502CA86970500009385E4
:10AEE000C5CC17B5FF1F1305251597000000E78097
:10AEF000E0F82A8425C99304C50097000000E78084
:10AF0000E0411946AA85268597100000E780801544
:10AF10008545268597100000E780601117750100B0
:10AF2000130505D64E95834505002685971000002C
:10AF3000E78020165C4831468145A1075CC85CC4A7
:10AF400083572401E1172319F40083570401E11703
:10AF50002318F4001C4C3E859770FFFFE780E06BE0
:10AF6000A3042501228541011773FFFF6700836950
:10AF70001773FFFFE70263674111AA842EC632C42C
:10AF800097100000E7806036004DB24522468347A7
:10AF900084000CC050C093F7F70393E70704230421
:10AFA000F40023180400268597100000E780803104
:10AFB00083479400A9462317A40013D73700050739
:10AFC0003307D7029D8B85072306F400A306E40010
:10AFD00083C70401D8488507230FF7FE17B7FF1F63
:10AFE0001307C7065843232A04009307440129E3A3
:10AFF00017B7FF1F232EF70417B7FF1F2328F704E7
:10B0000017B4FF1F13040405228597200100E78071
:10B0100000E11C44858B5D8D19E5814522859720D3
:10B020000100E78080ED41011773FFFF6700235E99
:10B030001CC317B7FF1F232DF700D9B71773FFFFE6
:10B04000E702A35A97050000938565B7014597006D
:10B050000000E78000B001451773FFFF6700235B26
:10B060001773FFFFE702635897000000E78080B086
:10B070001773FFFF6700A3598347C500A5E3177344
:10B08000FFFFE70283562A840355E500970000007E
:10B09000E78000C821C18347840093F7F7FB2304AE
:10B0A000F4001C4091C7DC4381C74C4001458297A6
:10B0B00097000000E78080B917B5FF1F130585F9D9
:10B0C00097200100E780A0E50355E4009700000009
:10B0D000E78020C61773FFFF6700635382801773F2
:10B0E000FFFFE702835097B7FF1F938727F6970567
:10B0F0000000938565C817B5FF1F1305A5F523A0AC
:10B10000070023A2070097200100E780E0CE177315
:10B11000FFFF6700C34F1C4D91CFDC4381CF1773F6
:10B12000FFFFE702834C8345070082971773FFFFF9
:10B130006700E34D828097B7FF1F9387E7F39C4337
:10B1400003C50700828097B7FF1F9387E7F29C43F0
:10B1500003C51700828097B7FF1F9387E7F19C43D1
:10B1600003C52700828097B7FF1F9387E7F09C43B2
:10B1700003C54700828097B7FF1F9387E7EF9C4383
:10B1800003C53700828097B7FF1F9387E7EE9C4384
:10B1900003C55700828097B7FF1F9387E7ED9C4355
:10B1A00003C56700828097B7FF1F9387E7EC9C4336
:10B1B00003C57700828097B7FF1F9387E7EB9C4317
:10B1C00003C58700828097B7FF1F9387E7EA9C43F8
:10B1D00003C59700828097B7FF1F9387E7E99C43D9
:10B1E00003C5A700828097B7FF1F9387E7E89C43BA
:10B1F00003C5B70011E11D45828097B7FF1F9387F4
:10B20000A7E79C4303C5C700828097B7FF1F9387BA
:10B21000A7E69C4303C5D700828097B7FF1F93879B
:10B22000A7E59C4303C5E700828097B7FF1F93877C
:10B23000A7E49C4303D50701828097B7FF1F93873C
:10B24000A7E39C4303C52701828097B7FF1F93871D
:10B25000A7E29C4303D54701828097B7FF1F9387DE
:10B26000A7E19C4303D56701828097B7FF1F9387AF
:10B27000A7E09C4303D58701828097B7FF1F938780
:10B28000A7DF9C4303C5A701828097B7FF1F938761
:10B29000A7DE9C4303C5B701828097B7FF1F938742
:10B2A000A7DD9C4303C5C701828097B7FF1F938723
:10B2B000A7DC9C4303C5D701828097B7FF1F938704
:10B2C000A7DB9C438857828097B7FF1F9387C7DA15
:10B2D0009C4303D5C702828097B7FF1F9387C7D9C6
:10B2E0009C4303D5E70219E11305800C828097B7D0
:10B2F000FF1F938767D89C4303C50703828097B7D6
:10B30000FF1F938767D79C43C85B828097B7FF1F57
:10B31000938707D68843828097B7FF1F938787D587
:10B320008843828019E17D558280F5DE984265DF91
:10B33000FDD917B7FF1F130727F71847AA877155BD
:10B34000058B631D072403C507001547E37DA7FC94
:10B3500003C737001305F0057D171377F70FE36474
:10B36000E5FC03C35700E30003FC83C86700E38CDC
:10B3700008FA03C77700494579171377F70FE36495
:10B38000E5FA03C7A70011481305F7FF1375F50F7A
:10B39000E36BA8F803CE97000D481305FEFF137565
:10B3A000F50FE362A8F803C8B70063090800651841
:10B3B0001378F80F1305600DE36705F703C5C700A1
:10B3C000794879151375F50FE36FA8F403C8D70012
:10B3D0000D457D181378F80FE36705F503D80701CD
:10B3E000930E40175118420813580801E3ED0EF36D
:10B3F00003C8E7007D181378F80FE36605F303C868
:10B4000027017D181378F80FE36F05F103C8870053
:10B41000C54E75181378F80FE3E70EF103D86701EE
:10B42000856E938EBEE06D18420813580801E3EC58
:10B430000EEF03D847016D18420813580801E3E4E2
:10B440000EEF03D887017918420813580801E36CFE
:10B4500005ED03C8A7017D181378F80FE36505ED26
:10B4600003C5B7011D487D151375F50FE36DA8EAF7
:10B4700003C5D701714879151375F50FE365A8EA7F
:10B4800003D5E7011308E00F7D1542054181E36C08
:10B49000A8E803C50702494879151375F50FE36459
:10B4A000A8E8C85301C937C834005915130858BF54
:10B4B000E36BA8E603A8870237C53400130555BF20
:10B4C0005918E36205E717B5FF1F2325C5BA03C660
:10B4D000050117B5FF1F2321F5BA0545E375C5E43E
:10B4E00003D82501D04933760603E31E06E203C6DE
:10B4F0001501E30A06E217B6FF1F232BB6B683C574
:10B50000270001466387A50003C61700F1453306EF
:10B51000B60283C707039305C00272971A07130781
:10B52000C70516031A9796084697B387B702415581
:10B530003E973297420741836362E8061773FFFF25
:10B54000E702A30A368597800000E780A06897008D
:10B550000100E78020482A8497A00000E780805AF5
:10B560002A9497F00000E78060262A9497900000C4
:10B57000E780A0812A9497F0FFFFE780E06F2A948C
:10B5800097400000E78060932A9497700000E7805E
:10B59000A09C22951773FFFF6700630782801773D3
:10B5A000FFFFE70283044111A307A10097A0000059
:10B5B000E780A0C59305F100170500001305E5B568
:10B5C00097F0FFFFE780802F014541011773FFFFD0
:10B5D0006700E3031773FFFFE702A3FE17B4FF1F23
:10B5E000130484CC0328840079599368180097B415
:10B5F000FF1F23AF14CB1378180063100802BA841E
:10B60000BE89368B328A2E89AA8A97F0FFFFE7809F
:10B61000E0A77D15269519E531594A851773FFFF77
:10B620006700A3FD97F0FFFFE78040A67D152695F4
:10B63000A167E353F5FE97B7FF1F9387A7FD9843D4
:10B640003E8C814B01CB014597F00000E780204400
:10B65000933B15004A85DA865686D285979000007E
:10B66000E780C04D2A8911CD1C44F99B17B7FF1FF5
:10B670002320F7C483270C00CDD3E3800BFA8297F5
:10B6800069BF268597B7FF1F23A207C297F0FFFF68
:10B69000E780809C4146CE8517B5FF1F130545CA3C
:10B6A00097300100E780C05697D00000E7804099AE
:10B6B0000325040B97D00000E780009D054597D037
:10B6C0000000E78000A4054597000000E78060EDDA
:10B6D000A9B797B7FF1F938727BD9C47858BEDC7F9
:10B6E0001773FFFFE70263F017B5FF1F130585C34C
:10B6F00097B7FF1F23AA07BA97B7FF1F23A807BA58
:10B7000097B7FF1F23A607BA97200100E780208183
:10B7100097500000E780E0F597100100E780A04C0B
:10B7200097100100E780A05297B7FF1F938747B695
:10B730009C4391C7054597800000E780402097B75C
:10B74000FF1F9387A79E9C4399C741657D159770FE
:10B750000000E78040A297F00000E780E03D97D02E
:10B760000000E780808F97B7FF1F9387A7C89C438F
:10B77000139717016356070097F00000E78000ADAC
:10B7800097B7FF1F23AE07BA97B7FF1F23AC07BABF
:10B7900097B7FF1F23AA07BA97B7FF1F23A807BAB7
:10B7A00097000000E780008C97000000E78000729F
:10B7B00097F0FFFFE780401897F00000E78040D641
:10B7C0001773FFFF6700A3E4828097B7FF1F93877B
:10B7D000A7AD884382801773FFFFE70203E19780DC
:10B7E0000000E780607597800000E780C0771773DE
:10B7F000FFFF6700C3E11773FFFFE70263DD2A84E1
:10B800009304140201112E85B289A685214636C6FD
:10B810003A8997300100E780403D0DE9B24638088B
:10B820002686CE851305940497500000E78060417A
:10B8300021462C084A8597300100E780003B1335EC
:10B84000150005611773FFFF6700C3DB0145D5BF16
:10B850001773FFFFE70263D99305450617B5FF1F6E
:10B860001305C58197100100E78020691773FFFF5A
:10B870006700E3D91773FFFFE70223D741112EC6F4
:10B8800097F0FFFFE780601BB24588C14101177345
:10B89000FFFF6700C3D71773FFFFE70263D3AA84D4
:10B8A0002E8497800000E780006CAA898545228558
:10B8B00097000000E780E07D83C7E40113899408C6
:10B8C00099E313890403CE85228597000000E78061
:10B8D000407C214693051902228597000000E780ED
:10B8E000607897B7FF1F9387279C8C43228597101A
:10B8F0000000E780C082214693858402228597005C
:10B900000000E78020761773FFFF6700A3CF17734F
:10B91000FFFFE70203CB397197F00000E780E0B446
:10B920009305400661E997800000E78000606302AC
:10B93000051497A7FF1F83C7277613B7170097A68D
:10B94000FF1F238BE674014499CFC16417B9FF1F11
:10B95000130989959309400EFD1497000000E780B4
:10B96000C0866342A40A97F0FFFFE780000D41699B
:10B97000B7290900096AFD7A2A8B81447D199389C8
:10B98000F97B130A0A71938A8AC797000000E7803F
:10B99000C08363D7A4041304400EB387840217B78F
:10B9A000FF1F130767900324070B3E948357C401BE
:10B9B0006382270B18403307EB4063EAE9008347B3
:10B9C00044008507B3874703D6976365F7080146A8
:10B9D0008145094597F0FFFFE780604EAA8B29E576
:10B9E00097400000E780808385476317F5068965E7
:10B9F0009385057117A5FF1F130545689710010072
:10BA0000E780A04F95A0B30734030327090BBA972B
:10BA100003D7C7016308970003C75700A382070035
:10BA20002382E700050415BF9305C5002285970012
:10BA30000000E78080E65E85228697650100938599
:10BA4000652597F0FFFFE780E0525E8597100000C4
:10BA5000E780608A850415BF97B7FF1F9387C78467
:10BA60009C478D83858BC1F721611773FFFF6700AA
:10BA7000C3B801468545094502D002D202D402D698
:10BA800097F0FFFFE780A043AA8479DD97F00000DC
:10BA9000E780E09C1389C4002A8481454A85970089
:10BAA0000000E780005F0C4041464A859700000097
:10BAB000E780405B832944006385090C4E8502D8EA
:10BAC00002DA02DC02DE97300100E78060402ACE15
:10BAD000141005462C0808184ECC97500000E7803B
:10BAE000E00A1375F50F51ED8355840093E52500A9
:10BAF0004A8597000000E780E05E11460C104A85F9
:10BB000097000000E7800056014697650100938585
:10BB1000E518268597F0FFFFE780C045268597004A
:10BB20000000E780407D5C40A1D3014685450D457E
:10BB300097F0FFFFE780A038AA841DD548401389FD
:10BB4000C40097300100E780A0382AC64A859700D4
:10BB50000000E780404C3246636FC5004C404A8588
:10BB600097000000E780005001468145268597F048
:10BB7000FFFFE7802040268597000000E780A07740
:10BB8000E5B583558400ADB71773FFFFE702E3A562
:10BB900097A7FF1F938747719C471DC193E78700B5
:10BBA00017A5FF1F1305854D17A7FF1F2322F77049
:10BBB00097100100E78040321773FFFF670023A54D
:10BBC000DD9B17A7FF1F2325F76E97300000E78046
:10BBD000E0647DF117A5FF1F1305454A971001008A
:10BBE000E780E033D1BF1773FFFFE702839D416910
:10BBF000AA892E8AB28A368BBA8B814417ACFF1F72
:10BC0000130C8C6A930C400E7D1997F0FFFFE780B0
:10BC1000C05B63C4A40001443DA033849403832724
:10BC20000C0B3E948357C401638627055A87D6863A
:10BC30005286CE851305040397000000E780E0BB21
:10BC400001C923800B0022851773FFFF6700E39A69
:10BC50008347F40185C35A87D6865286CE8513055D
:10BC6000940897000000E78040B909C58547238004
:10BC7000FB00D1BF850451BF835745006380071E79
:10BC80001773FFFFE702C39401112A849700000095
:10BC9000E780C04D09C985476309F506056117733B
:10BCA000FFFF6700239697E00000E780007C7DF5AA
:10BCB000835744004947ED9BE392E7FEC145228547
:10BCC00097000000E7804033AA8422859700000097
:10BCD000E780204F0357440002CE91472A89631A18
:10BCE000F700228597000000E780A0513C082ACC8D
:10BCF0003ECE97E00000E78080765C55C5D374089F
:10BD00004A86A6850545829751BF03574400D1470F
:10BD1000E3F6E7F8032A0400C169014997AAFF1F67
:10BD2000938A8A58130B400EFD1997F0FFFFE780A6
:10BD3000C049634FA90E2285032A04009700000022
:10BD4000E780C042A1452A89228597000000E7804C
:10BD5000A02AAA84228597000000E780804A144028
:10BD60002A86AA8978082685CA8597000000E78078
:10BD7000C0E7AA8405D503C7F40189476315F70016
:10BD80008347C10181DF5546D28513856400973012
:10BD90000100E780E0E7014597800000E780C019D7
:10BDA00001C583D7C401A5E797A7FF1F9387C74F96
:10BDB0009C4793551900858913D73700058B01CF10
:10BDC0008983858B6399B70001452EC697000000D3
:10BDD000E780C0DBB2454E8597800000E780601F9A
:10BDE0000346C1012A8493751900268597900000A7
:10BDF000E780E03935C1268597800000E780E018AC
:10BE0000268511C0014597800000E780004C9730DF
:10BE10000000E780A0408547E312F5E883C754009F
:10BE20001307F00FE38CE7E68507A382F400BDB5A6
:10BE3000B304690383A70A0BBE9483D7C401638B41
:10BE400037015546D2851385640097300100E7809D
:10BE5000C0D955DD0509D1BD5DD86DB782801763A6
:10BE6000FFFFE702E37697800000E780000C05C142
:10BE7000C164014417A9FF1F130909439309400E28
:10BE8000FD1497F0FFFFE7804034634EA40017A530
:10BE9000FF1F1305A51E97100100E780E00317633D
:10BEA000FFFF67002376330534038327090B3E9594
:10BEB0008357C5016388970023120500978000000F
:10BEC000E780A00C050475BF97A7FF1F9387C73DA8
:10BED0009C478D83858B8DE31763FFFFE702E3703B
:10BEE00017A5FF1F1305851997100100E780200390
:10BEF0001763FFFF6700A37182801763FFFFE702EC
:10BF0000C36E970500009385C5A017A5FF1F1305F5
:10BF1000E51697100100E78020EE1763FFFF67002A
:10BF2000036F1763FFFFE702436C8841B7E7040024
:10BF3000BC5B050542054181829709C58547230001
:10BF4000F50005051763FFFF6700636C83C7F5FF06
:10BF50002E858507A38FF5FE828083C7F5FFFD1729
:10BF600093F7F70FA38FF5FE99EF1763FFFFE70233
:10BF7000C367B7E70400BC571385F5FF82971763C3
:10BF8000FFFF6700C36882801C41035745008D8F07
:10BF9000BA951CC12312B5003E85828093D78500D7
:10BFA000A2051441DD8D835745001387E6FF18C1B4
:10BFB00089072312F50013D685004111238FB6FEA1
:10BFC000A38FC6FE4101828018419307F7FF1CC171
:10BFD0008357450085072312F500A30FB7FE828023
:10BFE000835745008D8F2312F5001C41BE950CC16F
:10BFF0002E858280AA8703D7470008410D8FAA9516
:10C000002392E7008CC38280184108453305A7407E
:10C01000828083574500035765001D8F1C410845EA
:10C020003385A7403305A74082801763FFFFE702EF
:10C03000C35B41112EC62A8497000000E780A0FD53
:10C04000B2456373B50001A0835744000840BE9514
:10C050002312B4003E9541011763FFFF6700235B85
:10C060001763FFFFE702635841112E84B28532C681
:10C0700097000000E780A0FB3246A28597300100C0
:10C08000E78000B941011763FFFF6700435817635A
:10C09000FFFFE70283552E84854597000000E78067
:10C0A00000F9230085001763FFFF670043561763FD
:10C0B000FFFFE702835341112317B1008945970021
:10C0C0000000E780C0F68347E1002300F5008347C6
:10C0D000F100A300F50041011763FFFF6700235340
:10C0E0001763FFFFE702635093D78500A205411154
:10C0F000DD8D2317B100894597000000E78020F30C
:10C100008347E1002300F5008347F100A300F50019
:10C1100041011763FFFF6700834F1763FFFFE702CB
:10C12000C34C1397850193D78501C166938606F0AA
:10C13000D98F13D78500758FD98FA2053707FF00D8
:10C14000F98D4111DD8D2EC6914597000000E780E5
:10C1500000EE6C00114697300100E78060AB4101B2
:10C160001763FFFF6700A34A1763FFFFE702E34778
:10C170001C41854503C4070097000000E78080E666
:10C1800022851763FFFF670083481763FFFFE702FD
:10C19000C3451C414111894503C7070083C71700E8
:10C1A0002307E100A307F10097000000E78080E388
:10C1B0000355E10041011763FFFF67004345176323
:10C1C000FFFFE70283421C414111894503C7070075
:10C1D00083C717002307E100A307F10097000000C1
:10C1E000E78040E08357E100410113D58700A207B3
:10C1F0005D8D420541811763FFFF6700434117636F
:10C20000FFFFE702833E0C4141112A84114668007A
:10C2100097300100E780C09F91452285970000007C
:10C22000E78040DCB247C166938606F0139787012A
:10C2300013D58701598D13D78700758F598DA207A4
:10C240003707FF00F98F5D8D41011763FFFF67001E
:10C25000033C1C45BE950CC18280AE87944391E699
:10C26000584101EF0CC15CC1828003C757001367BE
:10C270001700A382E700B687D5B70CC3EDB7AA872E
:10C28000084119CD1841D44398C36313D500D8C3CE
:10C290002A87034657009376160081E6232007007D
:10C2A0008280944381CA8C4203A847008CC3639365
:10C2B0000601CCC3799A14C3A302C7003687D1BF45
:10C2C0001C45DC471D8DB777DBB6938777DB098587
:10C2D0003305F502420541818280F147B385F502BD
:10C2E00048452E9582808347450085072302F50047
:10C2F00082801763FFFFE702432F2A8409E4176354
:10C30000FFFF6700C33083474400F5DBFD1793F759
:10C31000F70F2302F400E5F71C4403D727000507B5
:10C320002391E700DC4399C3228582974C4889CD4D
:10C3300083475400898B99E71C4422859C479C4382
:10C340009C478297232A04000040232004007DB7E5
:10C350001763FFFFE70263298357250041112EC6AB
:10C3600081EB0144228541011763FFFF6700232A07
:10C37000035705008147F146E305F7FEB385D70271
:10C38000404585072E948345440008C4F5F5B2471F
:10C39000AA8481E7232A040009A81C456C00228591
:10C3A0009C439C43829748C84DDD85472312F40087
:10C3B000B24723200400231804002319F4005C482A
:10C3C0005CC483D72400FD172391F40061BF176379
:10C3D000FFFFE702832197A7FF1F938727CC88439E
:10C3E0002326050023240500410597100100E7805E
:10C3F00000B31763FFFF670083211763FFFFE702A6
:10C40000C31E17A4FF1F130464C91C40411199CF18
:10C410009C472300B5002AC65CC197000000E78056
:10C4200040FB1C40DC4399C33245829741011763AE
:10C43000FFFF6700C31D0347450029E3584DAA8746
:10C440007D551DCF1763FFFFE702231A1CC3DC478E
:10C4500097A6FF1F23A4E6C4F156130507012390F6
:10C46000D700970500009385050297100100E7802B
:10C47000A09801451763FFFF670063197D5582800F
:10C4800082801763FFFFE702431601116146814571
:10C4900028009760FFFFE780401897A7FF1F93874A
:10C4A000E7BF9C4328009305F00FDC473EC697008A
:10C4B0000000E780C0F405611763FFFF67002315E4
:10C4C00097A7FF1F938787BD9C43D847A167938792
:10C4D000C702631EF70A397106DE22DC26DA800005
:10C4E0004AD84ED652D456D23285B2849700000034
:10C4F000E780C0C7AA89268597000000E78020C989
:10C500002318A4FC268597000000E78040C8231963
:10C51000A4FC268597000000E78060C783D744000D
:10C520000A8A231AA4FC858393F7F70F230EF4FCE1
:10C530008607BD0793F7073F3301F1408A8A014917
:10C540008347C4FD6367F902CE85130584FC232C61
:10C5500054FD97000000E78080EA5281130104FC3B
:10C56000F2506254D2544259B259225A925A21611D
:10C570008280268597000000E78060C1931719002C
:10C58000D69705092390A7001379F90F55BF82802C
:10C5900097A7FF1F938787B09C43D847A1679387CE
:10C5A000A702631AF70A397106DE22DC26DA800058
:10C5B0004AD84ED652D456D23285B2849700000063
:10C5C000E780C0BAAA89268597000000E78020BCD2
:10C5D000FD572318A4FC26852319F4FC97000000BE
:10C5E000E780E0BA83D744000A8A231AA4FC858333
:10C5F00093F7F70F230EF4FC8607BD0793F7073F69
:10C600003301F1408A8A01498347C4FD6367F90217
:10C61000CE85130584FC232C54FD97000000E78091
:10C6200000DE5281130104FCF2506254D25442598C
:10C63000B259225A925A21618280268597000000C1
:10C64000E780E0B493171900D69705092390A70057
:10C650001379F90F55BF828097A7FF1F938707A40F
:10C660009C43D847A16789076310F70A397106DE32
:10C6700022DC26DA80004AD84ED652D456D23285F1
:10C68000328997000000E78060AEAA894A8597004A
:10C690000000E780C0AF835749000A8A2318A4FC32
:10C6A000858393F7F70F230CF4FC8607BD0793F7F8
:10C6B000073F3301F1408A8A8144834784FD63E761
:10C6C000F402CE85130584FC232A54FD9700000054
:10C6D000E780E0D25281130104FCF2506254D2543C
:10C6E0004259B259225A925A216182804A85970052
:10C6F0000000E780C0A993971400D6978504239083
:10C70000A70093F4F40F55BF828097A7FF1F93876C
:10C71000E7989C43D847A1679387E704631EF70A0D
:10C72000397106DE22DC26DA80004AD84ED652D491
:10C7300056D23285B28497000000E78020A3AA89F0
:10C74000268597000000E78080A42318A4FC268596
:10C7500097000000E780A0A3231AA4FC2685970079
:10C760000000E780C0A283D744000A8A2319A4FCF2
:10C77000858393F7F70F230EF4FC8607BD0793F725
:10C78000073F3301F1408A8A01498347C4FD63674B
:10C79000F902CE85130584FC232C54FD970000007C
:10C7A000E780E0C55281130104FCF2506254D25478
:10C7B0004259B259225A925A2161828026859700A5
:10C7C0000000E780C09C93171900D69705092390B5
:10C7D000A7001379F90F55BF828097A7FF1F938792
:10C7E000E78B9C43D847A1679387C704631AF70A6E
:10C7F000397106DE22DC26DA80004AD84ED652D4C1
:10C8000056D23285B28497000000E7802096AA892C
:10C81000268597000000E7808097FD572318A4FC29
:10C820002685231AF4FC97000000E780409683D702
:10C8300044000A8A2319A4FC858393F7F70F230E7B
:10C84000F4FC8607BD0793F7073F3301F1408A8A5E
:10C8500001498347C4FD6367F902CE85130584FC53
:10C86000232C54FD97000000E78060B9528113012A
:10C8700004FCF2506254D2544259B259225A925A8C
:10C8800021618280268597000000E7804090931701
:10C890001900D69705092390A7001379F90F55BF02
:10C8A00082809797FF1F9387677F9C43D847A16734
:10C8B000DD076317F7041763FFFFE70203D37971FE
:10C8C0003285328497000000E780408A2AC622859C
:10C8D00097000000E780A08B2311A102228597001A
:10C8E0000000E780A088B2452300A1022808970035
:10C8F0000000E780C0B045611763FFFF670023D1E8
:10C9000082809797FF1F938767799C43D847A167D9
:10C91000938787046317F7041763FFFFE702E3CCED
:10C9200079713285328497000000E78020842AC61E
:10C93000228597000000E78080852311A1022285CF
:10C9400097000000E7808082B2452300A1022808FA
:10C9500097000000E780A0AA45611763FFFF67000A
:10C9600003CB82809797FF1F938747739C43D847D9
:10C97000A1679387A7046312F7021763FFFFE7021B
:10C98000C3C601112800814597000000E78020A759
:10C9900005611763FFFF670083C782809797FF1FBA
:10C9A0009387C76F9C43D847A16793875702631942
:10C9B000F7021763FFFFE70243C30111328597F0C7
:10C9C000FFFFE780A07A2308A10081452800970097
:10C9D0000000E780C0A205611763FFFF670023C363
:10C9E00082809797FF1F9387676B9C43D847A16707
:10C9F0009387E702631BF7041763FFFFE702E3BEB9
:10CA000001113285328497F0FFFFE7804078AA84D5
:10CA1000228597F0FFFFE7808077854709E9228527
:10CA200097F0FFFFE78080744205B337A00028002D
:10CA30008145231891003ECA97000000E780209CA2
:10CA400005611763FFFF670083BC82809797FF1F14
:10CA50009387C7649C43D84799476313F7081763C4
:10CA6000FFFFE70283B879713285328497F0FFFFC8
:10CA7000E780C06F2AC6228597F0FFFFE78020710C
:10CA80002310A102228597F0FFFFE780206E23018B
:10CA9000A102228597F0FFFFE780406DA301A1026C
:10CAA000228597F0FFFFE780606C2302A1022285B8
:10CAB00097F0FFFFE780806B2313A102228597F098
:10CAC000FFFFE780A06AB2452314A102280897005F
:10CAD0000000E780C09245611763FFFF670023B342
:10CAE00082809797FF1F9387675B9C43D847A16716
:10CAF0009387C7036313F7081763FFFFE702E3AEEB
:10CB000079713285328497F0FFFFE78020662AC66C
:10CB1000228597F0FFFFE78080672310A10222851E
:10CB200097F0FFFFE780A0662311A102228597F00E
:10CB3000FFFFE780A0632302A102228597F0FFFF99
:10CB4000E780C062A302A102228597F0FFFFE78081
:10CB5000E0612303A102228597F0FFFFE7800061D7
:10CB6000B245A303A102280897000000E7802089AE
:10CB700045611763FFFF670083A982801763FFFF8A
:10CB8000E702A3A601112A8497F0FFFFE780005E69
:10CB9000AA84228597F0FFFFE780605F228597F0E7
:10CBA000FFFFE780C05E035744008D4763F7E7004F
:10CBB000228597F0FFFFE780805D228597F0FFFFD9
:10CBC000E780E05C2800A68597000000E7802083CE
:10CBD00005611763FFFF670083A39797FF1F938784
:10CBE000E74B9C43D847A167FD07631FF700176316
:10CBF000FFFFE702839F328597000000E78040F83F
:10CC00001763FFFF6700A3A082809797FF1F93879A
:10CC1000E7489C43D847A167E5076315F708176302
:10CC2000FFFFE702839C79713285328497F0FFFF22
:10CC3000E780C0532AC6228597F0FFFFE780205582
:10CC4000228597F0FFFFE78080542310A102228500
:10CC500097F0FFFFE780A053520551812311A102F5
:10CC600022852302010297F0FFFFE7802050A302F4
:10CC7000A102228597F0FFFFE780404F2303A10226
:10CC8000228597F0FFFFE780604EB245A303A10223
:10CC9000280897F0FFFFE780807645611763FFFF64
:10CCA0006700E39682809797FF1F9387273F9C43F7
:10CCB000D847A1679387E703631FF7001763FFFF58
:10CCC000E702A392328597000000E78060EB1763CC
:10CCD000FFFF6700C39382809797FF1F9387073CEE
:10CCE0009C43D847A16793874704631EF7021763E5
:10CCF000FFFFE702838F79713285328497F0FFFF5F
:10CD0000E780C0462AC6228597F0FFFFE7802048CB
:10CD1000B245280897F0FFFFE780606E4561176312
:10CD2000FFFF6700C38E82809797FF1F93870737A7
:10CD30009C43D847A167938787026310F704176362
:10CD4000FFFFE702838A79713285328497F0FFFF13
:10CD5000E780C0412AC6228597F0FFFFE7800041A7
:10CD6000B2452300A102280897F0FFFFE780206961
:10CD700045611763FFFF6700838982801763FFFFA8
:10CD8000E702A386011197F0FFFFE780203EAA8506
:10CD9000280097F0FFFFE780806605611763FFFFBB
:10CDA0006700E3869797FF1F9387472F9C43D847D9
:10CDB000A167D107631FF7001763FFFFE702E38254
:10CDC000328597000000E780A0FB1763FFFF670034
:10CDD000038482809797FF1F9387472C9C43D847F3
:10CDE000A167C507631FF7001753FFFFE702E37F43
:10CDF000328597000000E780A0F81763FFFF670007
:10CE0000038182809797FF1F938747299C43D847C8
:10CE1000A167B907631FF7001753FFFFE702E37C21
:10CE2000328597000000E780A0F51753FFFF6700E9
:10CE3000037E82809797FF1F938747269C43D8479E
:10CE4000A167AD07631FF7001753FFFFE702E37900
:10CE5000328597000000E780A0F21753FFFF6700BC
:10CE6000037B82809797FF1F938747239C43D84774
:10CE700089476318F7021753FFFFE7020377011191
:10CE8000328532C897F0FFFFE780402EAA85280040
:10CE900097F0FFFFE780A05605611753FFFF67007B
:10CEA000037782809797FF1F9387471F9C43D8473C
:10CEB000A1678D076311F7041753FFFFE702E372C1
:10CEC00001113285328497F0FFFFE780202A130694
:10CED0006100AA844C00228597300000E780C023BF
:10CEE0002800A68597F0FFFFE78060510561175382
:10CEF000FFFF6700C37182809797FF1F9387471AD0
:10CF00009C4381CFDC4391CB1753FFFFE702E36DD6
:10CF100082971753FFFF6700836F82801753FFFFCD
:10CF2000E702A36C79713C08AE843ED2A165B707D5
:10CF30000A002A843ED448103C08DD053ED636C49B
:10CF400032C63AC297D0FFFFE780E02F1247481061
:10CF5000BA8597F0FFFFE780C01332464810B285CC
:10CF600097F0FFFFE780E014A2464810B68597F0DF
:10CF7000FFFFE7800012501001478146A6852285F9
:10CF800097D0FFFFE780805145611753FFFF67008F
:10CF900003681753FFFFE702436501117C00032973
:10CFA000C501AE843ECAA165B70707002A843ECCFE
:10CFB00048087C00C5053ECE97D0FFFFE780A0283B
:10CFC0008345D900480897F0FFFFE780800C5008A0
:10CFD00001478146A685228597D0FFFFE780004C58
:10CFE00005611753FFFF670083621753FFFFE702D6
:10CFF000C35F83C7950093F7F707A384F5009700F5
:10D000000000E78040F91753FFFF670043601753A4
:10D01000FFFFE702835D79713C08AE843ED2A165D3
:10D02000B70709002A843ED448103C08938545047C
:10D030003ED632C636C497D0FFFFE780C020A24656
:10D040004810B68597F0FFFFE780A00432464810ED
:10D05000B28597F0FFFFE780C00550100147814679
:10D06000A685228597D0FFFFE7804043456117538F
:10D07000FFFF6700C3591753FFFFE702035783C73A
:10D08000950041112A8493F7F707A384F5003285B0
:10D090002EC697F0FFFFE780800F85672AC4637074
:10D0A000F50297700000E78020E92246B24509EDBD
:10D0B00011478146228597000000E78060E6410124
:10D0C0001753FFFF6700A35401478346F501DDB7FF
:10D0D0001753FFFFE702C34F01113C003ECAB707D9
:10D0E0000A003ECC3C003ECE83C79500AA8932851B
:10D0F00093F7F707A384F5002E8497F0FFFFE780EE
:10D1000000098567637DF504A165AA84938585047C
:10D11000480897D0FFFFE78000132685977000002E
:10D12000E78080E12A8929E19145480897F0FFFFCF
:10D13000E78020F6A685480897F0FFFFE78060F7B4
:10D14000CA85480897F0FFFFE780A0F401478146B1
:10D150005008A2854E8597D0FFFFE78020340561F7
:10D160001753FFFF6700034A8145480897F0FFFF08
:10D17000E78020F20349090275BF1753FFFFE7025A
:10D18000234579711C103ECAB7070F003ECC404DB5
:10D190001C10AA84AE894808994532C636893ECE0D
:10D1A00097D0FFFFE780200A32464808B28597F003
:10D1B000FFFFE78000EE630C0902A545480897F0E1
:10D1C000FFFFE780C0E62546CA8597200100E7807B
:10D1D00020A4500801478146CE85268597D0FFFFC1
:10D1E000E780C02B45611753FFFF6700A3418355BC
:10D1F000C402480897F0FFFFE780A0EB0355E40264
:10D20000814505C5854785456301F502C167FD1761
:10D210009305F00F630BF5007D1597700000E78014
:10D22000208E9305150093F5F50F480897F0FFFF42
:10D23000E78020E683450403480897F0FFFFE78076
:10D2400040E583451403480897F0FFFFE78060E45A
:10D2500083552403480897F0FFFFE78080E5835556
:10D260004403480897F0FFFFE780A0E49DB71753F9
:10D27000FFFFE702833783C795008146014693F796
:10D28000F707A384F50097000000E78040EF1753ED
:10D29000FFFF6700C3371753FFFFE70203357971BC
:10D2A0003E841C103ECA2E89B7070F00A1653ECCF4
:10D2B000FD051C10AA84480842C03AC23ECE36C4BE
:10D2C00032C697D0FFFFE78000F832464808B285A3
:10D2D00097F0FFFFE780E0DBA2464808B68597F0AD
:10D2E000FFFFE78000DD12474808BA8597F0FFFF8F
:10D2F000E78020DC0248630C08029145480897F05B
:10D30000FFFFE780C0D21146A28597200100E78089
:10D310002090500801478146CA85268597D0FFFF97
:10D32000E780C01745611753FFFF6700432E89450B
:10D33000480897F0FFFFE78080CF83470400230071
:10D34000F50083471400A300F500E1B71753FFFF72
:10D35000E702032883C7950001112A8A93F7F7078C
:10D36000A384F5003285AE8432C697F0FFFFE780D4
:10D3700000E232462A89328597F0FFFFE78000DF1E
:10D3800085676373F902AA894A8597700000E78070
:10D39000A0BA2A8419ED114781464A86A68552858E
:10D3A00097000000E780C0B705611753FFFF6700D3
:10D3B00063259387E9FF93F7F70F0547E366F7FEC9
:10D3C0008347F50195EB8947E380F9FE8346F40135
:10D3D000528501474A86A68597000000E78040B441
:10D3E000A167D90748083ECC230A010002CE970066
:10D3F0000000E780A0B04DBF639EE7008947639EB1
:10D40000F90093071020231FF50097700000E780B4
:10D41000C0B76DBF0947E39BE7FA8D47E398F9FA78
:10D42000228597700000E78080DF9797FF1F938722
:10D4300027E69C4399E79797FF1F938727CF9C4345
:10D4400099C703D5040097800000E780A0CE231F72
:10D45000040022855DBF1753FFFFE7020319011186
:10D460003C003ECAB7070B003ECC3C003ECE83C713
:10D4700095002A89328593F7F707A384F500AE84D7
:10D4800097F0FFFFE780A0D093170501C187635A8B
:10D49000F006A1652A849385E502480897D0FFFF2E
:10D4A000E78060DAA285480897F0FFFFE78060C058
:10D4B0009797FF1F938787C79C43A9EB01449375F8
:10D4C000F40F480897F0FFFFE780A0BC9355844015
:10D4D00093F5F50F480897F0FFFFE78080BB935561
:10D4E000044193F5F50F480897F0FFFFE78060BA15
:10D4F000014781465008A6854A8597D0FFFFE780FF
:10D50000E0F905611753FFFF670063104165854629
:10D510000546A2857D1597500000E78060BD59DD66
:10D52000510597000100E780808F130440063344C3
:10D53000850271B71753FFFFE702230B0111B707ED
:10D5400006003EC683C7950021642A8993F7F70732
:10D55000A384F500AE8428009305A4040AC40AC875
:10D5600097D0FFFFE78020CE300001478146A68597
:10D570004A8597D0FFFFE78060F297E0FFFFE780E2
:10D58000801513049404480822CC230A010002CE1B
:10D5900097000000E780809605611753FFFF670042
:10D5A00003071753FFFFE702A302C1642A8901445E
:10D5B0009799FF1F938949CF130A8002FD1497E0C2
:10D5C000FFFFE78080C16347A40001451753FFFFB9
:10D5D00067004303B307440303A7C90ABA9703D7F5
:10D5E00007006306970083D727006384270105049B
:10D5F000F9B70545E1BF1753FFFFE70263FD2A8A2C
:10D600002E8999C123A0050081498144979AFF1F63
:10D61000938A4AA9614B97E0FFFFE78040C263C746
:10D62000A4004E851753FFFF6700C3FD33846403D6
:10D6300083A70A003E948357040099E76304090016
:10D64000232089008504C1BF4146D28513054400CB
:10D6500097100100E780605975F5A289E5B7175367
:10D66000FFFFE702E3F639717C083ED4B7070A00F2
:10D670003ED67C083ED883C795002A8A328593F728
:10D68000F707A384F5002E8932C697F0FFFFE780E5
:10D6900000B085676373F5083246AA84328597F037
:10D6A000FFFFE780A0AC8547AA8963E8A706A165CC
:10D6B00093858504281097D0FFFFE780C0B82685A2
:10D6C00097700000E78040872A8429ED9145281053
:10D6D00097F0FFFFE780E09BA685281097F0FFFFFB
:10D6E000E780209DCE85281097F0FFFFE780609AA5
:10D6F000014781463010CA85528597D0FFFFE780E9
:10D70000E0D9A1679387770448183EDC230A010219
:10D7100002DE97F0FFFFE780607E21611753FFFF75
:10D72000670043EE8145281097F0FFFFE780609681
:10D73000A685281097F0FFFFE780A0979797FF1F17
:10D74000938707ED9C4381CB22856389090097D09D
:10D750000000E78040248345040271B797D00000A1
:10D76000E780C022CDBF1753FFFFE70263E683C700
:10D7700095004111AA8993F7F707A384F500328534
:10D78000AE84328A97F0FFFFE78060A08567637FF1
:10D79000F5022A8997600000E780007A2A84914682
:10D7A00031C58347F50105476387E70291C70D47F8
:10D7B0006366F704AD461DA89305050303250A001B
:10D7C000414697100100E78040420DE9410117539F
:10D7D000FFFF670023E39305950803250A004146F0
:10D7E00097100100E7806040814669F54A86A6856A
:10D7F0004E8597000000E780C081C9BF83250A00DD
:10D800001305940897700000E780A02919C1C1464C
:10D81000F1BF9797FF1F9387A7A79C4399E7979717
:10D82000FF1F9387A7909C4399C72285978000008C
:10D83000E780208A69FD8547A30FF400228597B011
:10D840000000E7806084228597600000E780E07335
:10D850004E8581464A86A68597F0FFFFE780607B6C
:10D86000A1679387570448003EC42302010002C603
:10D8700097F0FFFFE780806891BF1753FFFFE70233
:10D8800043D483C795004111AA8993F7F707A3846E
:10D89000F50032852E89B28A97F0FFFFE780208F4E
:10D8A00085676374F50EAA8497600000E780C068FE
:10D8B0002A840DED416B014A979BFF1F938BCB9EF2
:10D8C000130C400E7D1B19A833048A0383A70B0B8E
:10D8D0003E948357C40163836705050A97E0FFFF01
:10D8E000E780A08EE342AAFE95460DA08357C501AE
:10D8F000639697029305050303A50A004146971016
:10D900000100E780802E994611E181462686CA856E
:10D910004E8597F0FFFFE780C06F85A883A50A00BA
:10D920001305040397700000E780A017C14679FD36
:10D930002285231E940097A00000E780E0742285D2
:10D9400097600000E78060649797FF1F938747CC3C
:10D950009C43A9C323000402228597D00000E780DE
:10D9600040F04E8581462686CA8597F0FFFFE78006
:10D97000406AA1679387070448003EC42302010060
:10D9800002C697F0FFFFE780605741011753FFFF82
:10D990006700A3C689472300F402E1B7397106DEA8
:10D9A00022DC4AD8800052D456D25AD026DA4ED63B
:10D9B0005ECE2E8A32892A8B97D0FFFFE780E07DEA
:10D9C0000605710541998A8A3301A140232224FC6E
:10D9D000231404FC97D0FFFFE780207C83479A0044
:10D9E0000605350593F7F7072315A4FCA304FA00F1
:10D9F0004A85232624FC97E0FFFFE78040799317B0
:10DA00000501C1876340F0025681130104FCF25006
:10DA10006254D2544259B259225A925A025BF24B82
:10DA200021618280AA844A8597E0FFFFE780207603
:10DA3000AA894A8597E0FFFFE7806075A165938515
:10DA4000C5022A89130544FC97C0FFFFE780A07F29
:10DA5000268597C0FFFFE780E073854511C94A8698
:10DA6000CE8597C0FFFFE780606DAA8B21E98945CD
:10DA7000130544FC97E0FFFFE780A061A68513052E
:10DA800044FC97E0FFFFE780C062CE85130544FCAD
:10DA900097E0FFFFE780E061CA85130544FC97E04B
:10DAA000FFFFE780006101478146130644FCD285F1
:10DAB0005A8597D0FFFFE780609EB9B7814513056F
:10DAC00044FC97E0FFFFE780C05CA685130544FC9B
:10DAD00097E0FFFFE780E05DCE85130544FC97E00B
:10DAE000FFFFE780005DCA85130544FC97E0FFFF58
:10DAF000E780205C814497D0FFFFE780006AE3D491
:10DB0000A4FA83A70B0113971400BA9783D50700D3
:10DB100099C5130544FC97E0FFFFE7808059850411
:10DB2000D9BF797106D622D44AD000184ECE52CC35
:10DB300056CA26D25AC8AE893289AA8A97D0FFFF20
:10DB4000E780A0650605690541990A8A3301A1406D
:10DB5000232A24FC231C04FC97D0FFFFE780E0630A
:10DB600083C7990006052D0593F7F707231DA4FC2D
:10DB7000A384F9004A85232E24FC97E0FFFFE78069
:10DB8000006193170501C187634FF00052811301B3
:10DB900004FDB250225492540259F249624AD24AC8
:10DBA000424B45618280AA844A8597E0FFFFE78067
:10DBB000005EA1659385A5022A89130544FD97C0DF
:10DBC000FFFFE7804068268597C0FFFFE780805C05
:10DBD000854509C9CA8597C0FFFFE78020592A8B70
:10DBE00029E18945130544FD97E0FFFFE780604A7E
:10DBF000A685130544FD97E0FFFFE780804BCA85AB
:10DC0000130544FD97E0FFFFE780A04A01478146E6
:10DC1000130644FDCE85568597D0FFFFE780008828
:10DC2000B5B78145130544FD97E0FFFFE7806046E7
:10DC3000A685130544FD97E0FFFFE7808047CA856E
:10DC4000130544FD97E0FFFFE780A046814497D08D
:10DC5000FFFFE7808054E3DBA4FA83270B011397CF
:10DC60001400BA9783D5070099C5130544FD97E0C2
:10DC7000FFFFE78000448504D9BF1753FFFFE70289
:10DC8000C39683474500404DD5EFFD575DC483469D
:10DC9000940009476363D70A0346B400854663EEE0
:10DCA000C6088306E40063CA06085C45F95623905B
:10DCB000D7009787FF1F83C7273F99E3A304E4009A
:10DCC0009787FF1F938787469C4381E78947A30671
:10DCD000F4009797FF1F9387A7939C4381E7894799
:10DCE0002306F4009705000093854506AA841305D2
:10DCF000040197F00000E7802010FD57231AF4027A
:10DD000081471CDC01489787FF1F23AB8738978723
:10DD1000FF1F93872739232E040304C0804397D025
:10DD2000FFFFE780C05161463306C5028145228569
:10DD30009750FFFFE780608E81473E851753FFFFB6
:10DD40006700E38CFD57D5BF1753FFFFE702E38958
:10DD50002A840355450297600000E780E01D19E51D
:10DD6000231E04001753FFFF6700638A8357E401F3
:10DD7000F5DB930504FF174501001305E52B97E03C
:10DD80000000E780E014F9BF1753FFFFE702E385C7
:10DD90002E89A16541119385E5032A8436C432C6D4
:10DDA000BE843AC297C0FFFFE780E0491247228550
:10DDB000BA8597E0FFFFE780C02D32462285B28505
:10DDC00097E0FFFFE780E02EA2462285B68597E028
:10DDD000FFFFE780002E630309029145228597E04B
:10DDE000FFFFE780C0241146A68597100100E78059
:10DDF00020E241011753FFFF6700638189452285B7
:10DE000097E0FFFFE780A02283C704002300F5000E
:10DE100083C71400A300F500E9BF1743FFFFE70223
:10DE2000C37C83C79500444D054793F7F707A38448
:10DE3000F5001C42411183C707006367F7062E8473
:10DE40002A89B1C003C7D400630FF7021787FF1FE9
:10DE50001307C72D184305C3A386F40097A000003D
:10DE6000E780404A83C7D40099E741657D15974014
:10DE70000000E780403083D72403918B89C797E067
:10DE80000000E780C0134A85A28597F0FFFFE78076
:10DE90008010A167C10748003EC42302010002C6EA
:10DEA00097F0FFFFE780800541011743FFFF670000
:10DEB00003761743FFFFE702437303D745008D47FF
:10DEC000AA8441112E8432892E8563E3E70297E00C
:10DED000FFFFE780C02BAA8523000900268597C095
:10DEE000FFFFE780A02841011743FFFF670023726F
:10DEF00097E0FFFFE780A0292AC6228597E0FFFF71
:10DF0000E780E028B24585472A862300F900268568
:10DF100097C0FFFFE7808022F9B7397106DE22DC67
:10DF200026DA80004ED652D456D24AD85AD05ECE87
:10DF3000AE89B284AA8A97D0FFFFE7800025060544
:10DF40001305250241990A8A3301A140232224FCAA
:10DF5000231404FC97D0FFFFE780202383C7990098
:10DF600006054D0593F7F7072315A4FCA384F900D4
:10DF70002685232624FC97E0FFFFE78040219317A6
:10DF80000501C1876340F0025281130104FCF25085
:10DF90006254D2544259B259225A925A025BF24BFD
:10DFA00021618280AA8B03AB040097C0FFFFE7804A
:10DFB000601E51E583D7440001498544F11793B7AA
:10DFC0001700A301F4FC834734FCA165C9C79385FE
:10DFD000E504130544FC97C0FFFFE780C026A68533
:10DFE000130544FC97E0FFFFE780A00ADE851305D8
:10DFF00044FC97E0FFFFE780C00B834734FC1146E9
:10E0000091E30946DA85130544FC97E0FFFFE780BA
:10E0100060058144630A0900416B7D1B97D0FFFFB7
:10E02000E780A01663CCA40201478146130644FC96
:10E03000CE85568597C0FFFFE7804046B1B7A685DD
:10E04000130634FC97000000E780E0E693341500E7
:10E050002A8986048DBF9385C504A5BF8327C9007F
:10E0600013971400BA9783D50700638865011305D9
:10E0700044FC97E0FFFFE780C003850445B71743E2
:10E08000FFFFE702035479711C103EC4B7070F006D
:10E090003EC61C103EC883C79500AA8A328593F7F6
:10E0A000F707A384F500AE89328497E0FFFFE7808D
:10E0B000000E93170501C187635AF0062A8A22854C
:10E0C00097E0FFFFE780A00C2A895285032B04000C
:10E0D00097C0FFFFE780000C39ED8357440081446F
:10E0E0000544F11793B71700A303F10083457100AE
:10E0F000DA872287CA865286280097000000E780C8
:10E10000E0C8014781463000CE85568597C0FFFFA5
:10E11000E780C038A1679387D70348083ECC230A1D
:10E12000810026CE97F0FFFFE78040DD4561174371
:10E13000FFFF6700834CA285130671009700000063
:10E14000E78060D7AA84094455D13544E30055FBE4
:10E150004A8597F0FFFFE78000450D4441D901440F
:10E1600097D0FFFFE7806002634DA400C16B0144BC
:10E17000FD1B97D0FFFFE7804001634EA4001544CC
:10E18000B5B7DC4413171400BA9783D7070063832D
:10E1900027030504F1B7D84493171400BA9703D79F
:10E1A0000700631B770123902701268597A00000B5
:10E1B000E78080DB01441DBF050465BF1743FFFFF7
:10E1C000E702034183C7950041112A8A93F7F707B5
:10E1D000A384F50032852E89328497E0FFFFE78023
:10E1E00000FB93170501C1876353F006AA892285B6
:10E1F00097E0FFFFE780A0F92311A1004E85832A55
:10E20000040097C0FFFFE780E0F839E5835744003A
:10E2100085440144F11793B71700A300F1000348A8
:10E22000110003572100D6875285CE862686CA85DF
:10E2300097F0FFFFE7806006A167F10748003EC442
:10E240002302910022C697F0FFFFE78020CB410117
:10E250001743FFFF6700033BA285130611009700D9
:10E260000000E78040C52A84894455D9835721009E
:10E2700011678544BA97C2071167C1831307F7EF87
:10E28000E36FF7F89787FF1F938787009C4381CB45
:10E2900085451305210097500000E78020758355C0
:10E2A00021002285814497C0FFFFE78040E525D902
:10E2B00023100500228597A00000E78040CD85B798
:10E2C0001743FFFFE702E32F83C7950041112A8B15
:10E2D00093F7F707A384F50032852E8A328497E0FE
:10E2E000FFFFE780C0EA93170501C1876351F0067D
:10E2F000AA8A228597E0FFFFE78060E92A89568590
:10E30000832B040097C0FFFFE780C0E831E5835707
:10E31000440081440544F11793B71700A301F100AD
:10E3200003483100DE875A854A87D6862286D28501
:10E3300097F0FFFFE78060F6A167ED0748003EC455
:10E340002302810026C697F0FFFFE78020BB410132
:10E350001743FFFF6700632AA28513063100970069
:10E360000000E78040B5AA8409445DD99167CA9747
:10E37000C2071167C1831307F7EF0544E362F7FA99
:10E38000CA8597C0FFFFE78080D7014451F98149D2
:10E3900097D0FFFFE78060E063DBA9009848939780
:10E3A0001900BA9703D7070005EF2390270197D0EC
:10E3B000FFFFE78080DE1544E384A9F6268597A059
:10E3C0000000E780C0BC9787FF1F938767EC9C43E2
:10E3D0000144B9D74A8597500000E780C05889B7F3
:10E3E00085097DB71743FFFFE702831E79713E84DD
:10E3F0007C083EC82E8AB7071400A1653ECAE50511
:10E400007C08AA89080836C4428932C6BA8AC684FA
:10E410003ECC97C0FFFFE78000E3CA85080897E07D
:10E42000FFFFE78000C732460808B28597E0FFFF8C
:10E43000E78020C8A246630A09049D45080897E0C2
:10E44000FFFFE780C0BE1D4681459740FFFFE78084
:10E45000C01C63890A089145080897E0FFFFE78020
:10E4600000BD1146A68597000100E780607A10087C
:10E4700001478146D2854E8597C0FFFFE7800002A5
:10E4800045611743FFFF6700E317B685080897E06B
:10E49000FFFFE78000C21C400808D8439355C7011E
:10E4A000858912075183B205D98D97E0FFFFE78078
:10E4B00040C01C40080883C5870097E0FFFFE78045
:10E4C00040BD1C40080883C5A70097E0FFFFE78018
:10E4D00040BC1C40080883C5970097E0FFFFE78019
:10E4E00040BB85BF8945080897E0FFFFE78020B45F
:10E4F00083C704002300F50083C71400A300F500C0
:10E50000BDB71743FFFFE702A30C83C79500411176
:10E51000AA8993F7F707A384F5003285AE84328485
:10E5200097E0FFFFE780A0C693170501C187635DF1
:10E53000F0042A89032A040097C0FFFFE78080C502
:10E5400019E9835744000548F11793B71700A3074B
:10E55000F100814631A81306F100A2859700000062
:10E56000E78060951DC51C459DC783D647000148BF
:10E570000347F10093078500D2884A86A6854E8519
:10E5800097000000E78040E641011743FFFF670066
:10E59000630709487DBF1D486DBF1743FFFFE702B2
:10E5A000230365715C083EC4B7077B013EC65C0867
:10E5B0003EC883C795002A8A328593F7F707A3845C
:10E5C000F500AE8997E0FFFFE78040BA8357E1008E
:10E5D000E1C78945280097C0FFFFE780C0C6814595
:10E5E000280097E0FFFFE780C0AA97C0FFFFE78001
:10E5F000A0CC9787FF1F9387A7019C431784FF1F19
:10E60000034484AAAA843334800099C31364240089
:10E610009787FF1F938787B19C4399C31364440076
:10E620009787FF1F9387C7C69C4399C313648400D1
:10E6300083D504002800014997E0FFFFE78060A729
:10E6400083D52400280097E0FFFFE78080A683D5CC
:10E650004400280097E0FFFFE780A0A597D0FFFFC8
:10E66000E780A0AE93150501C181280097E0FFFF68
:10E67000E78020A4A285280097E0FFFFE78060A341
:10E680009C446360F902014781463000CE85528583
:10E6900097C0FFFFE78080E059611743FFFF6700E5
:10E6A00063F6DC441314490028003E9497E0FFFF12
:10E6B000E7806096834744000347540089070607B4
:10E6C000BA978607E36AF5FC835524002800814A3F
:10E6D00097E0FFFFE780E09D83454400280097E036
:10E6E000FFFFE780009B83455400280097E0FFFF71
:10E6F000E780209A8347440063C9FA00814A834730
:10E70000540063C1FA020509A5BF1C4413975A00BF
:10E710002800BA9783D50700850A97E0FFFFE780B6
:10E720004099C9BF032BC40093975A0028003E9B11
:10E7300083552B00850A97E0FFFFE780809783557C
:10E740000B00280097E0FFFFE780A0964DBF17431E
:10E75000FFFFE70283E95C4993E717005CC997A0D4
:10E760000000E78020B61743FFFF670043EA174326
:10E77000FFFFE70283E72E84814597F0FFFFE780E4
:10E78000C0E705C583570500FD172310F50009C430
:10E79000835725002310F40097000000E78060FBFA
:10E7A00001451743FFFF670083E631457DD82310FD
:10E7B0000400C5BF1743FFFFE70283E183C795004D
:10E7C00041112A8A93F7F707A384F50032852E8931
:10E7D000328497E0FFFFE780809B93170501C18794
:10E7E0006356F006AA89C145228597E0FFFFE780BE
:10E7F000A0802A8B4E85832A040097C0FFFFE78004
:10E80000609931E983574400231101000544F11751
:10E8100093B71700A300F100814403481100035788
:10E820002100D6875285CE862286CA8597F0FFFFC3
:10E83000E780A0A6A1679387170248003EC4230281
:10E84000810026C697E0FFFFE780406B4101174338
:10E85000FFFF670023DB13061100A28597F0FFFF7F
:10E86000E7806065AA8409E523110100094475B7B2
:10E87000930521005A8597000000E78080EF8357B9
:10E8800021002A84D9DB9787FF1F938767A09C43C9
:10E8900081CB85451305210097500000E7800015C6
:10E8A000835521002685314497C0FFFFE7802085EE
:10E8B0002DD523100500268597900000E780206D58
:10E8C0000144A1BF1743FFFFE70223D241112E8964
:10E8D0006C00AA8402C697F0FFFFE78000D20DC14A
:10E8E0000357050005072310E50097000000E780A7
:10E8F00040E681473E8541011743FFFF670023D172
:10E900003247954765DBCA85268597300000E7804A
:10E91000400DC147E34005FE324485474146231080
:10E92000F40083570900A685130544002311F40061
:10E9300097000100E780C02D228545BF1743FFFFE8
:10E94000E70203C983C795004111AA8A93F7F70725
:10E95000A384F5003285AE89328497E0FFFFE7801B
:10E96000008393170501C1876356F0062A8AC145C3
:10E97000228597D0FFFFE7802068AA845285032B69
:10E98000040097C0FFFFE780E08031E9835744002F
:10E99000231101008544F11793B71700A300F1007C
:10E9A00001440348110003572100DA875685D286B7
:10E9B0002686CE8597F0FFFFE780208EA16793879C
:10E9C000070248003EC42302910022C697E0FFFFE1
:10E9D000E780C05241011743FFFF6700A3C2A28531
:10E9E0001306110097F0FFFFE780E04C2A8409E549
:10E9F00023110100894475B72685930521009700EE
:10EA00000000E78060ECAA8449FD8355210022853F
:10EA100097B0FFFFE780A06E49F5014997C0FFFF5F
:10EA2000E780A077635DA900184893171900BA978B
:10EA300003D707000DEF035721002390E70097C08D
:10EA4000FFFFE7808075630625039787FF1F938785
:10EA500027849C4399C70355210097500000E78005
:10EA600080F0228597900000E78060521DBF050965
:10EA700075B795443DB705C19307F00F630FF500D7
:10EA8000C547630CF5009307F5FF05453315F50001
:10EA90004205418182800145828041657D158280E9
:10EAA000B9E91743FFFFE70243B403450603328485
:10EAB00097000000E78060FC9305803EB305B50237
:10EAC000C205C18181CD0357E402854763F8E700A1
:10EAD0001305040197E00000E78020428357E40219
:10EAE00041677D176385E700FD172317F40217437D
:10EAF000FFFF6700C3B182801743FFFFE70263ACEB
:10EB0000004283C79500444D0349140093F7F7076B
:10EB1000A384F50083470400220911673369F900D3
:10EB2000A167B347F90041112A8BAE8A63ECE70E67
:10EB3000834724001307C00EB91793F7F70F6373C9
:10EB4000F71003473400C14763EEE70E83474400E4
:10EB50001307E00793C707086371F70C8349840024
:10EB600083477400A209B3E9F900856763F7F90ADE
:10EB7000034A6400834754004E85220A336AFA0030
:10EB800097500000E780403B61C123962403834BEC
:10EB90003400137AFA00239A3403238874032399E8
:10EBA000440393890401631C090023A604022398EB
:10EBB00004024E8597E00000E78060363DA00349DF
:10EBC00024004A8597000000E78020EB2397A402E9
:10EBD000834744004E85A388F402E38D0BFCE30BCE
:10EBE00009FC97E00000E780202F97900000E78065
:10EBF000007381460146D6855A8597E0FFFFE7807E
:10EC00000058A167938797033EC423020100480080
:10EC100002C697E0FFFFE780602E41011743FFFF28
:10EC20006700A39D8544A2862686D6855A8597E0EF
:10EC3000FFFFE780C054A167938797033EC4230278
:10EC40009100F1B7BD44C5B79144F1BF1743FFFF31
:10EC5000E702039801111C08404D3EC2B7070F00A0
:10EC60003EC41C083EC62A89AE8997C0FFFFE780D4
:10EC7000A0DA585C1C5C6346B70E6394E50063E25F
:10EC8000A70E3385A740B3B7A700B305B740130657
:10EC9000803E81469D8D97000100E78080B79314E8
:10ECA0000501C180A1659385C503480097B0FFFFAA
:10ECB000E78060598145480097D0FFFFE780603DBD
:10ECC00083550404480097D0FFFFE780803E8355BA
:10ECD0002404480097D0FFFFE780A03D814589CC00
:10ECE000C167FD179305F00F6388F40026859750E0
:10ECF0000000E780E0E0AA85480097D0FFFFE780AA
:10ED0000403903554404814501CDC167FD17930582
:10ED1000F00F6307F50097500000E78060DEAA85DA
:10ED2000480097D0FFFFE780C03683456404480061
:10ED300097D0FFFFE780E03583457404480097D003
:10ED4000FFFFE7800035500001478146CE854A85A8
:10ED500097B0FFFFE780807405611743FFFF6700EE
:10ED6000638A814481B71743FFFFE702038883C7A3
:10ED7000950093F7F707A384F50097000000E7805C
:10ED800020ED1743FFFF670083881743FFFFE7026B
:10ED9000238483C795004111404D93F7F707A3845F
:10EDA000F5002A8A3285B284AE8997D0FFFFE780CA
:10EDB000003E2A8B268597D0FFFFE780403D2A89B9
:10EDC000268597D0FFFFE780603A93170B0163CA4F
:10EDD0000702E177CA97C207C183116763E3E702BD
:10EDE00093070910C207C1831307B00F637BF700B5
:10EDF00093170901C187AA8A634AF000C54763FED9
:10EE0000570141011733FFFF6700C37F97B0FFFF32
:10EE1000E780C028E31725FFD5B763080B02630618
:10EE20000902814463890A02B7077F002310640541
:10EE3000231124057CC0568597000000E780E0C3BD
:10EE40009304803EB304950239A0B7077F002320C6
:10EE500004047CC081440355240497E00000E7804B
:10EE6000A0A3A1C497C0FFFFE78000BB269593D75E
:10EE7000F44133379500AE97BA9708DC5CDCCE8559
:10EE8000528597000000E780A0DC99E0232204046B
:10EE9000A1679387B70348003EC42302010002C65E
:10EEA00097E0FFFFE7808005A9BF814701481CDC90
:10EEB000232E0403E9B71733FFFFE702037397C05C
:10EEC000FFFFE780C037E1473305F50291459750D2
:10EED0000000E78000C5E55711C59777FF1F23A302
:10EEE000A71C81473E851733FFFF670043728547A4
:10EEF0001777FF1F230AF71A82801733FFFFE702F5
:10EF0000C36E9777FF1F9387A71980433DC0835730
:10EF100004046390A70683572404639CB7043689CE
:10EF2000B28497C0FFFFE78020AF5C5C63C3B70487
:10EF30006395B7001C5C63EEA7028347640463F328
:10EF4000F400A6872303F4048347740463F3970053
:10EF5000A687A303F4048357440441677D176385A0
:10EF6000E70085072312F4043C4481C7CA8526853F
:10EF700082971733FFFF670083699777FF1F938797
:10EF800027129C43014599C303C58700828017332C
:10EF9000FFFFE70283650111B70707003EC683C77D
:10EFA0009500584D0AC493F7F7070AC8A384F500E3
:10EFB0002A89AE8411CB1C4283C707002304F700C3
:10EFC00097900000E78000342164930554022800E4
:10EFD00097B0FFFFE780202797000000E78020FA26
:10EFE000AA85280097D0FFFFE780A00A30000147DC
:10EFF0008146A6854A8597B0FFFFE780204A130423
:10F000004402480822CC230A010002CE97E0FFFF09
:10F01000E780C0EE05611733FFFF6700435F1733DA
:10F02000FFFFE702835C01117C003ECAB7070700BF
:10F030003ECC7C003ECE83C795002E84AA8493F7F5
:10F04000F707A384F500A16593855502480897B09A
:10F05000FFFFE780401F97000000E78040F2AA858D
:10F06000480897D0FFFFE780C0025008014781465B
:10F07000A285268597B0FFFFE780404205611733E0
:10F08000FFFF6700C3589777FF1F938767019C4373
:10F09000094599C303C5970082809777FF1F93871F
:10F0A00027009C43094599C303C5D7008280977701
:10F0B000FF1F9387E7FE9C43014599C303C5A70043
:10F0C00082801733FFFFE702A3500111B707080042
:10F0D0003EC683C79500404D0AC493F7F7070AC898
:10F0E000A384F5002A89AE8429C41442854703C746
:10F0F000060063E0E70A834794000946814963807C
:10F10000C702B307F740A304E400B339F00083C794
:10F1100016002305F40097900000E780A01E035717
:10F120002403058B19C76386090097D00000E78088
:10F1300000E9216493058402280097B0FFFFE7806F
:10F14000801097000000E78040F4AA85280097D03F
:10F15000FFFFE78000F497000000E78080F5AA85B4
:10F16000280097D0FFFFE780C0F2014781463000BA
:10F17000A6854A8597B0FFFFE780403213047402EA
:10F18000480822CC230A010002CE97E0FFFFE78067
:10F19000E0D605611733FFFF6700C3461733FFFF53
:10F1A000E702A34401117C003ECAB70708003ECC29
:10F1B0007C003ECE83C795002E84AA8493F7F70780
:10F1C000A384F500A16593858502480897B0FFFFE9
:10F1D000E780600797000000E78020EBAA854808D9
:10F1E00097D0FFFFE780E0EA97000000E78060EC3F
:10F1F000AA85480897D0FFFFE780A0E9500801479B
:10F200008146A285268597B0FFFFE780202905610A
:10F210001733FFFF6700A33F9777FF1F938747E8E8
:10F220009C43014599C303C5B70082801733FFFF94
:10F23000E702A33B0111B70707003EC683C795004D
:10F24000404D0AC493F7F7070AC8A384F5002A893A
:10F25000AE8405C81C42054783C707006368F706EC
:10F260000347B400630FF700A305F4009790000074
:10F27000E78040098347B400B9CF97D0FFFFE7800C
:10F2800040BE21649305B400280097B0FFFFE780DB
:10F2900080FB97000000E78060F8AA85280097D0DF
:10F2A000FFFFE78000DF014781463000A6854A85E1
:10F2B00097B0FFFFE780801E2904480822CC230A6C
:10F2C000010002CE97E0FFFFE78040C305611733DE
:10F2D000FFFF6700C33397D0FFFFE78020BF55B71C
:10F2E0001733FFFFE702633001117C003ECAB70706
:10F2F00007003ECC7C003ECE83C795002E84AA84B6
:10F3000093F7F707A384F500A165AD05480897B00A
:10F31000FFFFE78040F397000000E78020F0AA8518
:10F32000480897D0FFFFE780C0D6500801478146C4
:10F33000A285268597B0FFFFE78040160561173349
:10F34000FFFF6700C32C9777FF1F938767D59C4308
:10F35000094599C303C5C70082801733FFFFE70241
:10F36000C32801117C00AE843ECAA165B70707001F
:10F370002A843ECCD1057C0048083ECE97B0FFFFE2
:10F38000E78060EC97000000E78020FCAA85480831
:10F3900097D0FFFFE780E0CF500801478146A68560
:10F3A000228597B0FFFFE780600F05611733FFFFED
:10F3B0006700E3251733FFFFE702232383C7950088
:10F3C00093F7F707A384F50097000000E78020F982
:10F3D0001733FFFF6700A3231733FFFFE702431F25
:10F3E00083C795000329C501411193F7F707A3844B
:10F3F000F5001C4283C90700854763E63707977706
:10F40000FF1F9387E7209C432E84AA8485CF970013
:10F410000000E78080F389476306F5026304090270
:10F420008347C900638037032306390197900000A2
:10F43000E78040ED83572903898B89C797D0000067
:10F44000E780E0B72685A28597000000E78020F1DD
:10F45000A167CD0748003EC42302010002C697E021
:10F46000FFFFE780A0A941011733FFFF6700831961
:10F470009777FF1F9387C7C29C431D4599C303C558
:10F48000E70082801733FFFFE70223160111B70759
:10F4900007003EC683C79500584D0AC493F7F70787
:10F4A0000AC8A384F5002A89AE8415C71C4283C705
:10F4B000070093968701E18663C40606854663814B
:10F4C000D7068346E7006388F6002307F700979086
:10F4D0000000E78020E321649305E400280097B052
:10F4E000FFFFE78040D697000000E780A0F8AA85DC
:10F4F000280097D0FFFFE780C0B901478146300060
:10F50000A6854A8597B0FFFFE78040F93504480893
:10F5100022CC230A010002CE97E0FFFFE780009E85
:10F5200005611733FFFF6700830E1733FFFFE70204
:10F53000C30B01117C003ECAB70707003ECC7C001C
:10F540003ECE83C795002E84AA8493F7F707A38441
:10F55000F500A165B905480897B0FFFFE780A0CE88
:10F5600097000000E78000F1AA85480897D0FFFFC8
:10F57000E78020B2500801478146A285268597B0D2
:10F58000FFFFE780A0F105611733FFFF6700230845
:10F590001733FFFFE702C303AA8401441779FF1F53
:10F5A000130949B0E14997C0FFFFE78040C96344B0
:10F5B000A400014519A833053403832709003E95AB
:10F5C000835725006397970011051733FFFF6700E6
:10F5D00063030504C9BF032E8500630A0E12177367
:10F5E000FF1F1303E3CA032303006315030029432A
:10F5F0006390061203234E01631503001D436399B4
:10F6000007101733FFFFE702C3FBC689428A3E8912
:10F61000BA8AB684328BAE8B2A84B5E103554E008C
:10F6200019E501431A851733FFFF670003FDA16742
:10F63000A98F116763FBE70097000000E78080F562
:10F64000814597F0FFFFE780C0120844B70700E04C
:10F650005841F98F18455CC1B707001FF98F1CC5C9
:10F660005C4991C7610597E00000E780408BE38A21
:10F6700009FA228597900000E78060C65DB7328561
:10F6800097C00000E78040430D4349DD1C441167EB
:10F6900003D54700A167A98F63FBE700970000002F
:10F6A000E78040EF814597F0FFFFE780800C032360
:10F6B000840093164B01D1828347B3000356630045
:10F6C0008588FD8BA305F300FD777D8E558EFD7635
:10F6D000FD16B204F18E83274301C58E23127301F8
:10F6E0002313D3002304530123052301A30443015F
:10F6F000BDDF228597B0FFFFE78020CDAA850844B3
:10F70000B5D1610597D00000E780207F8DB71D43FC
:10F710001A8582801733FFFFE70283EB0569AA840D
:10F72000AE89328A0144FD5A7D1997C0FFFFE780F8
:10F73000C0A56347A40001451733FFFF670083ECB2
:10F74000D84493171400BA9703D70700631F3703F1
:10F750002390570163070A00268597900000E780F1
:10F76000A0809C449DC383D76700B3F72701639EA5
:10F770003701D288014881470147814601468145CA
:10F78000268597000000E78040E5050479BF173320
:10F79000FFFFE702E3E379711C103EC4B7070F00D7
:10F7A0003EC61C103EC883C79500AA8A328593F7CF
:10F7B000F707A384F5002E89328497D0FFFFE780F6
:10F7C000009D93170501C187635AF006AA89228517
:10F7D00097D0FFFFE780A09B2A8A4E85032B040069
:10F7E00097B0FFFFE780009B39ED835744008144C9
:10F7F0000544F11793B71700A303F1008345710087
:10F80000DA872287D2864E86280097E0FFFFE780BE
:10F81000E057014781463000CA85568597B0FFFF03
:10F82000E780C0C7A1679387F70348083ECC230A47
:10F83000810026CE97D0FFFFE780406C45611733EB
:10F84000FFFF670023DCA2851306710097E0FFFF2E
:10F85000E7806066AA84094455D1528597E0FFFF8E
:10F86000E78060D40D4459D90546D2852685970096
:10F870000000E78060EA2A8451B71733FFFFE702F0
:10F88000C3D6835507000346270041112A842E85DD
:10F8900032C62EC497E0FFFFE780E0D001C93246B0
:10F8A000A245228597000000E78000E74101173359
:10F8B000FFFF6700C3D51733FFFFE70283D083C77D
:10F8C00095004111AA8A93F7F707A384F5003285C2
:10F8D000AE89328497D0FFFFE780608B93170501D4
:10F8E000C1876357F00AC1452A8A228597C0FFFF66
:10F8F000E78080702A8D228597D0FFFFE7802089DE
:10F900002A89228597D0FFFFE7804086930705F874
:10F9100093F7F70F1307E007AA8B637BF70622859F
:10F9200097D0FFFFE78080842A8C228597D0FFFF45
:10F93000E780C083AA8C5285032B040097B0FFFF99
:10F94000E780408539E98357440023110100814451
:10F95000F11793B71700A300F10005440347110006
:10F9600083562100938784005685DA882288528640
:10F97000CE8597F0FFFFE78020A7A167E907480041
:10F980003EC42302810026C697D0FFFFE7800057C0
:10F9900041011733FFFF670043C613061100A2851C
:10F9A00097E0FFFFE7802051AA8409E523110100B9
:10F9B00009446DB7930521006A8597F0FFFFE78042
:10F9C000A0F02A8441FD835521009356C9001316E7
:10F9D000490185486688E2875E87858A5182268547
:10F9E00097000000E78060BF2A848DBF1733FFFFB8
:10F9F000E70223BD83C7950041112A8B93F7F707D0
:10FA0000A384F5003285AE89328497C0FFFFE7807A
:10FA1000007893170501C1876352F00A2A8A22856C
:10FA200097C0FFFFE780A076AA8A228597C0FFFFD4
:10FA3000E780E0752A89228597C0FFFFE780007381
:10FA4000930705F893F7F70F1307E0072A8C6377FE
:10FA5000F706228597C0FFFFE7804071AA8C2285B8
:10FA600097C0FFFFE78080702A8D5285832B0400AA
:10FA700097A0FFFFE780007239E583574400854473
:10FA80000144F11793B71700A301F10003473100B8
:10FA9000930784005A85DE882688D6865286CE85CE
:10FAA00097F0FFFFE78040948D4748003EC4230253
:10FAB000910022C697D0FFFFE780404441011733F1
:10FAC000FFFF670083B3A2851306310097E0FFFFB5
:10FAD000E780603E2A84894455D99356C90013169D
:10FAE000490185486A88E6876287858A5182D6857A
:10FAF00097000000E78060AEAA8449BF1733FFFF7C
:10FB0000E70203AD2A8981440144617A916A176B47
:10FB1000FF1F130BEB7797B0FFFFE780006863C709
:10FB2000A40022851733FFFF6700C3AD83270900B8
:10FB300093991400CE9703D5070033074501420778
:10FB400041836364570305C103270B0019C785452B
:10FB50003E8597400000E78060E98327090005049F
:10FB6000CE972390070085047DB797000000E780BB
:10FB700060A2832709000504CE972390070065D56E
:10FB8000814597F0FFFFE780C0BEF1BF1733FFFF4D
:10FB9000E70203A483C7950041112A8A93F7F70768
:10FBA000A384F50032852E89328497C0FFFFE78059
:10FBB000005E93170501C187635AF004AA89832A5E
:10FBC000040097A0FFFFE780E05C31E58357440025
:10FBD00085440144F11793B71700A301F1000348CE
:10FBE0003100D68752850147CE862686CA8597D0B2
:10FBF000FFFFE780806AA167F50748003EC4230243
:10FC0000910022C697D0FFFFE780402F41011733B4
:10FC1000FFFF6700239FA2851306310097E0FFFFD7
:10FC2000E78060292A8489445DD99767FF1F9387FD
:10FC300027669C4381CF044997B0FFFFE780E055DA
:10FC4000AA85268597400000E78040DA1305040165
:10FC500097000000E780C0EA228597800000E780D7
:10FC600000338144ADBF1733FFFFE702839583C79D
:10FC700095004111AA8A93F7F707A384F50032850E
:10FC8000AE8932842311010097C0FFFFE780205026
:10FC900093170501C1876354F0062A8AC14522855E
:10FCA00097C0FFFFE7804035AA8B5285032B0400E5
:10FCB00097A0FFFFE780004E21E983574400854469
:10FCC0000144F11793B71700A300F1000348110096
:10FCD00003572100DA875685D2862686CE8597D0AF
:10FCE000FFFFE780805BA1679387270248003EC43F
:10FCF0002302910022C697D0FFFFE7802020410118
:10FD00001733FFFF6700638FA2851306110097E08A
:10FD1000FFFFE780401A2A8489444DD99767FF1F67
:10FD20009387075798433E8901CF044997B0FFFF57
:10FD3000E780A046AA85268597400000E78000CB93
:10FD40001305040197000000E78080DB97B0FFFFF8
:10FD5000E780A04495443DD9930521005E8597F046
:10FD6000FFFFE78060B6AA8435F11C4803572100E5
:10FD700022852390E70097800000E78040218327B9
:10FD80000900A9D70355210097400000E780A0BDD6
:10FD900035BF1733FFFFE702C38283C795004111C8
:10FDA000AA8A93F7F707A384F5003285AE893284D7
:10FDB00097C0FFFFE780A03D93170501C1876351FE
:10FDC000F0062A8A228597C0FFFFE780403C2A89F7
:10FDD0005285032B040097A0FFFFE780A03B31E58D
:10FDE0008357440085440144F11793B71700A301DA
:10FDF000F10003483100DA8756854A87D286268685
:10FE0000CE8597D0FFFFE7804049A167F9074800FA
:10FE10003EC42302910022C697D0FFFFE780000E68
:10FE200041011723FFFF6700437DA28513063100C0
:10FE300097E0FFFFE78020082A8489445DD9916715
:10FE4000CA97C2071167C1831307F7EF8544E362BE
:10FE5000F7FA9767FF1F9387A7439843BE8B01CF9D
:10FE6000044997B0FFFFE7804033AA852685974075
:10FE70000000E780A0B71305040197000000E780A9
:10FE800020C897B0FFFFE780403195443DD11C4822
:10FE9000228581442390270197800000E780200F6E
:10FEA00083A70B00B9D74A8597400000E780A0AB35
:10FEB00089B71723FFFFE70243732A844105B28401
:10FEC00097000000E780C0C311C52285978000001D
:10FED000E780E00B81460146A685228597800000D9
:10FEE000E780C04E1C4C89C7DC4799C322858297A6
:10FEF0001723FFFF6700A3719767FF1F9387471AB8
:10FF00009C43014599C31385070182809767FF1FB2
:10FF100093870719884382801723FFFFE702E36C6A
:10FF20009317C600DD8DC2054111C1812A8432C6F6
:10FF300097C0FFFFE780E017324622851182937554
:10FF4000F60F97C0FFFFE780C01441011723FFFFA2
:10FF50006700E36B1723FFFFE702836779713C08B3
:10FF60003ED2B7070C003ED43C083ED683C795006E
:10FF7000AE842A8993F7F707A384F500A1659385DA
:10FF80003504481097A0FFFFE780E02BC165FD1501
:10FF90000144176AFF1F130A2A31930A400EAE89E3
:10FFA0002E8B2EC697B0FFFFE780202242059317C5
:10FFB00004014181C183B24563E9A702C167FD170E
:10FFC0006387F500481097C0FFFFE780800E501050
:10FFD00001478146A6854A8597A0FFFFE780004C30
:10FFE00045611723FFFF6700E3613307540383274D
:10FFF0000A0BBA9703D6C701630A3601638A350133
:020000040001F9
:10000000481097000000E78060F1DA85050451BFD1
:10001000B285EDBF1723FFFFE702A35A79717C0871
:100020003EC8B70711003ECA7C083ECC83C7950086
:10003000AA89328593F7F707A384F5002E8997C024
:10004000FFFFE780C01485676378F504A165AA8483
:100050008905080897A0FFFFE780E01E26859740E6
:100060000000E78060ED133415000A04A28508083B
:1000700097C0FFFFE780E001A685080897C0FFFF53
:10008000E780200325CC014781461008CA854E85AC
:1000900097A0FFFFE780804045611723FFFF6700BF
:1000A000C355B30754030327CA0ABA9703D70700F7
:1000B000631C970003D62700638065050808970036
:1000C0000000E780A0E5DE8505042EC697B0FFFF9F
:1000D000E780A0104205931704014181C183B24516
:1000E000E3E1A7FCC167FD17E38FF5F8080897C0A7
:1000F000FFFFE78000FC41BFB285F9B7C165FD1580
:100100000144176AFF1F130A2A1A930A80022E8BD2
:10011000AE8B65BF1723FFFFE702234D18418347CE
:10012000170083460700A207D58FD207D1832390FB
:10013000F50083472700034717008D45A207D98F95
:1001400091832310F60097C0FFFFE780A0E91723F3
:10015000FFFF6700C34B1723FFFFE7026347C1643C
:1001600001441769FF1F1309291493098002FD1424
:1001700097B0FFFFE78060066347A400014517239F
:10018000FFFF67002348330534038327C90A3E95E0
:1001900083570500E38597FE0504D9BF1723FFFFAA
:1001A000E70203432A8AAE89B284B68A97400000E8
:1001B000E78080D819E591473E851723FFFF670048
:1001C00063442A894E8597C00000E780E08E2A8428
:1001D000638E0A048D476DD103570500C547E31DA3
:1001E00047FD0347F9018546AD47E317D7FC834731
:1001F000450081CF4146A6855D0597F00000E78068
:10020000C09E814755D9AD4745BF130965012302FB
:10021000E500CA85268597100000E780606231C13D
:10022000A547E38B0AF82302040079B705C1835779
:100230000500E39247F94146A685190597F00000AD
:10024000E780A09A81472DD99947BDB74E85970081
:100250000000E78080F02A84954739DD13095500B6
:100260004DBF4146A68523104401231134011305D7
:10027000190097F00000E780A09922859780000080
:10028000E780A0EA81470DBF1723FFFFE702E335B0
:1002900079717C003ECCB7070A003ECE7C003ED090
:1002A00083C79500B2842E8493F7F707A384F500E3
:1002B0001306A1002A892C00268597000000E780FC
:1002C000A0E5A16528088D0597A0FFFFE780A0F7AE
:1002D00090408355A100035581008546970000009A
:1002E000E78000ECAA84AA85280897C0FFFFE78072
:1002F00040DA0356A10083558100280897000000CA
:10030000E780C0C1300801478146A2854A8597A091
:10031000FFFFE780A018854748103ED423029102D2
:1003200002D697D0FFFFE78060BD45611723FFFF2E
:100330006700E32D1723FFFFE702232B79717C0071
:100340003ECCB7070A003ECE7C003ED083C7950066
:10035000B2842E8493F7F707A384F5001306A10057
:100360002A892C00268597000000E780E0DAA16545
:1003700028088D0597A0FFFFE780E0EC90408355AB
:10038000A10003558100814697000000E78040E10D
:10039000AA84AA85280897C0FFFFE78080CF03566C
:1003A000A10083558100280897000000E78000B76E
:1003B000300801478146A2854A8597A0FFFFE78064
:1003C000E00D48102302910202D402D697D0FFFF1D
:1003D000E780C0B245611723FFFF6700432317235F
:1003E000FFFFE702832097000000E78060DB172310
:1003F000FFFF6700C3219767FF1F9387A7CA884342
:1004000082801723FFFFE702431E83572500411117
:10041000AE842A842307B10017F5FFFF1305254694
:100420006C002316F10097A0FFFFE780204991C4DC
:10043000228597800000E780E0D6FD572310F40066
:10044000130620028145130554009720FFFFE78023
:10045000C01C41011723FFFF6700631B1723FFFF29
:10046000E702031779717C003ECCB7070A003ECE45
:100470007C003ED083C79500AA89AE8493F7F70726
:100480003285A384F5001306A1002C00970000001C
:10049000E78080C803558100114497400000E78041
:1004A000A0A915C50355A100014497B00000E7803D
:1004B000A06011CD035705008357810045446318A0
:1004C000F700854597000000E780E0F301442169CB
:1004D00093053900280897A0FFFFE780C0D6A285C2
:1004E000280897C0FFFFE780C0BA0356A1008355D4
:1004F0008100280897000000E78040A230080147EB
:100500008146A6854E8597A0FFFFE78020F9481019
:100510004AD42302810202D697D0FFFFE780009ED3
:1005200045611723FFFF6700E30D1723FFFFE70275
:10053000230A9767FF1F9387A7B62A8488432E89CB
:1005400015C5035745038357C4016311F7022326DA
:10055000050223180502410597D00000E780209C82
:100560006306090097800000E78060DB814497699B
:10057000FF1F938969D3130A800297B0FFFFE780BA
:10058000C0C563C4A4049767FF1F938727BA9C4321
:1005900099C70355C40197200000E780C0BD6307D9
:1005A0000900228597800000E780C0A01306400E56
:1005B000814522859720FFFFE7802006FD57231EF7
:1005C000F4001723FFFF6700E3033385440383A789
:1005D000C90A3E95035705008357C4016317F70006
:1005E000CA8597000000E78000E2850479B71723E9
:1005F000FFFFE702E3FD83C795004111AA8993F746
:10060000F707A384F5003285AE8497C0FFFFE7802B
:1006100000B885676378F5042A8997400000E78071
:10062000A091014401CD83D70400314463882701A0
:10063000854597000000E78080EF01444E85A28643
:100640004A86A68597D0FFFFE780A09CA167938785
:10065000170448003EC42302810002C697D0FFFF62
:10066000E780C08941011723FFFF6700A3F9172323
:10067000FFFFE702E3F59767FF1F938767A28043B9
:1006800029C4014597C00000E78000218147014847
:10069000C1641CDC232E0403232004041769FF1FFC
:1006A000130989C001449309400EFD1497B0FFFF60
:1006B000E780A0B1634FA400814517F5FFFF130544
:1006C000857F97A0FFFFE780601F1723FFFF67006C
:1006D00063F3330534038327090B3E958357C50124
:1006E00063879700854597000000E78040E4050494
:1006F00075BF9357050113D78700A380F5009317A3
:100700000501C183A1832380E5002381F500A38136
:10071000A50082801723FFFFE70223ED23000500D9
:1007200083C71500A300F50083C725002301F5004A
:1007300083C73500A301F50083C745002302F500F8
:1007400083C75500A302F50083C765009305950094
:10075000A30305002303F500230405003285970059
:100760000000E78040F91723FFFF670043EA1723E3
:10077000FFFFE702E3E54111E9540DCD85CD93F983
:10078000C5FF2E842A89AA84338AA900B7EA040007
:1007900063189A020D88854411CCB7E704009C5F6A
:1007A00082972AC622866C003305390197E0000043
:1007B000E7800046268541011723FFFF670083E499
:1007C00083A78A039104829793170501C183A183AC
:1007D000A38EF4FE93570501238FF4FEA183238E8D
:1007E000A4FEA38FF4FE6DB763E6D5021723FFFFC7
:1007F000E702A3DFB28741113686BE8536C697E091
:100800000000E780E040B246410136851723FFFF34
:100810006700E3DF81463685828083870500138782
:10082000F5003D05FD8793F77708834607007D15A2
:100830008606B58FA300F5006307B7007D178347D1
:1008400017009D83DDB782801723FFFFE702E3D9FE
:10085000B7E7040083A7070932872A863A8582977B
:10086000133515001723FFFF670063DA15C18147B1
:100870008DC11723FFFFE70243D7414697E00000F1
:10088000E780003985473E851723FFFF670023D89F
:1008900081473E8582801DCD1723FFFFE702E3D409
:1008A000414681452A849720FFFFE78000D74146D3
:1008B0008145130504039720FFFFE78000D6014719
:1008C000C1672322040438C87CC805451723FFFFED
:1008D0006700E3D30145828081473DCDB5CD172325
:1008E000FFFFE70283D0B2842E891306800581457D
:1008F0002A849720FFFFE78040D2CA8524C426853A
:1009000097000000E780C0F6414681452285972088
:10091000FFFFE78080D03044A28522859700000049
:10092000E780C0F293040401A285268597000000A9
:10093000E780E0EEA6851305040297000000E7803B
:1009400000EE228597000000E78020F585473E8570
:100950001723FFFF6700A3CB3E8582801723FFFF8D
:10096000E70203C74111E9540DCD85CD93F9C5FFC9
:100970002E842A89AA84338AA900B7EA04006398DE
:1009800044030D88814411CCB7E704009C5F829733
:100990002AC622866C003305390197E00000E78003
:1009A0002027268541011723FFFF6700A3C583A7E2
:1009B0008A039104829793170501C183A183A38EB3
:1009C000F4FE93570501238FF4FEA183238EA4FE2A
:1009D000A38FF4FE6DB765CD1723FFFFE70243BF7A
:1009E000B28411E605451723FFFF6700A3C12A84DF
:1009F0002E890145EDD93C487848B3E6E700E5D6B5
:100A00009386F7FFB3B7F6007D17032A4404BA971D
:100A100034C87CC863050A06C14913050A03B389B3
:100A200049412295637D3601B2862E86A6859700C0
:100A30000000E780A0DB7C40BE9464C065B7CE8632
:100A40002E86CE8597000000E78040DAC114D2944C
:100A50004E9923220404A2879306040103C70700CA
:100A600003C607038507318FA38FE7FEE398F6FEE1
:100A70003044A285228597000000E78020DD26997A
:100A8000C1493306994063EC9900A9DCA686A68586
:100A90001305040397000000E78040D579BF814724
:100AA000B306F4003307F6000347070083C50600CA
:100AB00085072D8F2380E600E39437FF3044A2851D
:100AC000228597000000E78060D8C1145DBF014512
:100AD00082800DC11723FFFFE70223B113068005B3
:100AE00081459720FFFFE78040B305451723FFFFAF
:100AF0006700E3B101458280814749C5C1C517231D
:100B0000FFFFE70283AEFC4141462E84AA8463992D
:100B1000C70413860501A2878146C14503C70700A4
:100B200003C507038507298F3305D6000345050054
:100B30008506298FA38FE7FEE392B6FE3044A28597
:100B4000268597000000E78060D02285970000008E
:100B5000E78060F885473E851723FFFF670023ABDA
:100B6000138507031D8E814522959720FFFFE7809F
:100B7000C0AA7C40130700F813060402A29723883A
:100B8000E70251BF3E8582801723FFFFE702E3A5FE
:100B90006D712E84B284AA85901028003689970042
:100BA0000000E780A0D309EDD55725A050400C40A8
:100BB000280097000000E78040E27DD5FD14210465
:100BC000F5F42C004A8597000000E78020F3814768
:100BD00061DD3E8551611723FFFF670043A31723A3
:100BE000FFFFE70283A041112EC432C62C00054648
:100BF00097000000E78080F941011723FFFF67009D
:100C000003A11723FFFFE702439E01112A842EC68A
:100C100002C802CA02CC02CE97E00000E780402B57
:100C2000B2462A86A285080897000000E78060FB8C
:100C30001375F50F05611723FFFF6700439D172309
:100C4000FFFFE702839A7971B2872A84214623083D
:100C5000B10013051101BE853AC436C697E0000005
:100C6000E78000FBB24693059101368597000000AE
:100C7000E78060A82285141035460C089700000014
:100C8000E78020F62A84224701E921460C103A85A4
:100C900097E00000E780C0F7228545611723FFFF3A
:100CA0006700E3961723FFFFE70223947171AE8478
:100CB000AA850A85328497000000E78060BB11C9CD
:100CC0000A86A685228597000000E78020B8814724
:100CD00011E1C5473E854D611723FFFF6700239350
:100CE0001723FFFFE702638D1D712A8AB289BE8434
:100CF00035468547130511012E8CB68A3A8BC28C76
:100D0000468D2308F10097E00000E78060F01010A6
:100D10000C085285231F010097000000E780C0F8EF
:100D20002A843DEDA1476313FD089307900591E0E8
:100D3000E5473546E2851305110113990A01230899
:100D4000F1001359090197E00000E78060EC1357A8
:100D5000890093978A00D98F90080C085285231F29
:100D6000F10097000000E78020F42A8415E9A1E44F
:100D70009387FA0091831379F9003EC66313090043
:100D80004149668B8144C14B854DB247639F970CA7
:100D90006A868C0033855C0197E00000E78040E7BD
:100DA000228525611723FFFF6700E38493079004E2
:100DB000C9F0A547BDBF834701050947C14B2308BB
:100DC000F10083471105A58FA308F1009387240044
:100DD000814463E1FB04014714083386E6008C0874
:100DE000B386E400BA95DA9683C6060083C505008B
:100DF0000507AD8E2300D600E390E7FE4147639CD4
:100E0000E70490080C08528597000000E780C0E9CD
:100E100025D181A0B3069B00BA871008B305F60060
:100E200090083E9603C50600034606008507850622
:100E3000298E2380C500E39277FF998F90080C08D4
:100E40005285BE9497000000E78000E6894701477D
:100E500049D12A84B1B790083E960346060014088B
:100E6000BE962380C600850759BFB24785046387B5
:100E7000971481471808B306F70098083E97338601
:100E8000F90003470700034606008507318F2380DA
:100E9000E600E39177FF90080C0852859700000068
:100EA000E78080E05DF53546E285130511012308F2
:100EB000B10197E00000E780A0D5139704014183BA
:100EC000939784002183D98F10180C085285231F13
:100ED000F10097000000E78020DD25FD8147101814
:100EE0003387F9003E960347070003460600B30622
:100EF000FB008507318F2380E600E39277FF65A82A
:100F00001808B306F70098083E973386F9000347A0
:100F10000700034606008507318F2380E600E3E1E2
:100F200027FFCA87639E770990080C0852859700AF
:100F30000000E78060D711FD81479800B306F700F5
:100F4000900818103E973E96034707000346060098
:100F50008507318F2380E600E39177FF3546E285F0
:100F6000130511012308B10197E00000E78040CA92
:100F7000139704014183939784002183D98F10181C
:100F80000C085285231FF10097000000E780C0D1B4
:100F9000E31105EC814710183387F9003E960347AB
:100FA000070003460600B306FB008507318F238048
:100FB000E600E3E227FFC109410BC1BB814785B7CA
:100FC0009408BE9683C6060018083E972300D700F3
:100FD000850789BF638006321713FFFFE702E35DD1
:100FE00059712A84BE89B28B854735461305110293
:100FF0002E8B468C4289BA8A368A2300F10297E00A
:101000000000E780E0C010180C10228523170102B1
:1010100097000000E78040C963180512A147631FCD
:10102000FC069307900563930900E5473546DA858A
:101030001305110293140A012300F102C18097E005
:101040000000E780E0BC93178A0013D78400D98F93
:1010500090080C1022852317F10297000000E7800A
:10106000A0C47DE1639209049307FA00BD889183CF
:1010700091E0C144C207C183DE8C814A3EC6414D26
:10108000B24763E2FA0E6286B3854B01881097E09F
:101090000000E78080B54DC93D557DA093079004C1
:1010A000E39609F8A54759B7834701050947C14C9D
:1010B0002300F10283471105B3C7F900A300F10231
:1010C00093872900814963E1FC04814618103306A7
:1010D000D7008C083387D900B69556970347070089
:1010E00083C5050085062D8F2300E600E390D7FE1B
:1010F00041476390E70690080C1022859700000096
:10110000E78080BA35D189A0B3863A01BA8710103A
:10111000B305F60090083E9603C506000346060098
:1011200085078506298E2380C500E39297FF3387C4
:10113000EC4090080C102285BA9997000000E780D7
:10114000A0B68947014741D165611713FFFF6700CA
:10115000834A90083E96034606001410BE962380EC
:10116000C600850779B7B247850A93990A01939D0E
:101170008A0093D909016391570F85473546DA856F
:10118000130511022300F10293D9890097E00000B2
:10119000E78000A8B3ED3D0190000C1022852317D5
:1011A000B10397000000E78020B059FD8147A68970
:1011B00063EA970626860C084A8597E00000E780D8
:1011C00020A581471810B306F700100898083E972D
:1011D0003E9603470700034606008507318F2380AC
:1011E000E600E3E197FE639FA90590080C102285B5
:1011F00097000000E78040AB21F981479810B306C3
:10120000F700900818183E973E96034707000346DC
:1012100006008507318F2380E600E391A7FF41098F
:10122000C10CB9BD18089000B306F7003E9633878D
:10123000FC0003470700034606008507318F238023
:10124000E600B5B798084E97034707001C10CE97E5
:101250002380E700850941BF85473546DA851305B8
:1012600011022300F10293D9890097E00000E78082
:10127000209AB3ED3D0190000C1022852317B10395
:1012800097000000E78040A2E31005EC81471808B2
:101290009000B306F7003E963387FC000347070033
:1012A000034606008507318F2380E600E391A7FF00
:1012B00041460C084A8597E00000E7806095814729
:1012C0001810B306F700100898083E973E9603479B
:1012D0000700034606008507318F2380E600E3916F
:1012E000A7FF90080C10228597000000E780C09BA4
:1012F0001DD599BD7D5582801713FFFFE702E32EB0
:1013000001112A842E8593055100328902C002C240
:1013100002C402C69304740097F0FFFFE780A03D6B
:101320001D46A6851305910097E00000E780408EDA
:1013300010088A854A8597000000E780E09619ED3D
:1013400093071400180883C60700034607008507A3
:101350000507B18EA38FD7FEE397F4FE056117133F
:10136000FFFF6700C32A1713FFFFE70263262E84DF
:101370008C414111AA89838715003289914463D336
:101380000700A1449757FF1F938787289C43A1C755
:10139000C1CA8D472310F10083C725004A85230168
:1013A000F10083C73500A301F10083C74500230284
:1013B000F10083C75500A302F10083C765009305C0
:1013C0009100A30301002303F1002304010097F01F
:1013D000FFFFE78040320C404A860A8597F0FFFF06
:1013E000E78080330328040083564400A6881D0844
:1013F00081470147E51642868A854E8597000000A1
:10140000E780408E2A8919E5A685228597B0FFFFDF
:10141000E780E0C14A8541011713FFFF6700831E83
:101420004A860A8597F0FFFFE780002F6DB71713F4
:10143000FFFFE702E3192E848C414111AA898387BB
:1014400015003289914463D30700A1449757FF1FC9
:101450009387071C9C43A1C7C1C68D472310F10089
:1014600083C725004A852301F10083C73500A30106
:10147000F10083C745002302F10083C75500A30292
:10148000F10083C7650093059100A30301002303C6
:10149000F1002304010097F0FFFFE780C0250C4016
:1014A0004A860A8597F0FFFFE780002783564400AD
:1014B000032804008A85858EC2061D08C182231276
:1014C000D400A68881470147E51642864E859700DD
:1014D0000000E78060B041011713FFFF670083122F
:1014E0004A860A8597F0FFFFE78000234DBF171358
:1014F000FFFFE702830FB335B000011185052A898C
:101500001315F601336515012308B1009305110188
:1015100036843AC632C03EC442C297F0FFFFE7802D
:10152000801DA2471248425593D68700230BF10035
:101530009305910193578800A30AD100A30BF100F2
:10154000230C010197F0FFFFE780E01A32470246C3
:1015500003280400B337E000835644009207914407
:1015600011C2A1444A85A68842860C0897F0FFFF65
:10157000E78040772A8919E5A685228597B0FFFF85
:10158000E780E0AA4A8505611713FFFF670023087B
:101590001713FFFFE702C30301113EC68647B335A9
:1015A000B0008505AA891315F6015D8D2308B100E9
:1015B0009305110136843A89B28442C446C297F039
:1015C000FFFFE78040132248924816459357880052
:1015D000A30AF1009305910193D78800230B010121
:1015E000A30BF100230C110197F0FFFFE780A0107F
:1015F0003247104083564400B337E0009207032877
:101600000900914891C0A1480C084E859700000040
:10161000E780809CAA8401E9835544004A8597B0FD
:10162000FFFFE780C0A0268505611713FFFF670055
:1016300063FDAA959307F00F17170100130747A33F
:101640006317B50013C5F7FF1375F50F8280050505
:101650008346F5FFB58FBA9783C70700D5B7035701
:10166000450014419307F00F17160100130646A01A
:10167000369742074183139506014181631BE500BC
:10168000AD8FB29703C50700130515F31335150089
:101690008280850603C5F6FFA98FB29783C707002E
:1016A000D9BF1713FFFFE70243F4B28736842E86B3
:1016B000BA86AA853E85BA8497F0FFFFE78060521C
:1016C000634F0500228597E00000E78060802A864E
:1016D000A686A285268597F0FFFFE7808050171326
:1016E000FFFF6700C3F21713FFFFE70263EE5D71B0
:1016F0002A8BAE8A17150100130505952C00B284BC
:10170000368ABA893E8997F0FFFFE780C04F2A8466
:101710005DE134104146DA85280097F0FFFFE7804D
:10172000404C2A8449E98547A303F100A6C29307E8
:1017300071002408BEC4A68685470D462C182810C3
:1017400002DC02DED6C0BEC697F0FFFFE780004491
:101750002A8435E183477102A6860D4693F7F70781
:101760002300FA00C1473EDE2C188947281026DCEA
:10177000A303F10097F0FFFFE78040412A8405EDC5
:101780004146A6854E8597D00000E78060488D478A
:10179000A6860D462C182810A303F10097F0FFFF32
:1017A000E780C03E2A8401E94146A6854A8597D054
:1017B0000000E780E045228561611713FFFF6700A5
:1017C00063E41713FFFFE70243E297F700009387F4
:1017D00027EF984383C7470079712A89AE8417158C
:1017E00001001305E5860C083AC42306F10097F0C2
:1017F000FFFFE78040412A8405ED14104146CA8569
:10180000080897F0FFFFE780C03D2A8415E114081F
:1018100015462C00081097F0FFFFE780803C2A84D3
:1018200001E921462C08268597D00000E780403E3C
:10183000228545611713FFFF670063DD1713FFFF64
:10184000E702A3DA97F70000938787E79C4779714F
:10185000AA842E8417150100130505800C083EC6C6
:1018600097F0FFFFE780203A0DE914104146A68566
:10187000080897F0FFFFE780C03605E1140811461D
:101880006C00081097F0FFFFE780A03519E583474B
:10189000F10193F7F7032300F40045611713FFFFED
:1018A0006700E3D61713FFFFE70223D43688A14869
:1018B00081470147E54697F0FFFFE780A0421713F5
:1018C000FFFF6700C3D41713FFFFE70203D2368878
:1018D000A14881470147E54697F0FFFFE780C06FC9
:1018E0001713FFFF6700A3D21713FFFFE702E3CF31
:1018F00001112A842E850C0832C697F0FFFFE7807D
:10190000803009ED32479706010093866673100810
:10191000C145228597000000E780E0D805611713D4
:10192000FFFF6700C3CE1713FFFFE70203CC41118F
:10193000C1472EC032C48A8509463EC23EC697F0D2
:10194000FFFFE780A02441011713FFFF670023CCAE
:101950001713FFFFE70263C94111AE861306100992
:10196000AA850A8502C002C202C402C697F0FFFF20
:10197000E780202741011713FFFF670043C91713B2
:10198000FFFFE70283C63287970601009386466D04
:101990002E869305000297000000E780C0D0171341
:1019A000FFFF6700C3C61713FFFFE70203C4797187
:1019B000C1472ACC2ED032D42C080D4628003ECE6A
:1019C0003ED23ED602C402C602C802CA97F0FFFF4A
:1019D000E780C01B45611713FFFF670043C3171360
:1019E000FFFFE70283C00111AA842E8417050100BE
:1019F000130585678A8597F0FFFFE780C02015E50E
:101A000014084146A6850A8597F0FFFFE780601D10
:101A100009ED8347E1010347F101A207D98FCA0706
:101A2000C9836177D98F2310F40005611713FFFF75
:101A30006700E3BD15CD1713FFFFE70203BB974710
:101A4000FF1F9387A76A90439745FF1F9385456AB9
:101A50001745FF1F1305856597D00000E78000C577
:101A60001745FF1F130585641713FFFF670023BA8F
:101A70001745FF1F1305856382808DCD1713FFFF68
:101A8000E702A3B69747FF1F938747669443011168
:101A90002E840A869745FF1F9385856597D00000A1
:101AA000E78040C60A850294014505611713FFFFD0
:101AB0006700E3B57D5582801713FFFFE702E3B2AD
:101AC00097D00000E78080D19747FF1F23A0A7622F
:101AD00017F5FFFF1305E5C997B00000E780C07454
:101AE0001713FFFF6700A3B21747FF1F13074762D3
:101AF0009317150008433E95FD572310F50082808B
:101B00001713FFFFE70263AE2A84084009E51713A5
:101B1000FFFF6700C3AF1C4158401CC06313E500C2
:101B20005CC08347550023200500F99BA302F50004
:101B300097A0FFFFE780207CC9BF1713FFFFE702D4
:101B400023A99747FF1F9387A75E98432A8411CB49
:101B50008347350093F7070289C703550500894578
:101B600002971305440197B00000E780403B83557E
:101B700004000355E40097300000E780A00C4858AB
:101B800019C597A0FFFFE7800077232A04021305F9
:101B9000840397000000E780E0F68144B149979004
:101BA000FFFFE780C06D63CBA4028347340023208E
:101BB000040493F727FCA301F40000489790FFFF6B
:101BC000E780E06C13161500814522859710FFFF12
:101BD000E780A0A41713FFFF6700C3A2B3873403F5
:101BE0000329040385043E994A8597000000E78095
:101BF00060F12304090065B78347350093F70702B6
:101C000099E3014582808357E500E39CB7FEC167F5
:101C1000FD176316F60005458280054599A8171340
:101C2000FFFFE702839C93170601C187B2842A84D1
:101C300001496359F002835705009DCB0145636755
:101C4000F600034584003E953325A6001375F50F75
:101C50000DA01C4813171900BA9783D70700E38E0D
:101C600097FA05099790FFFFE7806062E343A9FEBA
:101C700001451713FFFF670083991713FFFFE70262
:101C80002395AE89AA849790FFFFE78000562A84A7
:101C900097D0FFFFE780A02EAA8601471306840194
:101CA00097050000938585E41745FF1F13058546BA
:101CB0009790FFFFE780801C2A8925C98C44130474
:101CC000C50022859E0593F5050897A0FFFFE780D4
:101CD000403CCC4083877400E18163DD070493E5D9
:101CE0000508228597A0FFFFE780A03A0D4693855F
:101CF0004400228597A0FFFFE780C03683D504000B
:101D0000228597A0FFFFE780E03D83D52400228550
:101D100097A0FFFFE780003D03D6490083A5090097
:101D2000228597A0FFFFE780E0334A851713FFFF66
:101D30006700438D93F5F5076DB71713FFFFE702B3
:101D4000C38A01112A84328532C697A0FFFFE7803B
:101D5000E0279780FFFFE780603483570400174730
:101D6000FF1F130767543246231BF100930700F847
:101D7000A30DF1001C471843231AA1008983858B0A
:101D8000B307F740B28548083ECE231C0100230D5F
:101D9000010097000000E78080EE05611713FFFF48
:101DA0006700E3861713FFFFE702838200410145C6
:101DB0003DC49304C40026853289AE8997A0FFFFF5
:101DC000E780C02495452A8A2685035B040197A0F5
:101DD000FFFFE7802021268597A0FFFFE780603E78
:101DE0008D45AA8A268597A0FFFFE780A01F26853C
:101DF00097A0FFFFE780E03C5C48420A135A0A01C3
:101E0000D2975CC423186401814763983A01460560
:101E10004D81330625419337160013F5F70F17034D
:101E2000FFFF6700237E1703FFFFE70283798969BD
:101E30002A8BAE8B328AB68A81440144314CFD191B
:101E40009790FFFFE780A04363CDA4009790FFFF2A
:101E5000E780E045018D33B5AA001703FFFF670057
:101E6000C3793389840383270B003E9963170A00E3
:101E70008347890085043E94E1B703560A00DE8556
:101E80004A8533F6C90097000000E780E0F16DD184
:101E90000545E1B71703FFFFE702237501112A8407
:101EA0007C000355E5003ECAB70707003ECC7C0026
:101EB0003ECE97200000E78020082A898545480803
:101EC00097A0FFFFE78020399945480897A0FFFFBA
:101ED000E780E015AA844A8597200000E780A008E3
:101EE0002380A4009747FF1F9387073C9C434166CC
:101EF000130606F09396870113D78701558F93D663
:101F00008700F18E558FA207B706FF00F58FD98F96
:101F100011462C00138514003EC497D00000E780C2
:101F200020CF5008A3820400894522859700000035
:101F3000E780E0E019C9AA851305840397A0FFFF95
:101F4000E780E0313C4085073CC005611703FFFF97
:101F50006700E36B1703FFFFE70223699790FFFF1A
:101F6000E780E0342A8405049790FFFFE780203360
:101F70003305A402F14791453305F502972000008F
:101F8000E78020BA11E565551703FFFF6700236856
:101F90009747FF1F23A6A7189790FFFFE7802031E0
:101FA0002A8405049790FFFFE780602F3305A40281
:101FB0008945060597200000E780A0B669D59747B8
:101FC000FF1F23A7A7149790FFFFE780402E2A84C6
:101FD00005049790FFFFE780802C3304A402974705
:101FE000FF1F239987129790FFFFE780402C2A84D8
:101FF0009790FFFFE780A02A930714003385A7027C
:102000009747FF1F2399A71097070100938787C958
:102010001747FF1F2324F7100145BDB71703FFFF24
:10202000E702035BAA842E8901449749FF1F938925
:10203000A927130A80069790FFFFE7804026634791
:10204000A40001451703FFFF6700C35B330544038A
:1020500083A709024A86A6853E9597000000E7807F
:10206000E0B919E10504C1BF0545E9BF1703FFFF4A
:10207000E7022355AA8A2E8BB28B368C3A8A81448A
:1020800001448149974CFF1F938C0C22130D80064D
:102090009790FFFFE780A02063C9A40011E0854965
:1020A0004E851703FFFF670043553389A40383A7B9
:1020B0000C025E86D6853E994A8597000000E7802F
:1020C000E0B31DC19790FFFFE780601E0544636D7C
:1020D0004501D2866286DA85130509039700000060
:1020E000E780A0D411C1854985045DB71703FFFFC0
:1020F000E702034EC16441112A8901449749FF1F39
:102100009389891A130A8006FD1436C632C42EC27A
:102110009790FFFFE780A01892452246B246634899
:10212000A400014541011703FFFF6700A34D3305DC
:10213000440383A709023E9509C683473500C18B36
:102140009DC791C68347350093F707028DC3630689
:1021500099008357E500639C27010357050001CBD5
:1021600063E7E50083478500BA97E3CDF5FA0504F8
:1021700069BF1703FFFFE702A345C1642A89014431
:102180009749FF1F93894912130A8006FD149790FF
:10219000FFFFE780C0106346A4001703FFFF67003E
:1021A00063463305440383A709023E958357E50040
:1021B000638A9700630499006396270197000000E3
:1021C000E780E0970504E1B71703FFFFE702E33E6E
:1021D00089692A8AAE8A328BB68B8144174CFF1FDD
:1021E000130C8C0C930C8006314DFD199790FFFF5A
:1021F000E780E00A63C6A4001703FFFF6700A33F60
:102200003389940383270C028355CA015A863E9969
:102210004A8597000000E780609E31C1814D15A07E
:102220003384AD038327090303D60B00D68533F629
:10223000C9003E94228597000000E780E0B609E9D6
:10224000850D9790FFFFE7808003E3CBADFC01A8ED
:10225000228597000000E780E08A230404008504BB
:1022600071B71703FFFFE702C3354169AA8A014A24
:10227000174BFF1F130B4B037D19C14B054C979058
:10228000FFFFE780C0016346AA001703FFFF670056
:10229000C33693098006B3073A0383290B02BE991C
:1022A00083D7E900638E270163842A01639A57016B
:1022B00003A4890301E84E8597000000E780C0BDB4
:1022C000050A75BF83570401639977099304C40015
:1022D000268597A0FFFFE78060D385452A8D268558
:1022E000835C040197A0FFFFE780C0CF268597A0FD
:1022F000FFFFE780A0E762056185635905048D450E
:10230000268597A0FFFFE780E0CD8945268597A029
:10231000FFFFE78020CD8945268597A0FFFFE78056
:1023200060CC8545268597A0FFFFE780E0CC8347FA
:102330000500094793F7F707639AE7009945268553
:1023400097A0FFFFE78040CBA30285014848337D7B
:102350002D01231894016A9548C40040A1BF1703BA
:10236000FFFFE702832837E404008327041D8297D8
:102370009747FF1F83C747E01715FF1F1305456BDE
:10238000A300F5008327441C82978327841C814681
:102390001306F00F8145014582971703FFFF670081
:1023A00003271747FF1F130727CD18439745FF1F24
:1023B00083C585DC9747FF1F938787DA83468703AA
:1023C000034697036397D5009747FF1F2386C7DA15
:1023D000828083C587010347A7036317B600974729
:1023E000FF1F238BE7D8828003C687016317C700CE
:1023F0009747FF1F2382D7D8828083C687011307A0
:1024000050026319D700930760021747FF1F230587
:10241000F7D6828083C68701130660026315D60053
:1024200093077002DDB783C7870155BF9747FF1F2A
:10243000938707D3D44B0947638DE6081703FFFF43
:10244000E702A31A1749FF1F1309C9CE3E84834729
:102450000900918B9DCFB7E4040083A7041D8297E8
:1024600083A7441C1745FF1F130545CD829783A7FB
:10247000841C81461746FF1F034646CE8145014511
:10248000829721C583470900ED9B1747FF1F230350
:10249000F7CA8347040093F7F70F85CB9147174797
:1024A000FF1F2329F7CC97000000E78080EB9700FF
:1024B0000000E78040EFB7E70400BC4F414691457C
:1024C0001745FF1F034545CA82971703FFFF6700A3
:1024D000031482801703FFFFE70223118D47411188
:1024E0006306F504C5476308F50285476310F502E6
:1024F0009747FF1F2384A7C8B7E70400BC4B930589
:1025000000101745FF1F034525C682974101170399
:10251000FFFF6700C30F85471747FF1F2300F7C65C
:10252000B7E70400BC4B93050020E1BF9747FF1FAE
:10253000938707C3D44B1147638DE600B7E70400C8
:1025400083A7071D8297B7E70400BC4B93050004DF
:102550004DBF05491747FF1F232E27C183C707001B
:1025600032C62E8493F7F70FD5D3B7E4040083A7C0
:10257000041D7D141374F40F8297E37689FCB24531
:10258000994703C61500E3F0C7FCFC44090617454C
:10259000FF1F1305E5BE8297BC4893050008174549
:1025A000FF1F034565BC829779BF1703FFFFE70252
:1025B000C3031747FF1F1307A7BA4047184B1C4018
:1025C0009746FF1F23A4F6BA6316E4001747FF1FC0
:1025D0002320F7BA130584FE9790FFFFE78000AA37
:1025E000035564FF9780FFFFE780807297A0FFFF8D
:1025F000E78060D01703FFFF670063011703FFFF49
:10260000E702A3FE9747FF1F938787B5D84BDC47A8
:1026100089C797000000E78080F985471747FF1FAB
:10262000232AF7B49747FF1F938707A59C43930579
:1026300000021745FF1F034525B383C787031747CC
:10264000FF1F230BF7B2B7E70400BC4B82971703B9
:10265000FFFF6700C3FB9747FF1F23A5A7B082803A
:102660001703FFFFE702C3F637E404007C4CA145E3
:102670001745FF1F034545AF82977C48A145174585
:10268000FF1F034565AE9744FF1F938464AD829797
:10269000DC4489EB97000000E78080D91703FFFF37
:1026A000670043F603D567FF9780FFFFE78040662A
:1026B000AA896DD1D84891476310F7027C4C9145A7
:1026C0001745FF1F034545AA82977C48914517454A
:1026D000FF1F034565A9829703A9490103D4090196
:1026E0008947B7E904001747FF1F2325F7A883A7E9
:1026F000091D21044204829783C784011715FF1F17
:102700001305053361191717FF1FA303F73283A7BA
:10271000491C418082979747FF1F238107A683A703
:10272000C91C814609469375F40F4A85829711E9C1
:102730009747FF1F83C7C7B489C79710FF1FE7805C
:10274000209CB7E70400BC4F2146A1451745FF1F59
:10275000034585A1829799B71703FFFFE702E3E8D6
:1027600093F7052001112E8481CF97000000E780A8
:1027700020E91345042005611703FFFF670023E9E3
:1027800093F70510A9CF9744FF1F9384649DDC48FD
:1027900097000000E78020C11747FF1F1307C78D70
:1027A000184383C78401034787036318F700DC4499
:1027B00089C797000000E78080DF85471747FF1F24
:1027C000232AF79AB7E70400BC4B9305000217458C
:1027D000FF1F0345659982971345041069BF93F75E
:1027E0000508BDC79747FF1F83C79799E917194683
:1027F0009745FF1F9385E5981305D10093F4F70FD4
:102800001749FF1F0349C99797C00000E780404060
:1028100093970401C1831747FF1F1307E796231DF2
:10282000F100231CF1009747FF1F938767933ACE6F
:102830003ACAD8432306010009CBDC43931589012A
:1028400054080D46E185680082971345040825B7B2
:1028500093F72500A5C39747FF1F93876790D84B31
:1028600089476306F7029747FF1F83C7A78C13F7B3
:10287000270011EF918B99CFB7E70400BC4F1306E7
:10288000000A89451745FF1F0345058E82971345AA
:102890002400D5B59737FF1F9387077E9C4383C7D6
:1028A00087031747FF1F2309F78C97000000E78075
:1028B00060DBF1BF93F7050281CB97000000E78052
:1028C00060DA1345040245BD93F7850081CB97007C
:1028D0000000E780E0D21345840071BD93F7150036
:1028E00081CB97000000E780A0B41345140061B5C8
:1028F00093F7450081CB97000000E78060B3134554
:10290000440095BD93F7050495C39747FF1F83C700
:10291000278591CB97000000E780A0A49147174737
:10292000FF1F2329F78413450404B1B593F705016C
:102930000145E38207E49747FF1F93876782D84BDF
:1029400091476310F7049737FF1F9387A77E9C4337
:1029500013D727008583D98F858B91E7B7E70400CC
:1029600083A7071D8297B7E70400FC4F91451735F1
:10297000FF1F0345657F829785471737FF1F232B6E
:10298000F77E13450401C5BB9747FF1F238AA78E17
:1029900082801703FFFFE70243C59737FF1F23A776
:1029A000077C9737FF1F23A5077C85471734FF1F38
:1029B0001304846C1737FF1F232EF77A1C4083C73C
:1029C00087031737FF1F2309F77A9790FFFFE780E8
:1029D000409329C59717FF1F23A0A7061C40170582
:1029E00000001305A5D783C787031737FF1F2305EB
:1029F000F7781717FF1FA30DF7029737FF1FA38163
:102A00000776B7E7040083A7070882979737FF1F69
:102A1000238CA7741703FFFF670063BFB7C7898EB6
:102A2000938767ED1717FF1F2328F70045BF173758
:102A3000FF1F0347E772795555E79737FF1F9387C5
:102A4000277203C7170005079736FF1FA38AE67092
:102A500003C717008D463377D7029736FF1FA38130
:102A6000E67083C617001737FF1F1307E760184388
:102A700093F6F60FA9EE834787031737FF1F230D41
:102A8000F76E85471737FF1F230CF76C9737FF1F2B
:102A90009387476A9C430145998BA9E71703FFFF7A
:102AA000E702A3B437E404007C48C1451735FF1F93
:102AB0000345856B82973C4885451735FF1F0345C5
:102AC000A56A829701451703FFFF670043B483C7D8
:102AD000170085466395F6008347970379BF8347C0
:102AE000A70361BF82809737FF1F83C76767A1CFA6
:102AF0001703FFFFE70263AF37E404009737FF1FB8
:102B0000238007667C4885451735FF1F0345C5654B
:102B100082977C4C91451735FF1F0345E5648297EA
:102B20007C4891451735FF1F0345056482973C4853
:102B3000C1451735FF1F03452563829701451703DC
:102B4000FFFF6700C3AC795582801703FFFFE702E0
:102B5000C3A92A84035565FF9780FFFFE780401BC8
:102B60009737FF1F9387C75FD847BE841DEF9790A5
:102B7000FFFFE78080779C48232004009DEB973778
:102B8000FF1F23A7875E9737FF1F23A1875EB7E745
:102B90000400BC4B89451735FF1F0345E55C829750
:102BA00001451703FFFF670083A6630A87001843E8
:102BB00075BF80C39737FF1F23AC875AC9BF7955AC
:102BC000CDB71703FFFFE70243A29737FF1F938795
:102BD000676B88432326050023240500510597A031
:102BE0000000E780C0331703FFFF670043A217030D
:102BF000FFFFE702839F1734FF1F1304A4681C40E4
